:020000000C945E
:10000200E60D0C9400000C9400000C9400000C947B
:1000120000000C9400000C9400000C94E1570C9426
:1000220000000C9400000C942E150C9400000C940B
:1000320000000C9400000C9400000C9400000C943E
:10004200F9140C9400000C94B9550C9400000C9413
:10005200D5550C9400000C9400000C9400000C94F4
:1000620000000C9400000C9400000C9400000C940E
:1000720000000C9400000C943E560C9400000C946A
:1000820080570C9400000C94000000000100020054
:10009200040008001000200040008000000100025F
:1000A200000400080010002000400080000102044B
:1000B2000810204080000C03780B80100000100311
:1000C200780B821F00001A03780B810300002203C1
:1000D200780B010402002C03790B0106020036039F
:1000E2007B0B018000004203820B020F00004A03D7
:1000F2007C0B020F000052037E0B020FD0125A0338
:10010200800B011000006403D00B011000006E038D
:10011200810B000100007603840B010801008003BB
:10012200850B030801008E03860B0307000096036C
:100132009C0B017F3F00A0039B0B01050000AA035B
:10014200870B03040000B2039A0B01641E00BE0376
:10015200880B00010000CA03890B00010000D603CE
:10016200990B01020000E2038A0B00010000F00378
:100172008B0B020F0000FC038D0B020FE70306043A
:10018200CF0B016300006404D10B011000006E0468
:10019200D20B0102020012048F0B030801001804A3
:1001A200900B030800001E04910B030800002404B6
:1001B200920B030800002A04930B0308000030048A
:1001C200940B030800003604950B030800003C045E
:1001D2009D0B040A2E004404A70B040A2E004C04B3
:1001E200B10B040A2E005404BB0B040A2E005C045B
:1001F200C50B040A2E0000000000FF000000760478
:1002020000027E040404840408078A040C058A049C
:100212008C06900480099804100BA004500CAA04C8
:100222004003B204140ABC041808C4041C010000F0
:10023200000200002A0054007F00800E5631008127
:100242000E563200820E5633000031000B00312070
:10025200414243000032000B003220444546000078
:1002620033000B003320474849000043000C004391
:1002720000000000000034000B0034204A4B4C0008
:100282000035000B0035204D4E4F000036000B00AC
:100292003620505152000030000B003020202E201A
:1002A2002C0037000B003720535455000038000B48
:1002B200003820565758000039000B003920595A8F
:1002C2002F00003D000A0043520000000000706F42
:1002D2007274696F6E696572656E00002E666F6C6E
:1002E20067650000506F7274696F6E656E20736986
:1002F200636865726E0050726F64756B74200000E3
:10030200537061727465202000005F4944005F529F
:1003120073323332494400005F526F746174650076
:100322005F54617374656E5800005F546173746545
:100332006E5900005F44656661756C744B657900A7
:100342002A436F64653000002A436F646531000000
:100352002A436F64653200002A4D61784D6F6475DF
:100362006C005F4572774D6F64756C002A54697337
:10037200636845005F4D795465726D4E72005F4D42
:1003820061737465725465726D7300005F454D6FE1
:10039200646500005F4543726564577472005F5282
:1003A20073304D6F646500005F5634756E643500BE
:1003B2005F50756C736554696D6500005F41736BC6
:1003C20043726564697400005F53656E64446562DC
:1003D200697400005F4372656469744D6F646500FF
:1003E2005F4372656469744D6173746572002A5467
:1003F20061626C655374617274002A5461626C6547
:10040200456E64002A4669727374426F6E50000032
:100412002A4A6F6231002A4A6F6232002A4A6F62A8
:1004220033002A4A6F6234002A4A6F6235002A4A30
:100432006F6236002A4A6F6237005F4572726F72CE
:1004420031005F4572726F7232005F4572726F7275
:1004520033005F4572726F7234005F4572726F7261
:1004620035005F4672656967616265005F4B6F6D5B
:100472006D61000054617374657200004C69745AB6
:1004820000004C656974540050756C73000054612F
:1004920073742030000073657269656C6C0073655B
:1004A2007269656C2032000054617374203200005E
:1004B20054617374207061720000466F6C676554FA
:1004C20000005377697463680000436865662D4DC8
:1004D200656E75004B206C697374656E00004B206D
:1004E2006C6F65736368656E00004B2064727563A0
:1004F2006B656E0054206C697374656E0000542045
:100502006C6F65736368656E000054206472756376
:100512006B656E0053797374656D0000506F727471
:10052200696F6E004B726564697465004B72656435
:100532002E436C7200006D616E2E506F7274696F83
:100542006E00546573740000506172616D6574656C
:10055200720050726F64756B746500004B656C6C51
:100562006E65720056656E74696C650030CC04313C
:10057200D60432E00433EC0434F604350005360CBC
:1005820005461605411E05432605442E054A380533
:1005920000000000301605374405394A0538540575
:1005A200425E05456605000000004572726F7200EA
:1005B2004F70742E0000496D70756C7300005469A1
:1005C2006D656F757400AC05E60B00030000B205A3
:1005D200E90B00030000B805E70B00030000C005AB
:1005E200E80B001400002E202C30414243314445D8
:1005F2004632474849334A4B4C344D4E4F355051A1
:1006020052365354553756575838595A2F390500D0
:10061200C11100000300D90B00000300C111030047
:10062200170E0300D90B00000500E00800000A00C5
:10063200C1110A00170E0A00D90B0A00C1110A00E3
:10064200170E2800D90B000000000F00E003EF0393
:1006520000780F78E07BEF7BF7BD1F00E007FF0714
:1006620000F81FF8E0FFFFFF00000000000000009C
:100672000000000000000000000000000000000078
:100682000000000000000000070018C02020202009
:100692004D904D904010401048904710202020204F
:1006A20018C007000000000007001FC03FE03FE045
:1006B200727072707FF07FF0777078F03FE03FE009
:1006C2001FC007000000000000000000000018C06A
:1006D2003DE03FE03FE03FE01FC00F800700020027
:1006E2000000000000000000000000000000020006
:1006F20007000F801FC03FE01FC00F8007000200ED
:1007020000000000000000000000000007000F8051
:100712000F800F8037607FF07FF07FF0326007003C
:100722000F80000000000000000000000200020034
:1007320007000F801FC03FE03FE03FE01AC0070004
:100742000F80000000000000000000000000000018
:100752000000000006000F000F000600000000006D
:100762000000000000000000FFF0FFF0FFF0FFF0CB
:10077200FFF0FFF0F9F0F0F0F0F0F9F0FFF0FFF029
:10078200FFF0FFF0FFF0FFF00000000000000000AB
:1007920006000900108010801080108009000600F9
:1007A2000000000000000000FFF0FFF0FFF0FFF08B
:1007B200F9F0F6F0EF70EF70EF70EF70F6F0F9F01D
:1007C200FFF0FFF0FFF0FFF000000000000001E08A
:1007D20000601EA0332061806180618033001E00B2
:1007E20000000000000000000000000007800CC0B4
:1007F2001860186018600CC00780030003000FC067
:10080200030003000000000002000300038003C095
:1008120002C002C00280020002000E001E001E0082
:100822000C000000000000000C000E000B0009800C
:100832000CC00E400B4009C038C07840784031C02F
:1008420003C003C001800000000002000200272054
:100852001FC018C030607070306018C01FC02720E1
:10086200020002000000000000000000100018005A
:100872001C001E001F001F801F001E001C0018000D
:100882001000000000000000000000000080018055
:10089200038007800F801F800F8007800380018004
:1008A20000800000000000000000020007000F802E
:1008B2001FC0020002000200020002001FC00F80DF
:1008C2000700020000000000000019801980198052
:1008D20019801980198019801980198019800000E7
:1008E200198019800000000000001FE036C066C0B9
:1008F20066C066C036C01EC006C006C006C006C0BE
:1009020006C006C00000000000001F8030C030009A
:1009120030001F8030C030C01F8000C000C030C017
:100922001F80000000000000000000000000000026
:1009320000000000000000000000000000001FE0B6
:100942001FE01FE000000000020007000F801FC030
:100952000200020002000200020002001FC00F801B
:10096200070002001FC000000000020007000F8005
:100972001FC0020002000200020002000200020088
:10098200020002000000000000000200020002005B
:100992000200020002000200020002001FC00F80DB
:1009A200070002000000000000000000000000003C
:1009B2000100018001C03FE001C001800100000090
:1009C2000000000000000000000000000000000025
:1009D20004000C001C003FE01C000C00040000009E
:1009E2000000000000000000000000000000000005
:1009F20000000000000000004000400040004000F5
:100A020040007FE000000000000000000000000045
:100A1200088018C038E07FF038E018C00880000075
:100A220000000000000000000000000000000000C4
:100A32000000020007000F801FC03FE07FF00000AF
:100A420000000000000000000000000000000000A4
:100A520000007FF03FE01FC00F800700020000008F
:100A62000000000000000000000000000000000084
:100A72000000000000000000000000000000000074
:100A82000000000000000000060006000F000F003A
:100A92000F000F000F000600060006000000000015
:100AA2000600060000000000000000001980198006
:100AB2001980198000000000000000000000000002
:100AC20000000000000000000000066006600660F2
:100AD2003FF00CC00CC0198019807FC03300330076
:100AE2003300000000000000060006001F803FC027
:100AF200360036003F801FC006C006C03FC01F80C0
:100B0200060006000000000000000000001038305F
:100B1200387038E001C0038007000E001C0038E086
:100B220070E060E000000000000007000D80198006
:100B320019801B000E001E003E00336033C031805E
:100B42003BC01E60000000000E000E000E000600FA
:100B520006000C0000000000000000000000000081
:100B62000000000000000000038006000E000C00E0
:100B72001C001C001C001C001C001C000C000E00B1
:100B820006000380000000001C00060007000300AE
:100B92000380038003800380038003800300070037
:100BA20006001C000000000000000000000036C02B
:100BB20036C01F800F003FC00F001F8036C036C0F6
:100BC2000000000000000000000000000000000023
:100BD2000600060006003FC03FC0060006000600F1
:100BE2000000000000000000000000000000000003
:100BF20000000000000000000000000000000E00E5
:100C02000E000E0006000C000000000000000000B4
:100C12000000000000003FC03FC0000000000000D4
:100C220000000000000000000000000000000000C2
:100C320000000000000000000000000000000E00A4
:100C42000E000E00000000000000001000300070D6
:100C520000E001C0038007000E001C003800700095
:100C620060000000000000000F803FE03060607014
:100C720060F061B0633066306C3078307030306074
:100C82003FE00F8000000000030007001F001F006C
:100C9200030003000300030003000300030003003A
:100CA2001FE01FE0000000001FC03FE070706030D6
:100CB200607000E001C0038007000E001C003800D5
:100CC2007FF07FF0000000001FC03FE070706030D6
:100CD200003000700FE00FC00060003060307070B4
:100CE2003FE01FC00000000001C003C007C00EC0EB
:100CF2001CC038C070C060C07FF07FF000C000C070
:100D020000C000C0000000007FF07FF060006000C3
:100D120060007FC03FE000700030003060307070D3
:100D22003FE01FC00000000003C007C00E001C000F
:100D3200380030007FC07FE07070603060307070CB
:100D42003FE01FC0000000007FF07FF00060006005
:100D520000C000C0018001800300030006000600FD
:100D62000C000C00000000000F801FC038E0306053
:100D7200306038E01FC03FE07070603060307070EB
:100D82003FE01FC0000000001FC03FE070706030F5
:100D9200603070703FF01FF0006000E001C003801F
:100DA2001F001E0000000000000000000000000004
:100DB2000E000E000E000000000000000E000E00EB
:100DC2000E00000000000000000000000000000013
:100DD2000E000E000E000000000000000E000E00CB
:100DE2000E00060006000C0000C001C003800700D0
:100DF2000E001C00380038001C000E0007000380A3
:100E020001C000C00000000000000000000000005F
:100E120000003FE03FE0000000003FE03FE0000054
:100E22000000000000000000300038001C000E002E
:100E32000700038001C001C0038007000E001C00F0
:100E420038003000000000001F803FC070E060608A
:100E520060E001C0038007000600060006000000F3
:100E620006000600000000001FC03FE0306067B0CF
:100E72006FB06DB06DB06DB06DB06FE067C07000F7
:100E82003FC00FC000000000060006000F000F0068
:100E92000F0019801980198030C03FC03FC06060C8
:100EA20060606060000000007F007F8061C060C001
:100EB20060C061C07F807FC060E06060606060E0B1
:100EC2007FC07F80000000000F801FC038E03060CC
:100ED200600060006000600060006000306038E028
:100EE2001FC00F80000000007F007F8061C060C0D3
:100EF20060606060606060606060606060C061C02F
:100F02007F807F00000000007FE07FE060006000E3
:100F1200600060007F807F80600060006000600091
:100F22007FE07FE0000000007FE07FE06000600083
:100F3200600060007F807F80600060006000600071
:100F420060006000000000000FC01FE03860300049
:100F52006000600063E063E06060606030603860A1
:100F62001FE00FE000000000606060606060606091
:100F7200606060607FE07FE0606060606060606031
:100F820060606060000000001F801F800600060095
:100F9200060006000600060006000600060006001F
:100FA2001F801F8000000000006000600060006081
:100FB200006000600060006000606060606070C09F
:100FC2003FC01F8000000000606060E061C063807D
:100FD20067006E007C007C006E006700638061C069
:100FE20060E060600000000060006000600060007F
:100FF20060006000600060006000600060006000EF
:101002007FE07FE000000000606070E070E079E067
:1010120079E06F606F60666066606060606060600B
:101022006060606000000000606070607060786006
:101032006C606C60666066606360636061E060E083
:1010420060E06060000000000F001F8039C030C007
:1010520060606060606060606060606030C039C025
:101062001F800F00000000007F807FC060E0606092
:101072006060606060E07FC07F8060006000600050
:1010820060006000000000000F001F8039C030C007
:1010920060606060606060606060636033C039C0DF
:1010A2001FE00F60000000007F807FC060E0606092
:1010B2006060606060E07FC07F806700638061C0C5
:1010C20060E06060000000001F803FC070E0606070
:1010D200600070003F801FC000E00060606070E050
:1010E2003FC01F80000000003FC03FC00600060056
:1010F20006000600060006000600060006000600BE
:1011020006000600000000006060606060606060D1
:10111200606060606060606060606060606030C09D
:101122003FC01F800000000060606060606030C0EF
:1011320030C030C01980198019800F000F000F00D5
:101142000600060000000000606060606060606091
:10115200606060606060666066606F6079E070E049
:1011620070E06060000000006060606030C030C00D
:1011720019800F00060006000F00198030C030C031
:1011820060606060000000006060606030C030C07D
:10119200198019800F000F000600060006000600E5
:1011A20006000600000000007FE07FE000C000C0F3
:1011B20001800300060006000C0018003000300019
:1011C2007FE07FE000000000666066600F000F00B5
:1011D2000F0019801980198030C03FC03FC0606085
:1011E20060606060000000006F605FA039C030C0C6
:1011F20060606060606060606060606030C039C084
:101202001F800F00000000006060606000006060EE
:10121200606060606060606060606060606030C09C
:101222003FC01F80000000001F801F8018001800B0
:1012320018001800180018001800180018001800EC
:101242001F801F800000000000000000000000005E
:10125200000000000000000000000000000000008C
:10126200000000007FF07FF0000007000700070089
:10127200060006000300000000000000000000005D
:10128200000000000000000000000000000000005C
:1012920000001FC03FE000601FE03FE06060606050
:1012A2007FE03FE00000000060006000600060003E
:1012B20060006F807FC070E060606060606060E0CE
:1012C2007FC07F80000000000000000000000000DE
:1012D20000001F803FC070606000600060007060AE
:1012E2003FC01F80000000000060006000600060DE
:1012F20000601F603FE071E060606060606070608D
:101302003FE01FE0000000000000000000000000BD
:1013120000001F803FC070607FE07FC060007000EF
:101322003FC01F800000000007800F801C001800D3
:10133200180018007F007F0018001800180018001D
:10134200180018000000000000000000000000006B
:1013520000001FE03FE07060606070E03FE01F60EF
:10136200006000E03FC03F806000600060006000FD
:1013720060006F007F8071C060C060C060C060C0EC
:1013820060C060C00000000000000000060006000F
:1013920000000E000E000600060006000600060011
:1013A2001F801F80000000000000000001800180FB
:1013B20000000380038001800180018001800180A0
:1013C200018019801F800F00300030003000300093
:1013D20030003180338037003E003E0037003380DA
:1013E20031C030C0000000000E000E0006000600F2
:1013F20006000600060006000600060006000600BB
:101402001F801F800000000000000000000000009C
:10141200000059807FC07FE066606660666066603B
:10142200666066600000000000000000000000002E
:1014320000003F803FC030E030603060306030609C
:10144200306030600000000000000000000000007A
:1014520000001F803FC070E060606060606070E00C
:101462003FC01F80000000000000000000000000DC
:1014720000007F807FC060E06060606070E07FC0DD
:101482006F8060006000600000000000000000004B
:1014920000001FE03FE070606060606070E03FE06D
:1014A2001F6000600060006000000000000000009B
:1014B200000037C03FE038603000300030003000BC
:1014C20030003000000000000000000000000000BA
:1014D20000003F007F8060007F003F80018001802C
:1014E2007F803F0000000000000018001800180074
:1014F20018007F007F00180018001800180018005C
:101502001F800F80000000000000000000000000AB
:10151200000060606060606060606060606070E0F9
:101522003FE01F600000000000000000000000001B
:1015320000006060606030C030C0198019800F0008
:101542000F00060000000000000000000000000084
:101552000000666066606660666066606F603FC0DD
:1015620039C01080000000000000000000000000F0
:10157200000060C071C03B801F000E001F003B8056
:1015820071C060C000000000000000000000000008
:10159200000030C030C0198019800F000F00060013
:1015A20006000C000C001800000000000000000003
:1015B20000007FC07F80030006000C00180030008E
:1015C2007FC07FC0000000000000000060600000DB
:1015D20000001FC03FE000601FE03FE0606060600D
:1015E2007FE03FE0000000000000000060600000BB
:1015F20000001F803FC070E060606060606070E06B
:101602003FC01F800000000000000000606000007A
:10161200000060606060606060606060606070E0F8
:101622003FE01F600000000000003F007F8060C0BC
:1016320060C061C0678067C060E06060606060E059
:1016420067C067800000000000000000000000008A
:1016520006000F00198030C0606060607FE07FE0AC
:1016620000000000000000000000F8000000FF0081
:101672000000FF0000007F80001E0F80007FE7C097
:10168200007FFFE0003FFFE00007FFC00001FFC056
:101692000001FF800001FF0003FFFE0007FFFC00C6
:1016A20007FFF00003FFF00003FFFE00001FFFC072
:1016B20001FFFFF001FFFFF801FFFFF8007FFFF8D5
:1016C2000007FE00003FFF00007FFF80007FFF80D9
:1016D200007FC100001FE000001FF000001FF000AB
:1016E200000FE0000007C0000007C0000007C000B4
:1016F2000007800000030000000300000002000059
:1017020000000000000000000000E00000000000F7
:101712000003900000000000000E1800000000000E
:10172200003808000000000000C01800000000009F
:1017320003807000000000000C01C0000001800660
:10174200300700000003C00F401C00000006E01D2F
:10175200C0700000000C3039C1C0000000181871C0
:10176200C7180000001C0CE1DC7C0000000E07C35F
:10177200F1C4000000070386070600000003800E84
:101782001C0200000001C01C300300000000E03811
:1017920018010080000070700FC183C0000038E0A3
:1017A20003E08E6006001DC00020FC200F000F80A9
:1017B20000307030198007000010003030C0000087
:1017C200001800E060600000000803806030000044
:1017D200000C0E003018000000043800180C000045
:1017E2000006E0000C060000000380000603000073
:1017F2000000000003018000000000000180C00022
:101802000000000000C0C000000000000060C00036
:10181200000000000030C000000000000030C000E6
:10182200000000000030C000000000000030C000D6
:10183200000000000030C000000000000030C000C6
:10184200000000000030C000000000000030C000B6
:10185200000000000030C000000000000030E00086
:10186200000000000030700000000000003018008E
:101872000000000000300C000000000000300400F6
:1018820000000000003FFC0000000000003FFC00E0
:1018920054696E792062616400507772552000426B
:1018A2004F7574200057646F672000454570726F52
:1018B2006D20006C7C736368656E203F0058006E7B
:1018C20065696E006A61003E3E006B65696E204B81
:1018D200726564697400546573740020204B653A24
:1018E200002020496E3A0043616C6962726174693A
:1018F2006F6E004F4B00567320312E353500546FFA
:1019020074616C20002D2D2D2D006B65696E2045B4
:101912004570726F6D006E6F20546F756368004979
:101922006E697469616C697A656400494420004596
:10193200452036346B0066616C73636865722054AF
:10194200697363682000546973636820766F6E2040
:101952004B20004665686C6572200056656E74699E
:101962006C20616B7469760054696D656F757400E3
:10197200435349204E722000436F646520006B651B
:10198200696E204B72656469740066616C7363688A
:1019920065722054697363680054697363682076C2
:1019A2006F6E204B005831393931303000504C5570
:1019B20020203A00436F6465203A005469736368DB
:1019C200203A004D42005053004D31004F31005338
:1019D200500043500044590062757379004D500025
:1019E2002067657370657272740025640000533F4E
:1019F20000004162726563686E756E67004B656CCC
:101A02006C6E65722000546F74616C004D6F64756A
:101A12006C2000202000433F0073656300496D7015
:101A220000504C553A20005370617274653A2000A0
:101A32005072313A20005072323A200046756E637D
:101A420074203A20005479703A20003A20563A2005
:101A520020302B2030003A003A20544F3A20003AEE
:101A62002050733A200053703A004B204D6F64654A
:101A7200204A6F62204A6F62466C616773004B2096
:101A8200004D6F646520004A6F62202000562020BE
:101A9200204572722050676C20496D7020544F00AF
:101AA2005620005061757365004B656C6C6E6572F3
:101AB2003A004D49004D42004D43004D50004D4CFF
:101AC2000074657374202E2E004F4E004B2300428B
:101AD2005300422100424600542300544F00495211
:101AE200004D5A00425100425200435300565300E7
:101AF200564300494C00426600002530325800250A
:101B020030345800253664002533642E2530326483
:101B12000025356400256400253264002533640005
:101B2200444400004B230054230042450043450037
:101B3200424100445300434200235022415343494F
:101B4200492D492F4F222C22312E3030222C323077
:101B520030382D30312D30313B0023482245636F20
:101B6200222C22312E3030222C323030382D30319E
:101B72002D30313B0023532245636F222C22312E1C
:101B82003030222C323030382D30312D30313B0084
:101B9200504F00504632333B5055002564002B30E5
:101BA2002B303B0025640025303258002E303000A7
:101BB2004F4E0000206E616E6F0001002D4E414EAF
:101BC20000000100A10EBC1B0000F894EE27ECBB44
:101BD200F1E0F5BFE5BFE0936C00F8E1F1BDE1BDD6
:101BE2008DE0A2E0BB27ED938A95E9F780E090E1D2
:101BF200A0E0B1E0ED930197E9F7E4ECFBE1859118
:101C02009591009761F0A591B59105901590BF014E
:101C1200F00105900D920197E1F7FB01F0CFEFEF94
:101C2200EDBFE0E1EEBFC0E0D3E00C949B160A9951
:101C320002C0E1E00895E0E00895089508951A933E
:101C420010E0E0E0E093E807E0EEEA930E94096129
:101C5200E43551F4E2EEEA930E940961E093E80769
:101C6200A091E807A130C8F41F5F0E9485660E9418
:101C72002A74A091E807A03011F4153008F001C0D1
:101C8200E3CF0E948A660E948F660E946D5DE2E940
:101C9200F8E10E949466A895FECF19910895E88113
:101CA200E03011F01D9801C01D9A27C40E94986669
:101CB2000E9498660E949D660E94A2660E94A76684
:101CC20008950E94AB660E94B16619F50E94B7663C
:101CD2000E9498660E94BC66E1E2EA930E949866BE
:101CE2000E9498660E94C5660E94A2660E94BC6617
:101CF2000E94C8660E9498660E94C5660E94CB66D2
:101D02000E94D0660E9498660E944746EBE9F0E086
:101D120022C00E94D3660E9498660E94BC66E1E2DD
:101D2200EA930E9498660E9498660E94D8660E9472
:101D3200A2660E94BC660E94C8660E9498660E94C3
:101D4200D8660E94CB660E94D0660E9498660E9466
:101D52004746E1EFFFEFFA93EA930E94DB660E94A7
:101D6200E0660E9498660E94474608951A93E0E052
:101D7200E0930B0410E0133020F50E94E3663196E5
:101D8200049000920A040E94E966E2E3F0E00E94F5
:101D9200A57434960E94EC66EEE2F0E0FA93EA93C0
:101DA200E3E2F0E0FA93EA930E94E366E491EA93B5
:101DB2000E94E36632960E94F3660E9447461F5FC6
:101DC200DACFE0910B04E0930A040E94F66646C360
:101DD2000E942D770E94925D0E94FA66ECE00E94BA
:101DE2000067E8E7F0E0FA93EA930E948F66E3E285
:101DF200F0E00E940667E1E2EA93EFEBF8E10E946D
:101E0200F3660E944746EBE00E9400670E948F66DD
:101E12000E948F66EEE6F0E00E940667E091F10B09
:101E2200F091F20BE491EA93E091F10BF091F20B55
:101E320031960E9458750E94F3660E94474631E02F
:101E42000E940D670E94106711F03F5FF9CF0E9458
:101E52001E67301718F4E0E0E093BB050E941E678E
:101E620011E00E9426670E94106711F0143008F0FA
:101E720023C00E948F660E94E966E0E2F0E00E94C1
:101E8200A5743496FA93EA930E942967EAE1F0E096
:101E92000E942E670E943167E491EA930E942667AE
:101EA2000E94316731960E9458750E94F3660E9423
:101EB20047460F5F1F5FD5CF0E94F6660E943477B8
:101EC2002EC327970E942D7730E00E94FA660E9467
:101ED200AB6610E0133010F00C94B70F00E0043042
:101EE20010F00C94B50F0E943D6732960490009258
:101EF2000A04E0E0E0930B04FE013496FA93EA93BD
:101F02000E943D673496FA93EA930E948C63EB85B4
:101F1200E03039F4AD81A13210F4E0E0ED83E0E08D
:101F2200EE83A02FB0E0E8E2F0E00E94A5743296C2
:101F3200FA93EA930E94E966E0E2F0E00E94A57457
:101F4200B096FA93EA93E4E2F0E00E9406670E94F8
:101F52003D67E491EA930E949866FE013F960E94D3
:101F620043673F5F0F5FBBCF1F5FB4CF0E940E601E
:101F72004DC40E942B770E9498660E9498660E9428
:101F82006D5D3091D5070E9447670E94FA6610E0A6
:101F9200E091790B1E1700F500E0E091780B0E1727
:101FA200C8F40E94546799F00E945B670E946767B9
:101FB200519FF0010E9471670E947667E1E4FBE0A5
:101FC2000E9443674E2F3A934A930E9436193F5F0D
:101FD2000F5FE3CF1F5FDCCF0E94F6660E9432776D
:101FE200DAC122970E942B77E9E0F7E0EE83FF83C4
:101FF20040E0443190F4AE81BF8111960E94846723
:102002001396EFEFEC93AE81BF81EC93EE81FF81EB
:102012003496EE83FF834F5FECCF0E944767309187
:10202200D5070E94896710E0E091790B1E17D0F561
:1020320000E0E091780B0E1798F50E94546769F161
:10204200A091510BE0E8EA23E03819F40E945B67A3
:1020520006C0E7E0E0930B04E8E0E0930A040E9484
:1020620067670E9490670E94E9660E94A574339692
:10207200FA93EA930E947667E1E4FBE00E944367E9
:102082004E2FA091D507E32F0E949367EA0FFB1F03
:1020920043833A934A930E9436193F5F0F5FC9CF39
:1020A2001F5FC2CFE0910B04E0930A040E94B16665
:1020B20041F50E949A6771F40E94B7660E94986681
:1020C2000E94BC66EFE7EA930E9498660E949866B7
:1020D2000E9447460E94B7660E94A2660E94BC66A2
:1020E2000E94C8660E9498660E94C5660E94CB66DE
:1020F2000E94D0660E9498660E944746EBE9F0E093
:1021020027C00E949A6771F40E94D3660E94986663
:102112000E94BC66EFE7EA930E9498660E94986666
:102122000E9447460E94D3660E94A2660E94BC6635
:102132000E94C8660E9498660E94D8660E94CB667A
:102142000E94D0660E9498660E944746E1EFFFEF28
:10215200FA93EA930E94DB660E94E0660E94986608
:102162000E9447460E940E600E943C2E0E943277D7
:10217200289608950E948967E0E0E0930B04ECE062
:10218200E0930A040E948F660E949F67E1E2EA934D
:10219200E1ECF8E10E94F3660E944746EAE0E09330
:1021A2000A04E2E5F0E0FA93EA930E949F67EDE306
:1021B200EA93E6ECF8E10E94F3660E9447460E9429
:1021C2000E6008951A93A981A23019F40E949A67A9
:1021D20009F024C00E94AC670E94AF67BF01E98189
:1021E2000E94B6670E94C0671E2FEFE00E94006740
:1021F200E7E8F0E0FA93EA93EB810E94B667329641
:102202000E94C9670E94D067FA93EA93EFE7EA93C4
:10221200E9ECF8E10E94F3660E9447461FC10E9462
:10222200925DE0E0E0930B04A881A13051F40E949A
:102232008A660E94D3670E946D5DECECF8E10E9411
:1022420094660E949A6769F4E2E0EA93BBDFE8E3EE
:10225200F2E00E94D867EAE3F2E00E94D8670E94A7
:1022620028602FDD4AC1E8810E94B667FA93EA939B
:102272000E94DD670E94AF67FA93EA930E94C45DF1
:10228200E881EA939FDF39C11A930A93EC81EA93BA
:10229200EADF1BE90E94E0670E94AF67BF01EC81A1
:1022A2000E94B6670E94C0670E2FAC81A43019F459
:1022B2000E949A6709F009C012E8AA81BB811B96A5
:1022C200E0E0EC93EC81EA937DDF0E945B67EC81B6
:1022D2000E94E367FF93EF930E94D367EE810E940F
:1022E200B66731960E94E9670E942E67FA93EA93D5
:1022F200EC85E058EA930E949866ED85FE850E947F
:102302004367AF91BF91EC93EC810E94B667FA9359
:10231200EA93EE81F0E00E94AF67FA93EA930E949B
:1023220028601981088125960895E7C01A930A93B7
:10233200E091790BAFE70E94AF740E2F11270E9434
:1023420098660E9498660E949D661A930A930E945C
:10235200A7660E948A660E948A660E946D5DEC8171
:10236200FD810E949466AA81BB81A030E0E8BE078D
:1023720031F0EA81FB81FA93EA930E94DF430E94E3
:1023820085660E94BD450E9498661A930A930E9430
:10239200286019810881269608950E941F63E0E053
:1023A200E0930A04E0930A040E94B16619F4E1E999
:1023B200F0E002C0E1EFFFEFFA93EA93E0E6F0E02B
:1023C2000E940667EEE1F0E0FA93EA930E94E0666B
:1023D2000E9498660E94474608951A9311E00E944F
:1023E2003D1B0E94EC670E94F167B8970CF414E061
:1023F2000E9498660E94D0670E94F767E9810E9456
:10240200FD670E9409680E94F7670E940D680E949A
:102412001268E981EA930E94E41AE983AAEDB6E020
:102422000E94AC670E9416683B9754F0AAEDB6E092
:102432000E94AC670E9416680E941D68E9E40BC006
:10244200AAE9B6E00E94AC670E9416680E94216861
:102452000E94C743E3E7EA930E94FF5C1881229639
:1024620008950E9498660E9498660E946D5DE8ED4C
:10247200F8E10E9494660E9498660E9426680E9473
:102482009D66ECE3F0E00E942B680E9498660E9431
:102492008A660E946D5DE09116060E942E68EDED3F
:1024A200F8E10E949466E091E707EA930E94F14303
:1024B2000E9498660E943068E0912D060E942E6864
:1024C2000E9498660E94D3670E946D5DE091440667
:1024D2000E942E68E3EEF8E10E949466E0910B06FA
:1024E200EA930E94F1430895E881E064E7B9369ADD
:1024F200349BFECF349AE4B1F5B121960895E88178
:10250200F981AA81BB81AE17BF071CF4EA1BFB0B42
:1025120006C0A881B981EA81FB81EA1BFB0B2496E4
:10252200089528970E942D77EFE0E09361000E94C2
:10253200B16611F4E1E001C0E4E4E093620085E8F1
:102542008A95F1F7E5E0E093610085E88A95F1F775
:102552000E943368E0936A05F0936B05E09176057B
:10256200F0917705E0936805F0936905E1E0EA935D
:10257200BBDFE0937605F0937705EFE0E09361002F
:102582000E94B16611F4E2E001C0E8E0E09362006B
:1025920085E88A95F1F7EAE0E093610085E88A959B
:1025A200F1F70E943868E0936605F0936705E091C1
:1025B2007405F0917505E0936405F0936505E0E01C
:1025C200EA9392DFE0937405F09375050E943868F0
:1025D200A0916605B0916705EA0FFB1FA0917405F3
:1025E200B09175050E943D688F010E943368A091E9
:1025F2006A05B0916B05EA0FFB1FA0917605B091B9
:1026020077050E943D689F01E0916605F09167059C
:102612000E944468FF93EF930E9438680E944468C6
:10262200AF91BF91EA0FFB1FFF93EF93E091740507
:10263200F09175050E944468AF91BF91EA0FFB1FAC
:10264200E0937005F0937105E0916A05F0916B05D6
:102652000E944A68FF93EF930E9433680E944A687F
:10266200AF91BF91EA0FFB1FFF93EF93E0917605C5
:10267200F09177050E944A68AF91BF91EA0FFB1F64
:10268200E0937205F0937305A0917005B091710506
:10269200E4E1F0E00E9477740E2EA0917205B091F1
:1026A2007305E4E1F0E00E947774E02919F00E94DA
:1026B200F747ACC000936C0510936D0520936E052F
:1026C20030936F05A0915F05A23328F4E0915F0576
:1026D200EF5FE0935F050E945068989724F40E9490
:1026E200556898970CF00EC0A0915F05AA3019F4B6
:1026F200E1E0E0935C05A0915F05A83219F4E2E005
:10270200E0935C050E945068AB35E0E0BE0734F010
:102712000E945568AB35E0E0BE070CF477C0E0914B
:102722006205EF5FE09362050E945A680E9450685A
:102732000E945F680E9466680E946B68E0EAF0E0AF
:1027420060E070E00E94AA747F936F93FF93EF930F
:102752000E9470680F010E945A68DF01F001EA1BB3
:10276200FB0BAF91BF918F919F910E9475680E9460
:1027720066680E947A680E9455680E945F680E949B
:102782007F68E0E8F0E060E070E00E94AA747F9366
:102792006F93FF93EF930E9488680F010E947A68FB
:1027A200DF01F001EA1BFB0BAF91BF918F919F916B
:1027B2000E9475680E947F680E94257764F4AC814C
:1027C200BD818E819F81A038E0E0BE07E0E08E07E8
:1027D200E0E09E070CF01AC0E885F985E093540505
:1027E200F0935505EC81FD81E0935605F093570572
:1027F200E0915405F0915505FA93EA93E09156055C
:10280200F0915705FA93EA930E947F470E9434772A
:102812002C9608950E94925DEAE0F0E00E94C9675A
:102822000E94865DE9EEF8E10E949466E4E1EA9393
:102832000E9458430E948D68E4E1EA930E94584343
:10284200A0916205A13010F0A895FACF0E94986677
:102852000E9493680E94865D0E949868EBE10E9444
:102862009E68A0916205AF3110F4A895FACF0E943C
:10287200A268A0E0B0E00E9483750E9498660E9460
:1028820093680E94AB680E9498660E94B2680E9498
:10289200865D0E945A680E941D68A0916205AE3151
:1028A20010F0A895FACF0E9498680E94B7680E941B
:1028B200865DEAE10E949E68A0916205AF3110F444
:1028C200A895FACF0E94A268A2E0B0E00E948375A8
:1028D2000E94B7680E94AB680E94B2680E94B26808
:1028E2000E94865D0E9470680E941D68A091620528
:1028F200AE3110F0A895FACFE2E0E0930804E6E4E6
:10290200F0E00E94F3660E94865DE8E1EA930E948D
:10291200FF5CE1E0E0930804A0916205AF3110F49E
:10292200A895FACF0E94BC68A4E0B0E00E9483752B
:10293200E6E4F0E00E94F366E8E1F0E00E94C96795
:102942000E94A7660E94C5680E94CA680E94865DAE
:102952000E947A680E941D68A0916205AE3110F053
:10296200A895FACF0E9498680E94B268EFE5F0E05D
:102972000E94CF68E9E10E949E68A0916205AF3192
:1029820010F4A895FACF0E94BC68A6E0B0E00E94BD
:1029920083750E94B268EFE5F0E0FA93EA93E8E10A
:1029A200F0E00E9406670E94A766E8E2F0E00E945B
:1029B200EC660E94865D0E9488680E941D68A09154
:1029C2006205AE3110F0A895FACFE2E8F0E00E947D
:1029D200D3680E94865DE5EFF8E10E9494660E944A
:1029E200D668A8950E94D668A8950E94925D08951F
:1029F2000E94DC68E2EBE2BF7894A9E1BBE00E94AE
:102A0200EB680E9441478DDD0E947D1BE2B3EF78A7
:102A12000E2EA091CB07B091CC07E7E0F0E0AE27F5
:102A2200BF27EA23FB230E945374E029E2BB0E94E2
:102A3200375CE091F90BEF5FE093F90BA091F90B92
:102A4200AE3149F4A0910504E3E8EA27E0930504D6
:102A5200E0E0E093F90B199112C00E94DC680A933E
:102A6200E3E8E4BDE0B1E295E7700E2F11271A9377
:102A72000A930E94541B0E94115C09911991E991D9
:102A8200EFBFF991E991B991A991999189917991C0
:102A92006991F990199009901895E8EFFFEFE0938A
:102AA200020CF093030C0E94925D0E941F630E942D
:102AB2008A660E943068E8EFF8E10E9494660E94FC
:102AC2002E630E94F1680E942A7408950E94C05BDE
:102AD2000E94FF400E94771808951A93A8950E94B9
:102AE2006B45E13011F00C94BF15E091C105E15046
:102AF2001E2FA091C005A13021F40E94F668E0309B
:102B020009F40BC00E94FD68BF010E94FD68E081CC
:102B1200E260DB01EC930E940369A091C005A23040
:102B220011F0A43089F40E94F668E093D6050E9461
:102B3200F668E03029F00E94FD68E081E27009F455
:102B420003C01A930E940869A091C005A33019F42A
:102B52001A930E943821A091C005A53029F4E09172
:102B6200C105EA930E946821A091C005A73031F403
:102B7200E091C105E093D6050E947A43E0910504F5
:102B8200E07839F1E0910504EF77E09305040E94C3
:102B92004C60E0910504E07131F0E0910504E270CF
:102BA200EA930E94675CA091E807A13330F0E4EE5B
:102BB200EA930E9409611E2F01C010E0103808F04C
:102BC20010E0E091F70BE11711F41093E70710936F
:102BD200F70B7CDF4EC01A930E94925D0E948A66B8
:102BE2000E9498660E946D5D10E00E94FA660E9443
:102BF20098660E94D0670E941268E091D707E03081
:102C020049F4E0E0F9E10E9494660E940C690E9496
:102C1200B1431E5FA091D707A130F0F0E091D70732
:102C2200E150EA930E949830A0916A0BAD3229F4E8
:102C32000E9417690E941D7779F00E9424690E9400
:102C420029690E940D680E9412680E9417690E94F9
:102C52005C750E94B1431E5FE091D707EF5FE0937E
:102C6200D707163020F4A091D707AB3008F001C087
:102C7200BECF199108951A930E94925DE981E030C6
:102C820019F4E0E0E093D507A981A230A9F410E09D
:102C9200A091D507A13010F0163008F00DC0E091D8
:102CA200D507E150E093D5070E942D6919F40E94DF
:102CB2003B6909F01F5FECCF0E94FA6610E00E94A8
:102CC20098660E94D0670E941268A091D507A0342E
:102CD20000F50E942D6919F40E943B69B9F0E09158
:102CE200D5070E94FD670E9409680E9412680E942F
:102CF20046690E941D68E8E7EA930E94FF5C0E9411
:102D02004B690E944F690E94B1431E5F0E945A693B
:102D120007C0E7E0F9E10E9494660E945A691E5FCB
:102D2200163020F4A091D507A23408F001C0C7CF15
:102D32000C94B71A14B7E0E0E4BFE5BFE0936D006E
:102D4200E0936C00EBBBEFEFEABBE0E0E8BBE7BB74
:102D5200E5BBEFEFE4BBE0E7E2BBE1BBE0E3E3B9F5
:102D6200E8EBE2B9E0E0E0936200E0936100E09317
:102D72006500EFE0E0936400E0E0E0BFE7E0E3BF7E
:102D8200E2EBE2BFE0E0E1BFEFBDEEBDEDBDECBDC9
:102D9200E7BDE6BDEBBDEABDE9BDE8BDE093790064
:102DA200E0937800E3E0E5BDE3E8E4BDE0E0E3BD05
:102DB200E0938B00EAE0E0938A00E0E0E093890090
:102DC200E0938800E0938100E0938000E2E1E093E9
:102DD2008700E4E3E0938600E0E0E0938500E0937F
:102DE2008400E0938300E0938200E0936A00E0E3D2
:102DF200EABFE0E4E9BFE8BFE1E4E7BFE0E0E09377
:102E02007D00EBB9E8EDEAB9E6E0E0939500E0E099
:102E1200E0939000E3E3E9B9E0E0E0939B00E8EDA2
:102E2200E0939A00E6E0E0939D00E0E0E0939800F2
:102E3200E9E1E0939900E0E8E8B9E0E0E0BDE0E430
:102E4200E7B9E7E8E6B9E0B5EF7EE0BDE0E1E0939F
:102E52007000E0E0E0937200E4E4E0937400EEE1DD
:102E6200E1BDEEE0E1BD0E943C480E941A4810FF1D
:102E720003C0AAE0B0E00CC012FF06C0ABE0B0E0B5
:102E82000E9477750E94606913FF06C0ACE0B0E053
:102E92000E9477750E9460690E946A69E057F84F44
:102EA20010830E946A69EF56F84FA9E00E94706988
:102EB200F4DD0E948A660E9477690E9496550E94FC
:102EC200200EE4E0E0936100EFE0E0936200000096
:102ED20000000000E0B1E170E13019F0E1E0E093C0
:102EE200F80BEBE0E0936200000000000000009BA2
:102EF20003C0E1E0E093F80BE8E0E0936100EFE06B
:102F0200E0936200000000000000E0B1E270E230F5
:102F120019F0E1E0E093F80BE7E0E09362000000D3
:102F220000000000019B03C0E1E0E093F80B0E9467
:102F3200762FE030D1F40E948A660E947769ECE035
:102F4200F9E10E949466A8950E947A690E947F69BD
:102F52000E94CA680E942A740E947A690E947F694C
:102F6200ECE2F1E00E948569EECF0E94272F78946F
:102F7200E091F80BE03021F0E8E1F9E10E9494667B
:102F8200A091F80BA03089F40E945A680F010E94A8
:102F920070680E161F0644F40E947A680F010E94A0
:102FA20088680E161F060CF001C002C00E940B14A6
:102FB2000E942633E030C9F00E948A660E948F6622
:102FC2000E946D5DE1E2F9E10E9494660E948566CD
:102FD2000E942A74A8950E9485660E942A74A89568
:102FE2000E9485660E942A74A8950E948969E5312B
:102FF20028F0A9E0B0E0E0E00E948B750E948A66AA
:103002000E948F660E946D5DEDE2F9E10E94946676
:103012000E948969EA930E94F1430E948A660E9493
:103022007769E1E3F9E10E949466E091F80BE03000
:10303200D9F4E0E0E093040CA091040CA03540F434
:10304200EAE0F0E00E948569A8950E948E69F4CFBB
:10305200A091040CA03520F0A0916205AF3108F4D4
:1030620002C00E940B1438C0E0E0E093040C0E94FE
:103072008969A091040CAE1760F4A8950E94946926
:103082000E947F690E9429670E942A740E948E69A9
:10309200EECFA8950E948D68E0E0E093040C0E94B8
:1030A2009969A091040CAE1760F4A8950E949469E6
:1030B2000E947F690E9429670E942A740E948E6979
:1030C200EECFA8950E948D68A8950E948D68E09128
:1030D2000504EF77E09305040E94495C0E946E1597
:1030E2000E94B12A0E946035F9CFFFCF0E949E69EB
:1030F200A43009F43FC01091E50700910F0CE09154
:10310200E707E03059F0E093E507689424F80E945D
:10311200A369E0E0E093E607E0E520C0E091E6077E
:10312200E03021F0E093E507E2E518C0E0E0E0934B
:10313200E507E0930F0CE0917B0BE03031F0E0917A
:103142007B0BE150EA930E94C130A091EB0BA1707E
:1031520039F0E0917B0BE093E507E4E4E0930F0C98
:10316200A091E5071A1721F4A0910F0C0A1711F08C
:10317200689423F80991199108951A930A930E9469
:103182006A69E057F84F8F01D8011196EBE0EC9392
:10319200EC81D8011696EC93EB81D8011796EC934B
:1031A200D8011896E0E0F0E0ED93FC93D801129676
:1031B2000E94A969D80114960E94A9690E94AE6969
:1031C20025C11A930A930E946A69E057F84F8F014A
:1031D200D8011196ECE0EC930E94AE694BC21A93AF
:1031E20018E0113108F5E091CB07F091CC07A981E5
:1031F200BA81EA27FB27BF010E94BA69E623F723B7
:10320200309781F00E94BA69A981BA81EA23FB232F
:10321200309731F01A93E0E0EA931A93AEDF02C0DE
:103222001A93CFDF1F5FDDCF24C2A091D10BA9304B
:1032320030F0E091170CA091160CEA1709F414C0B3
:10324200E091170CE03021F4E3E6EA93BADF08C01C
:10325200E091D10BEA93E0E0EA93E3E6EA938DDFB3
:10326200E091170CE093160C08951A93A091D007E1
:10327200A13011F0A93009F4FCC110E0153088F436
:103282000E94C569E081E03029F00E94CB69AA81E1
:10329200EA1709F004C00E94D2690E94D7691F5F31
:1032A200EDCFE7C1A091510BECE1EA230895A09183
:1032B200510BA07411F0E2E00895A091510BA07897
:1032C20009F0EFC10DC0A091400BAF3F09F4E9C175
:1032D200E9DFE43009F4E5C1E5DFE03109F4E1C1F9
:1032E200E1E008950895A881AF3F11F4E0E07DC1C7
:1032F200D9DFE43011F4E1E078C1E0E076C1A881E1
:10330200A23019F4CFDFE83011F0E1E06EC1E0E065
:103312006CC1A881B981AC91A130A8F0A881B98112
:10332200AC91A43180F4A881B981EC910E94EC6740
:10333200E050FD4FE081EF770E2EA881B981129601
:10334200EC91E01509F002C0E1E011C1E0E00FC12B
:10335200A881A13118F0E881E051E883E8810E9458
:10336200DC690E94E669A091870BA13018F0A88160
:10337200A43009F006C0E6E9F0E00E9458750E9408
:10338200E66933C1A881A13010F0A43008F006C06C
:10339200E8810E94F169EC5DF94F26C1E0E025C1A8
:1033A200A881A13010F0A43008F006C0E8810E9484
:1033B200F169E75DF94F18C1E0E017C10E942D776E
:1033C200EC81EA93EDDFEF731E2F1030E1F0EC8118
:1033D200EA93E6DFE0743E2FE12FE150A1E00E9484
:1033E2004B74A0910806EA230E2F303011F40030FE
:1033F20009F002C0E1E008C0303011F0003009F4F9
:1034020002C0E1E001C0E0E00E9434772596089511
:103412000E942B7700E00330A0F50A930E9401314D
:103422000E94F669A7E10A9FF001E95EF94F0E9446
:10343200FD690E9426680E946163E091E70BDA0150
:103442005096EC93A091E60BEFE3EA23AE2FE091C6
:10345200E90BE295E07FEE0FEE0FEA0FDA015596E7
:10346200EC93E091E70BE1503E2F3F3F41F0E091BA
:10347200E80B0E94026ADA015196ED93FC930F5F0A
:10348200CACF10E01034D0F51A930E9458301A9324
:103492002ADFE13089F5E091540BEA9373DFE150C2
:1034A2000E2F0F3F49F10E94F669E12FDA011396C0
:1034B200EC93E091540BDA011496EC93E0915A0BE1
:1034C200F0915B0BDA011696ED93FC930E94086A69
:1034D2000E946774A4E6B0E080E090E00E94AA74C3
:1034E200DF01CB01E0915A0BF0915B0B0E947568F2
:1034F200DA011A96ED93FC931F5FC4CF0E943277D4
:1035020026960895A091D007A23031F0A83021F07C
:10351200A73011F0A53009F40AC00E940D6AEFEF3E
:10352200F0E00E94106A74DFE0E0E093590608952B
:103532001A93E981E058E98310E01530B0F40E9453
:10354200CB69AE2FE981EA1759F4A3E21A9FF00181
:10355200E55AF94FE081AE2FE091E507EA1709F04D
:1035620002C0E12F03C01F5FE8CFEFEF1881229660
:1035720008950E942D77ED81EA93DADF1E2F1F3F17
:10358200F1F00E94C5699F01D9011296EC91EF7783
:10359200EC93EC81D901EC930E94EC67E45FFC4F61
:1035A200BF01EC810E94EC67E45FFC4FE081EF77A2
:1035B200DB01EC93EC810E94EC670E94D769E12F5A
:1035C2000E943477D2C40E94146AE081E03051F440
:1035D200E091090CEF5FE093090C0E94146AA0913C
:1035E200090CA0830E94146AE081219608951A931F
:1035F2001FEFE0918B0BF0918C0BA981BA81AE1772
:10360200BF073CF0E0918D0BF0918E0BEA17FB07A0
:103612000CF412C00E94196A0E949D2F1E2F1030B6
:1036220031F01F3F21F0E091E507E11729F4E1E0D5
:10363200E093170CE0E01DC0E0E0E093170C18C027
:103642001A930E94196AD3DF1E2F103089F01F3F90
:1036520039F4E8E3F9E1FA93EA93EB81FC8104C0DF
:10366200E8E4F9E10E94E967FA93EA930E9497116C
:10367200E12F188123960895E0916005E03009F06A
:103682000895E0911106E03009F008950AC0E09132
:103692006105E03009F00895E0911206E03009F08A
:1036A2000895E0E008950E942D77E0910B06F091D5
:1036B2000C06AC81BD81EA27FB279F0110E0133085
:1036C20090F4F901E17049F0A7E11A9FF001EA5E76
:1036D200F94FDF01EC91EF5FEC93D9010E941E6A72
:1036E2009F011F5FECCFEC81FD81E0930B06F0930D
:1036F2000C060E94347739C428970E942B773091A8
:103702000B0610E01330B8F5A7E11A9FF001E65D51
:10371200F94F0081E12FA1E00E944B742E2FE22F7E
:10372200E32391F0003810F0003C08F001C00F5F75
:10373200003C31F4E22FA0910806EA2BE093080640
:10374200003808F400E80FC0003408F40F5F0034BA
:1037520039F4EFEFE227A0910806EA23E093080686
:10376200003808F000E0A7E11A9FF001E65DF94F8A
:1037720000831F5FC7CFE0E0E0931106E0E0F0E0D6
:10378200E093CD07F093CE07E091170CE03021F0E3
:10379200E091D10BEA93DCDDE091D407EF5FE09397
:1037A200D407E0919A0BA091D407EA1751F4E09163
:1037B2009A0BF0E0A0E0B1E00E946C75EA1BE09386
:1037C200D407A091D007A13019F0A93009F096C012
:1037D200A091190BB0911A0BE4E1F0E00E9402757E
:1037E200309719F4E1E0E093D60746DFE03019F0B4
:1037F2004EDFE07809F462C04ADFEF775E2F5A931A
:103802000E9458300E949067E65AF94F508150301A
:1038120011F40C945F1C57DDE13031F4E091D107D3
:10382200EA936DDDE03009F449C00E94236AAE0FCD
:10383200BF1FEC91EC71EC3021F4E091D407E078F9
:1038420051F40E94296AEC91EA9382DD0E94316A66
:10385200EC91EA937DDD0E94296AAC91A63070F565
:10386200AAE9B6E00E9490670E94396A0E94EB685A
:103872000E94296AEC91EA9385DD1E2F1130F0F047
:103882000E943E6A0E94416ACF010E943E6A0E94E3
:10389200396A6D917C91E12F0E94F169EA5EF94FDC
:1038A200E081F0E0E60FF71FDC01ED93FC93E12FDE
:1038B2000E94F169EA5EF94FA0E0A08310E01330A4
:1038C200E8F40E94466A13965C915F3FA9F05A930E
:1038D2007ADE5E2F0E94506A0E943E6A0E94416A0E
:1038E200BF010E943E6A0E94396A0E94566AAE81F6
:1038F200BF811296E0E0EC931F5FE1CFA091D00769
:10390200A23039F0A83029F0A53019F0A73009F01B
:10391200E4C100E0053010F00C946E1EA3E20A9F91
:10392200F001E65AF94FEA87FB87AA85BB85AC917D
:10393200A03019F0A281A07809F0CDC1AA85BB857B
:1039420013960E944975309771F0AA85BB8513962C
:103952000E94636A0E94696A29F4AA85BB8513964C
:103962000E94A969B8C193DEE03021F00E94696A21
:1039720009F4B1C120E030E0333010F00C94171E8E
:103982000E94736ADF010E940D670E94796AA27029
:1039920031F4E885F985A481B581109709F414C141
:1039A200E885F985A181A47011F40C943A1DA181D6
:1039B200A87021F40E941B2CE03009F459C00E9427
:1039C2006A690E94846AEBE0EC93A885B9850E943B
:1039D2008C6AA885B9851396EC91AC85BD8517963E
:1039E200EC93EC85FD8538960F01E885F985A18178
:1039F200E1E0EA230E94936AED93FC93A885B985DE
:103A020014960E944975AC85BD851296ED93FC9380
:103A12000E94966AAC85BD851496ED93FC93A02F07
:103A2200EAE0EA9FF001E30FEF5F0E949C6AE885FB
:103A3200F985A085B185E2E0F0E00E94A574A88531
:103A4200B9851896ED93FC930E94966A309739F4E3
:103A5200A885B9851896E8EEF3E0ED93FC93E88526
:103A6200F985A181E8E0EA2BA885B9851196EC9346
:103A72006CC0E885F985A181A17031F4A885B9856A
:103A820014960E94636A41C00E94A56A7BDCE150E1
:103A92001E2F0E94466A1296EC91E030F1F4AE813C
:103AA200BF8153960E94EB68EE81FF81A189B289A2
:103AB200109751F003881488AE81BF8151960E94FD
:103AC2004975E015F1050CF007C00E94AA6A11F0D1
:103AD2000E94B26A0E94BA6A0EC0E885F9853496DD
:103AE2000E94C26A0E94936A0E94CA6A0E94CF6AB6
:103AF20053960E94A969E885F985A581AA232AF42B
:103B0200A885B98514960E94A969A885B985EC9102
:103B1200EC71EC3021F4E091D407E078B1F4E8855F
:103B2200F985A481B5815E971CF4A181A07209F484
:103B320004C0E885F985A28106C00E94A56A08DC56
:103B4200E885F985A381AA9303DC0E94966A3097DF
:103B520081F0A885B98518960E94636A0E94966AC8
:103B6200309739F40E94AA6A11F00E94B26A0E9448
:103B7200BA6A0E94A56A22DCE03031F10E94AA6A88
:103B820089F00E94B26AAA85BB85EC910E94EC671B
:103B9200E45FFC4FBF01AA85BB85EC910E94EC67F4
:103BA2000E94D66AAA85BB851296EC91E058AA8536
:103BB200BB851296EC93E3E0E09309060E94A56AA6
:103BC200EFDBEF73E0930A06A885B98514960E948D
:103BD2004975309749F52F5F323030F5A885B985A0
:103BE20016960E944975309789F0E885F985A68175
:103BF200B7810E94DD6AAA85BB851396ED93FC937B
:103C0200A885B98516960E94A9690EC00E94736A9A
:103C1200DF01E32FEF5FF0E00E94796AEDEFEA2324
:103C2200A885B9851196EC933F5FA6CE233011F09B
:103C32000C946C1E0E941B2CE03079F00E946A6981
:103C42000E94846AE8E0EC93AA85BB850E948C6A94
:103C5200AA85BB85EC910E949C6A0E94AA6A11F017
:103C62000E94B26AAA85BB85E0E0EC93EA85FB85F7
:103C7200A581ECE1EA23E83071F50E948969AE2F53
:103C8200EA85FB85E38DEA1741F4EA85FB85E48D3D
:103C9200E150EA930E94532F1EC00E941B2CE03079
:103CA200D1F00E946A690E94846AE3E0EC93AC85D9
:103CB200BD85EFEFEC931896EA85FB85E38D0E94B4
:103CC200E26AAC85BD851296EA85FB85E48D0E9489
:103CD200E26A0E94E66A0F5F1DCE0E94EC6A49F416
:103CE200A091D007A23021F0A83011F0A53009F43C
:103CF20001C050C010E0133010F00C94CB1E0E9493
:103D0200466A13965C915F3F11F40C94C91E0E949F
:103D1200506AAE81BF81BD010E94566AEE81FF8169
:103D220038960E94C26A0E94F26A0E94CF6A0E947A
:103D32004975DF010E942177B4F4EE81FF81A681EB
:103D4200B7810E9421777CF4AE81BF810D901C90D7
:103D5200AE81BF8116960E944975D001AE1BBF0B82
:103D62000E9421770CF014C0AE81BF81BD010D907D
:103D72001C90EE81FF81A681B781F001EA1BFB0B4B
:103D8200DB01ED93FC935A93E5E0EA930E948B45A5
:103D92001F5FB1CFE091D307E03041F4E091CD074E
:103DA200F091CE07E093CB07F093CC070E943277D5
:103DB2002E9608950E942D770E94F66A1E2F2FE3F9
:103DC20030E00091D507A091CF0BA13080F0E091B7
:103DD200CF0BE150A091D507AE1728F0E091CF0BA1
:103DE200E1503E2F04C0E091CF0BE2502E2FEC8128
:103DF200E03049F1EF3F51F4A091D507A11BA31781
:103E020020F0E091D507E11B0E2F1DC0EE3F59F4C3
:103E1200E12FA091D507AE0FA21720F4A091D507EC
:103E2200EA0F0E2F10C0EC3F49F4A091CF0BA13046
:103E320020F0E091CF0BE1500E2F05C0AC81A150D4
:103E42001A9FF0010E2FE091D507E01751F00A9367
:103E52000E945830A091410BAD3209F4032F009318
:103E6200D5070E94925DA091D007A83019F40E9454
:103E7200F20F02C00E94BA0F0E943477259608956D
:103E82000E942B770FDAE03111F40C94B31F20E07B
:103E920030E040E050E010E0133050F50E94FD6A3F
:103EA2000E941668309711F10E94006B0E94DC6933
:103EB2002E2B3F2B0E94006BEA9380DAE03029F030
:103EC200E3E0E0930906E0E04EC00E94076B0E9427
:103ED200DC692E2B3F2B0E94076BEA936FDAE030EE
:103EE20029F0E3E0E0930906E0E03DC01F5FD4CF94
:103EF20000E0053068F5A3E20A9FF001E65AF94FA7
:103F0200E081E03019F110E0133000F50E94736A8D
:103F1200DF010E94D0670E940E6BAE0FBF1F129688
:103F2200EC910E94DC694E2B5F2B0E94736ADF01C9
:103F32000E94D0670E940E6BAE0FBF1F1396EC91CA
:103F42000E94DC694E2B5F2B1F5FDECF0F5FD1CF4C
:103F5200F901E423F523309729F0E1E0E093090623
:103F6200E0E001C0E1E00E943277269608951A93BC
:103F7200E0910D0CE03011F40C941220E0919B0BB7
:103F8200E13059F4A0910D0CA13311F4EFE001C01E
:103F9200E0E0EA930E940E5644C0E23059F4A09148
:103FA2000D0CA13311F4E6E001C0E5E1EA930E94B1
:103FB2000E5637C0E53061F4A0910D0CA13319F40F
:103FC200E091500B01C0E0E0EA930E940E5629C036
:103FD200E330B1F410E0173040F40E94D067EA50A9
:103FE200F74F0E94156B1F5FF6CFA0910D0CA13306
:103FF20011F4E1E301C0E0E3EA930E940E5611C01E
:104002000E94196BE9E4EA930E945A59E0910D0C5F
:10401200EA930E945A59E0E0EA930E945A590E9498
:10402200E45A40C222970E942B7730E0A091D00739
:10403200A23029F0A83019F0A53009F014C1A985E1
:10404200A03410F00C943321E091E507E03009F43C
:104052000AC1E9850E94206BE03131F4E1E3E0938B
:104062000D0C85DFE1E0FFC02ED9E03009F4FBC082
:1040720010E0153080F40E94C569E081E03031F033
:104082000E94CB69AE2FE985EA1709F002C0E0E091
:10409200EAC01F5FEECFF4DEE03011F40C9433215E
:1040A20010E00E94C569EE83FF83AE81BF81EC916F
:1040B200E03011F00C942C2113960E94A96900E0C3
:1040C200033010F00C94FD20A3E21A9FF001E15A94
:1040D200F94FDF010E9426670E94256BAF01DA01CA
:1040E20016960E94A9690E942D6BDA011296EC9332
:1040F2000E94346BDA011396EC93A091510BEEEF10
:10410200EA23DA01EC930E943B6BDA011196EC93FD
:10411200C9D8E43139F0FA01A181E2E0EA2BDA01EF
:104122001196EC930A93EBD8E03011F40C94DF2053
:10413200FA01A281AA9326D9E1502E2F2F3F81F0B6
:10414200A7E12A9FF001EA5EF94FA0E0A083A7E170
:104152002A9FF001E95DF94FA0E0B0E0A083B183AE
:104162000E94436B0E941668DA011496ED93FC9349
:10417200013030F00E94436B0E941668309709F0BC
:104182000EC0AE81BF811596E02F0E94466B0E9441
:104192000E6BAE0FBF1F1196EC91E062EC93AE81F5
:1041A200BF815A96EC91E062EC93023030F40E94A7
:1041B200496BDA0116960E94E26A04C0DA0114968B
:1041C2000E94A9696FD8EC3019F4E0E0E093D407BB
:1041D2000E94506B0E94026ADA011896ED93FC93DA
:1041E200FA01A281A63030F0A181E4E0EA2BDA01E3
:1041F2001196EC930F5F64CFA091D007A23011F01B
:10420200A53019F4A885AF3F08F007C0E091E50793
:10421200EA93EA85EA930E94A731E885AE81BF81DD
:10422200EC93E091E507AE81BF811196EC93E985AD
:10423200AE81BF811296EC93A885A43128F4E8855B
:104242000E94EC670E94D769AE81BF811696EC91FD
:10425200ED7FEC9331E01F5F303011F4153008F040
:1042620001C01FCFE32F0E9432772A9608950E9441
:104272009E69A23021F0A091D007A53021F40E94BE
:10428200576B0E940869A091D007A830E1F40E9400
:10429200576BE1E0EA930E94F75DE091990BE03001
:1042A20081F4EA81ADE0EA9FF001E050FD4FE08148
:1042B200EF771E2FABE01A9FF001EF51FA4FA0E00B
:1042C200A083689420F81981088123960895649741
:1042D2000E942B77A091D007A23039F4E091E50734
:1042E200EA93EB8DEA930E94A731A091D007A83000
:1042F20011F00C94D9210FEF20E0233050F4A7E104
:104302002A9FF001E95EF94FE081AE2FEA8DEA17AC
:1043120009F402C02F5FF1CFA7E12A9FF001EC5E02
:10432200F94FAF01DA0115960C910F3F11F40C947D
:10433200D9210E94626B10810E94686BECF4A3EE9B
:10434200BBE00E94636A0E94726B0E94786BA0833A
:10435200B1831A930E946436ABE00A9FF001E752E0
:10436200FA4F30810A93FE0137960E947D6B3A9391
:10437200FE0137960E94816B0E94876BC9F40E94EE
:10438200626BAFEFA083DA011396EFEFEC93DA01E1
:104392001596EC930E94726B0E948D6B0E94926B39
:1043A2001A930E9464360A930E943411689420F88A
:1043B2000E9432776B9608951A9310E01031B0F490
:1043C200A7E11A9FF001E75DF94FE081EF73AE2F8D
:1043D200E981EA1729F41A930E94DF19E03009F4FF
:1043E20003C0E1E01881DFC01F5FE8CFE0E0188181
:1043F200DAC01A93E091100CF091110CFA93EA933F
:104402000E94F1680E940763E030F9F00E949B6B02
:1044120010E01330D0F4A091140CAF5FE3E00E94DF
:10442200FF74E093140CEF5FEA93C6DFE03059F0BB
:10443200E3E0E0930906E091140CF0E0EF5FFF4E39
:10444200E0930A062FC01F5FE4CF2CC01A93E091BD
:104452000806E0930C0CE8E7F0E0FA93EA93ECED3F
:10446200F0E0FA93EA930E94C45D10E01330D0F4B6
:10447200E12FEF5FEA93A0DFE03091F00E949866AF
:10448200E12FEA5F0E94A26BE5E5F9E10E949466E2
:10449200ADE9BBE00E94D0670E94256B0E94A46B2D
:1044A2001F5FE4CF19910895A4DFE0910906E1307E
:1044B20029F4EDE5F9E10E94A76B3CC0E23029F452
:1044C200EAE6F9E10E94A76B35C0E33051F4E5E575
:1044D200F9E1FA93EA93E0910A06F0E0E050F04F36
:1044E20029C0E43019F4E2E7F9E11FC0E53031F404
:1044F200E0910A06EA930E94961120C0E63019F470
:10450200EAE7F9E112C0E73029F4E0E8F9E10E94B4
:10451200A76B10C0E83029F4ECE8F9E10E94A76B20
:1045220009C0E93059F4EBE9F9E1FA93EA93E09131
:104532000A06F0E0FA93EA930E949711E0E0E09312
:1045420009060895A881B9811196E1E0EC930E94D1
:10455200AC6BA881B9811296ED93FC930E94581915
:10456200A881B9811796EC930E948969A881B981C3
:1045720018960E94E26AE091C105A881B981EC9384
:10458200E091E00BA881B9811696EC93E091400B83
:10459200A881B9811A96EC930E94086AA881B98110
:1045A2001496ED93FC932296089564970E942D77BA
:1045B200A091990BA230E1F4EB8DEA930E9458305E
:1045C2000E945819A3EEBBE00E94E26AA1EEBBE092
:1045D200EB8D0E94E26AE091E507E093E00B0E9416
:1045E200B16B309721F00E94B16B0E94B66B14C080
:1045F200AA8DAF3F09F4CEC0EA8DEA930E945D36E0
:10460200AB8DAF3F29F40E94AC6B0E94BB6BEB8F6A
:10461200EB8DEA930E9458300E9458190E2FA98DF3
:10462200AF3F21F00E946419E03009F001C0B2C02E
:104632000E94786B0E942667AE17BF071CF020DC31
:10464200E13009F0A7C0A091880BA03021F4A0911D
:10465200990BA23021F50E948969E13041F00E9454
:104662001B2CE03021F00E94312CE03009F004C014
:104672000E946A690E94BF6B0E948969E13021F43D
:104682000E94212CE03009F409C00E94C66BE75A4F
:10469200F84FFA93EA9356DF0E94CC6B79C0EB8D08
:1046A200EA93EA8DEA93BEDC1E2F113011F00C94CE
:1046B200C923A0918A0BA13069F4E091E507EA933E
:1046C2000E94AC6BFA93EA93EFEFFFEFFA93EA934F
:1046D2000E9433430E94786B0E9426670E94CA6A36
:1046E2000E94D26B689420F8A091990BA03019F423
:1046F200A88DAF3F09F437C00E94D76BE352FA4F3F
:104702000E94786BA083B183E88D0E94E3673081B9
:10471200E88DEA93FE0135960E947D6BE88D0E943A
:10472200E367E081EA93FE0135960E94816B0E9465
:104732005319E03131F00E94D76BEF51FA4FA1E0EB
:1047420005C00E94D76BEF51FA4FA2E0A0830E94EE
:10475200D76BE152FA4FFF93EF930E94FB62AF9146
:10476200BF91ED93FC930E94876B19F4E0E0E09314
:10477200E00BEA8DEA930E946436E091E507EA9342
:104782000E94B16B0E942E67FA93EA930E946334EF
:10479200E1E001C0E0E00E9434776C96089570DB9E
:1047A200E13041F40E941B2CE03021F00E94312CB8
:1047B200E03009F009C00E94B16B0E94B66B0E9402
:1047C2006A690E94BF6B25C22DC20E94DC6B0E94E7
:1047D200E26B0E9498660E9498660E946D5DA091AD
:1047E200D207A23021F4EFEAF9E10E949466A09187
:1047F200D207A13021F4E6EBF9E10E949466E09140
:10480200D207E03021F4EDEBF9E10E9494660E94B8
:10481200EC6B0E946D5D0E94F16B0E94F66BFA9345
:10482200EA93E0915A05F0915B050E94FC6B0895B2
:10483200E1E003C0E0E001C0E2E0E093D207C5DFBF
:1048420008950E945319EC3109F0ECC1E091500B2C
:10485200E33631F4A091D007A23009F4EBDF17C0A0
:10486200E23631F4A091D007A23009F4E5DF0FC09F
:10487200A091C005A23011F0A63021F4E091500BB6
:10488200EA9398DAA091C005A43009F4D1DFC1C13E
:104892001A930A93A0E023FCA1E0A03019F0AA81A8
:1048A200A03009F014C0E89423F8E7E0E093CF07C2
:1048B2000E94AA5CA091E707A03019F40E94006C44
:1048C20009F405C00E94056C88D7E89424F824FEF8
:1048D20025C0E091E907F091EA070E94EC660E9488
:1048E2000763E13019F0AA81A130B9F4A3D7E0300F
:1048F200A1F00E940A6C0FEF1FEF0E94116CE030D2
:1049020021F40091DD071091DE07EB81EA93E0913B
:10491200E507EA931A930A9360D710C0E091E9077A
:10492200F091EA07FA93EA93ECE2F1E00E94196C43
:10493200E13021F40E941D6CE093E60719810881A1
:1049420055C4E1E0E09309040E9498660E949866CB
:104952000E94216C0E9498660E9498660E946D5D7A
:10496200E0EDF2E00E949466E091D1070E94256C8E
:10497200EEEDF2E00E949466E2E0E093090408950D
:104982000E940D6AE0ECF0E00E94106AE881E030DB
:1049920009F406C0A091D107AF5FE3E00E94FF7463
:1049A200E093D107E1E0E093090C0E94091A22C2C8
:1049B2000E942D7710E0103410F00C942C250E94E8
:1049C200D067E65AF94F30813F3F11F40C942A2503
:1049D2001A930E94583000E00E94296C0E941668C7
:1049E2003B97C4F00E942C6C0F010E94296C0E941C
:1049F2001668D001ED93FC930E94236AEA0FFB1F15
:104A02000F010E94236AAE0FBF1FEC91EE7FD0010F
:104A1200EC9301E00E94326C0E9416687597A4F034
:104A22000E942C6C0F010E94326C0E941668D00109
:104A3200ED93FC930E94236AEA0FFB1F0F010E9471
:104A4200236A0E94356C01E0013019F41A930E9426
:104A520081301F5FB0CFC8C30E949E69A93011F494
:104A62000E943C6C23FE06C0E7E0E093CF070E9461
:104A7200056CB3D60E949E45E030A1F1E0E00E94B1
:104A8200436C103838F5113231F4E7E0E093CF0788
:104A92000E94056CA2D61D3439F40E944A6C0E9411
:104AA200875AE3E0E093CF071B3271F40E944F6C08
:104AB200EAE2EA93E8ECF9E1FA93EA93E091D107AA
:104AC200E05DEA930E94875A1F3219F4E1E0EA930B
:104AD20071D937DF103830F00E94556C1A930E945A
:104AE200E41AAFDE0E94481B0E2F003810F40C941B
:104AF200BA250F770034E0F5E091D607E03069F08F
:104B02000A930E94E41AA091D007A13019F40A93E3
:104B12000E94EE11E0E0E093D607E091150CE01759
:104B220039F10A930E9458300E94296AAC91A83048
:104B320028F40E94316AAC91A830A8F0E02FEF5F10
:104B4200E09359060A930E94E41A0E94296AEC91A2
:104B5200EA930E94316AEC91EA93E0915906EA9352
:104B62000E94BE1803C0E0E0E09359060093150CC2
:104B72000EC0A091150CAF3F51F0E0915906E03004
:104B820019F0EA930E94E218EFEFE093150C0991F5
:104B920019910895A881A03310F0AA3308F01DC01E
:104BA2000E94596CE8EEF3E00E940275AAE0B0E0C0
:104BB2000E94A574DF01E8810E945E6CEA0FFB1F70
:104BC200E093DB07F093DC07E1E0E09309040E9445
:104BD200EC6B0E94216C0E94F16BA881A33441F41A
:104BE2000E94E26B0E94EC6B0E94216C0E94F16BAE
:104BF20001C1E0917E0BF0917F0B0E94616C11F478
:104C0200E2E00895E0917C0BF0917D0B0E94616CD3
:104C120011F4E1E00895E091820BF091830B0E9480
:104C2200616C11F4E0E00895EFEF0895E0E0E093A5
:104C3200D207A091D007A23021F40E94925D0E9477
:104C4200BA0FA091D007A83009F425D6A091D007B9
:104C5200A53009F433D10895E2E0EA930E94584363
:104C6200E1E0E0930904E881EA9394DFA881AF3799
:104C720021F4E0911006E37009F403C0E2E0E0934E
:104C8200CF07A881A13239F0A33421F40E94596CD4
:104C9200109709F004C0A091D007A23009F00FC00C
:104CA200A091D207A33009F4C7DDA091D207A230A8
:104CB20009F4BCDFE091D207E03009F4BBDDA88142
:104CC200AD3311F00C94B9260E94AA5CE091D20790
:104CD200E03089F4E091DB07F091DC070E94656C1B
:104CE20041F4E091DB07F091DC070E946B6C9EDFE0
:104CF20001C0A0DD3DC0E13069F47BDFEF3F41F050
:104D0200E3E00E94706C0E944A6C0E94766C01C0C3
:104D12008DDF2EC0E230F1F40E94596CA034E0E045
:104D2200BE07B4F4E091DB07EA930E947D6CE1E0F8
:104D3200E09309040E9498660E9498660E946D5D45
:104D42000E94816C0E94BB10E3E0E093D20701C095
:104D520073DD0EC0E33061F4E091DB07EA930E9459
:104D62005830E091DB07EA93EEEFEA935BD964DD1A
:104D7200A881AD3409F45CDDA881A43521F4A091A9
:104D8200D007A23009F001C055DDA881AB3221F471
:104D9200EEEFEA930E94DB1EA881AD3221F4EFEF21
:104DA200EA930E94DB1EA881A73421F4E1E0EA9392
:104DB2000E94DB1EA881AB3421F4ECEFEA930E943F
:104DC200DB1E18C00E94831A0E94925DE0E0E0930D
:104DD200D207A881A13039F40E94006C21F0A09181
:104DE200810BA03009F402C025DD04C00E94BA0F75
:104DF2000E94116C219608951A930A930E943C6CAA
:104E02000E94846C71F10E948C6C58F10E94556C66
:104E120018DDE03031F50E94946C0E94BA1AEF3F1F
:104E220009F0D8C40E94996C21F40E946419E130FF
:104E320009F017C00E945319E83119F40E949E6CC0
:104E420009F001C0C7C40E94946CECD80E2F013047
:104E520021F4A091500BA03009F403C01A930E94D0
:104E62009611A0911306AF3F41F110911306EFEF97
:104E7200E09313061A930E9458300E94996C21F411
:104E82000E946419E13009F018C00E945319E831F8
:104E920019F40E949E6C09F001C09CC41A93EEEFB3
:104EA200EA93C0D80E2F013021F4A091500BA0300C
:104EB20009F403C01A930E9496118CC40E94831AAB
:104EC2000E94091AE89421F8E0E0E093D5070E94D5
:104ED200A56C0E94925D0E9498660E9498660E944C
:104EE2006D5DE09117060E942E68E09118060E94FF
:104EF2002E680E9498660E948A660E946D5DE0910B
:104F020024060E942E68E0911E06F0911F060E9460
:104F12001D6808950E942D770E943C6CC5DA0E949C
:104F22009E45E03049F00E948C6C30F00E94556C36
:104F320088DCE03009F433DCE091120CF091130CC0
:104F42000E94D3680E940763E03011F40C940B288E
:104F52000E94A56C0E949866E2E0F0E00E94F7676A
:104F6200E0911C06F0911D060E941D68E09120064A
:104F7200F09121060E941D6800E0033010F00C94AD
:104F82000B28A7E10A9FF001EC5EF94F9F01F9019E
:104F9200A381AF3FE9F1D9011A960E9449750E9497
:104FA20067747F936F93FF93EF930E94AC6CAF9102
:104FB200BF918F919F910E9467740E94AA74DF0132
:104FC200CB010E94B16CD9011C96ED93FC93F901BF
:104FD20004841584D9011E960E944975E015F105D5
:104FE200B9F0F90104841584A685B785F001EA1B9E
:104FF200FB0BE093630BF093640BD1DBE13041F4E4
:10500200D9011C960E944975D9011E96ED93FC9315
:105012000F5FB3CFE9C00E942D770E943C6C0E94C3
:10502200846C11F40C949F280E94A1450E2F0A93C0
:1050320013DE003820F0A091C105A03808F42BC07F
:105042000F770A930E94B86CFA93EA930E942B3668
:105052001E2FA091990BA03011F41F3F09F416C026
:1050620030E0333098F4ABE03A9FF001E952FA4F66
:10507200E081E11749F43A9FF001E752FA4FE081EB
:10508200EF5FE093C105232F3F5FEBCF0A930E94AE
:10509200946C2A9352C0A091990BA03021F400384D
:1050A20010F0033808F00AC00F770E94626B10817B
:1050B200EFEFEA930E94946C0A9377DAA091990B2E
:1050C200A03011F0003808F439C00F770A930E941B
:1050D2005830B7DBE03091F50E94BB6C0E94BA1ADF
:1050E200EF3F09F081C00E946419E13039F50E9456
:1050F2005819E03049F40E94BB6C0E941320E03042
:1051020011F00E94C06C1AC00E945319E83141F498
:105112000E949E6C21F00E94BB6C0E9413200EC064
:10512200A091D507E02F0E949367AE0FBF1F1C917D
:105132000A930E94946CEFEFEA9337DAA091130678
:10514200AF3F09F100911306EFEFE09313060A93C4
:105152000E94B86CFA93EA930E942B361E2F0A9390
:105162001A93EEEFEA93EFEFEA931FDA1F3F41F44F
:10517200A091540BA03021F4A091570BA03009F05C
:1051820002C00E94C06C20FE0AC0E89420F8E091A0
:10519200990BE03019F4C4D311D501C06CD530E0BD
:1051A200333010F50E94C66CE03031F00E94CD6CB5
:1051B2000E94D66CE03069F40E94C66CE23041F481
:1051C2000E94CD6C0E94D3680E940763E03009F40C
:1051D20009C0ABE03A9FF001EF51FA4FA0E0A08383
:1051E200689420F83F5FDCCF0E94347724960895BC
:1051F2000E942B77A091D007A33011F40C94B02A0F
:10520200E091F007ED3411F00C94DB29E091F10705
:10521200EA3511F00C94902924FC81C0E091F20748
:10522200E0532E2FE091F307E0533E2FE4EFF7E037
:105232000E94DB6C0E94E06CAB3429F40E94E66CA5
:105242000E949B580E2F0E94E06CA43529F40E9404
:10525200E66C0E949B58AF01E091840BE31731F595
:10526200E0E0E0930B0C0E940A6C4093DD07509340
:10527200DE07A091E6070A1759F0E7E0E093CF07AF
:105282000093E60720930A0CE0E0E093E5070DC0E7
:10529200A0910A0C2A1721F0A091E407A03009F08E
:1052A20004C02093CF0720930A0C35C0A091E607D3
:1052B200A03049F4A091850B0E940D67E255FF4F83
:1052C200E491EA2309F40CC0E7E0E093CF072093CE
:1052D2000A0CE0E0E093E507E091EF07E0930B0CA6
:1052E200E091EF07A0910B0CEA17A9F44093DD07B8
:1052F2005093DE070093E6070E940A6CA0910A0C05
:105302002A1721F0A091E407A03009F004C02093ED
:10531200CF0720930A0C273011F40E94A369E09171
:10532200F107E93439F4E7E00E94706C0E941D6CC9
:10533200E093E507E091F107E23439F4E4E00E94FA
:10534200706C0E941D6CE093E507E091F107E03577
:1053520019F4E1E0E093CF07E091F107EC3449F46E
:10536200E4E0E093CF07E091F207E053EA930E9472
:105372003C16E091F107E334E9F4A091F207A1337E
:1053820020F0A091F207A93308F014C00E94E96C42
:10539200E091D807EA930E94CC32E091EF07EA93BA
:1053A200EBECF9E1FA93EA930E94EF6C0E945C75D0
:1053B2000E947B5AE091F007E03521F4A091D007DA
:1053C200A13009F003C00E944F6CBBDAE091F007F4
:1053D200EF3459F4E091F107EE3439F4E091EF073C
:1053E200EA93EEECF9E10E94F46CE091F007E33508
:1053F20069F5E091F107EF3349F5A091F207A03387
:1054020020F0A091F307A03308F420C00E94E96CB9
:10541200E091F307E0531E2FA091D807A63010F4B5
:105422001A3008F013C0103011F40E941332E091C8
:10543200EF07EA93E1EDF9E1FA93EA930E94FA6C3D
:105442000E94016D0E945C750E947B5AE091F007F8
:10545200E33411F00C94782AE091F107EF3311F064
:105462000C94782AE091F307E03319F4EFEFE0931C
:10547200D907A091F207A033F8F00E94E96CA0913D
:10548200D807A630C8F4E091D907EF5FE093D907B7
:10549200E091D807EA93E091D907EA930E94963205
:1054A200A091D50BB091D60B109721F4A091D907FA
:1054B200A03408F001C0E7CFE091D907EA930E9437
:1054C20058300E94066DE4EDF9E10E940B6D0E94D6
:1054D20046690E9421680E940F6D0E944F690E94D6
:1054E2000F6D0E94156D0E94F5590E94455AE09178
:1054F200F007E434A1F5E091F107E43481F514E01A
:10550200E1E0E093EF08103538F40E94D067E251F1
:10551200F84FE081E03208F41AC00E94D067E251ED
:10552200F84FE081E33259F40E94D067E151F84F1D
:10553200E081E053EA930E940E561F5F06C00E946C
:10554200D067E251F84F0E94156B1F5FDCCF0E94BB
:10555200066DE7EDF9E10E940B6D0E94455A72C497
:105562001A930A930E94EC6A11F40C941D2BE0E04A
:10557200E093170CE091CF07EF770E2F0093CF0740
:105582000E94925D0E948A660E948F660E946D5DF3
:10559200013021F0A091D007A13009F00BC0E6EE56
:1055A200F2E00E94946604DA0E94F1680E94BD450E
:1055B2000E94925D073049F40E94831AE0E0E09372
:1055C200D2070E94CE110E942722043031F4EAED64
:1055D200F9E10E9494660E94620E083019F40E945A
:1055E2001A6D59D1053019F40E941A6D67DC013029
:1055F20039F40E94276D0093D007A3D90E94BA0FF5
:10560200093059F40E94276D0E94BA0F0A93E1E013
:10561200EA933ED9E1E0E093170C023029F40E94AC
:105622001A6DE1E0EA93CEDB033011F40E942F40C1
:105632000093D0070E941619A091D007A73011F04D
:105642000C94CC2BE091100CF091110C0E94D368B9
:105652000E940763E03021F0A091D207A03009F048
:105662000AC00E949B6BE0910C0CA0910806EA17FD
:1056720011F00E9427220E949E45E030E9F0E2E00C
:105682000E94436C1A9386DA1D3409F4D1D81D3373
:1056920099F40E94AA5CADDAEF3F41F0E3E0E093B7
:1056A200CF070E944A6C0E94766C06C0E7E8E0933E
:1056B200CF07E0E0E093D207A091E507A03031F0F8
:1056C200E091E507A091E407EA1709F455C0E091DB
:1056D200E507E150EA930E94C130A091EB0BE1E0B3
:1056E200EA23E13021F4E0911006EF7C09F429C0AD
:1056F200E0E0E093E407E0910A0CE03019F0E09377
:10570200CF071EC012E0E0911006EC7009F018E01D
:10571200E0917B0BA091E507EA1781F0E09110067A
:10572200E07439F011E0EAE2EA93EFEDF9E10E9468
:10573200F46CE0911006E07809F019E01093CF07BD
:105742001BC00E94925D0E94CE110E948A660E9436
:105752008F660E946D5DEBE4EA930E94FF5CE0912C
:10576200E507EA930E94F143E2EEF9E10E949466B2
:10577200E091E507E093E407A091E507A03021F46A
:10578200A091E407A03009F406C0E0E0E093E4074A
:10579200E7E8E093CF07A091D007A33011F40E946D
:1057A2002F3EA091D007A13009F456D9A091D0077D
:1057B200A23009F421DBA091D007A83009F42BDC38
:1057C200A091D007A53009F4A5DBA091D007A9309C
:1057D20009F442D90991199108950E946A69EF5614
:1057E200F84FA6E0A0830E946A69E057F84FAB81A8
:1057F200A0830E946A69EA56F84FAA81A0830E9498
:105802006A69EE56F84FA881B981A083B1830E94DC
:10581200E66A0E94FF400C9429300E94326DA881F2
:10582200B981AC91A53020F0A881B981E0E0EC9378
:1058320022960895A091CA07BB27E091C90705C027
:10584200A091C807BB27E091C707F0E031960E94FC
:10585200CA6A3596DF01E5E0F0E00E94027508951C
:105862001A931091CA07E091C907E11791F00E94BB
:10587200386DE13021F00E94386DE23011F4E1E040
:105882004DC0EDB7FEB7FA93EA931F93C6DF1F919F
:10589200EACFE0E043C01A930E94831AE7EDF5E0F5
:1058A2000E94FD69E1E2F0E00E94106A10E013300C
:1058B20068F40E943F6DAFEFA083ABE01A9FF00146
:1058C200E352FA4F0E948D6B1F5FF1CF10E013304D
:1058D20048F4A7E11A9FF001E75EF94FAFEFA0830A
:1058E2001F5FF5CFE0911006E37019F00E94006C83
:1058F20009F402C0689401C0E89421F8EFEFE09344
:10590200E307E091990BE03029F40AD057D1E894EB
:1059120020F804C00E94925D0E94F20F199108952E
:1059220022970E942B7700E0033058F40E94456DC5
:10593200A0E00E944B6DE652FA4FA0E0A0830F5FF9
:10594200F3CF00E00330C0F50E94626BE081EF3FCD
:1059520089F10E94626BE0810E94506DB9F00E9451
:10596200726BDF010E9449750E94786BEA17FB0790
:1059720051F00E94726B0E94786BA083B1830E94E7
:10598200576DA1E0A0830E94456D12C0ABE00A9F53
:10599200F001EF51FA4FE081E03061F40E94626B56
:1059A200AFEFA0830E94726B0E948D6B0E94576DB5
:1059B200A1E0A0830F5FC6CF0E944F361E2F1F3F6C
:1059C20011F0E1E001C0E0E0E093170C1F3F11F499
:1059D2000C943D2D50E000E0033048F40E94626BCD
:1059E200E0811E1711F451E002C00F5FF5CF503075
:1059F200E1F500E00330C8F50E94626BE081EF3F01
:105A020091F50E94626B10830E94726B0E94786B08
:105A1200A083B183ABE00A9FF001E552FA4FA09157
:105A2200E00B0E944B6DE452FA4FFF93EF930E94FA
:105A3200AC6B0E94BB6BAF91BF91EC930E94576D10
:105A4200A1E0A0830E94456DA1E00E944B6DE1524E
:105A5200FA4FFF93EF930E94FB62AF91BF91ED93D8
:105A6200FC9351E002C00F5FC5CF503029F01A936A
:105A72000E9456361E2FAACF30E0333010F00C941D
:105A8200832DA7E13A9FF001EC5EF94FEE83FF838D
:105A920050E000E0033048F5503029F5ABE00A9FB2
:105AA200F001E452FA4F20812A930E9458300E945A
:105AB200456DE081E13059F42A930E947419E13076
:105AC20031F4A32FAF5FE091540BEA1709F00BC03A
:105AD200E22FAE81BF811396EC93E02FAE81BF819E
:105AE2001596EC9351E00F5FD5CF503049F4AE815B
:105AF200BF811396EFEFEC93AE81BF811596EC93C5
:105B02003F5FBBCF0C9454300E942D77AC81BD8196
:105B1200EBE4EC93EC81FD8131960E945D6DE552E0
:105B2200FA4FE0810E94686D00E00E94726DEC9174
:105B3200E03011F00F5FF9CF0E94726DE0E2EC935A
:105B42000F5F0E94786D0E945D6DE352FA4FDF0194
:105B52000E9449750E9421680E947F6DEE81ABE030
:105B6200EA9FF001E452FA4F10811A930E945830D2
:105B720000E00E94726DEC91E03011F00F5FF9CFFE
:105B82000E94726DE8E7EC930F5F0E94726DE0E293
:105B9200EC930F5F30E03A3050F40E94786D0F01C1
:105BA200A1E4BBE00E94846D0F5F3F5FF4CF0E94CF
:105BB200726DEC930E9434772796089564970E9441
:105BC2002D7700E010E0133040F40E943F6DE08139
:105BD200EF3F09F40F5F1F5FF6CF033021F0A09172
:105BE200E307A03009F406C0E0E0E093E307EA939C
:105BF2000E94101110E0133068F5ABE01A9FF0011B
:105C0200E652FA4FE081E03019F10E948B6DB1F05B
:105C12001A93FE0135960E947D6BABE01A9FF0014C
:105C2200E452FA4F30813A930E9458301A93FE019F
:105C32003596FA93EA930E9445110AC01A930E947C
:105C42003411ABE01A9FF001E652FA4FA0E0A083B4
:105C52001F5FD1CF033021F4A091E307A13009F4F3
:105C620006C0E1E0E093E307EA930E9410110E946C
:105C72003477689608950E942B77A091990BA230F1
:105C820009F4E0C030E0343168F40E94936D0E9460
:105C9200966DDA011296E0E0EC93DA01EFEFEC9305
:105CA2003F5FF1CF0E944F360E2F0F3F11F0E1E020
:105CB20001C0E0E0E093170C0F3FA1F10E94AC6B32
:105CC200FA93EA930E940C301E2F1F3F31F1A091EC
:105CD200D507E12FEA1B3E2F3431F8F40E94936D71
:105CE2000E94966DFA0132960F01E081AE2F0E945A
:105CF2009C6DB0E0EA0FFB1FD001EC93FA01A28188
:105D0200A43620F0DA011296E3E6EC93DA01AC91C4
:105D1200AF3F19F4E02FDA01EC930A930E94563652
:105D22000E2FCACF0E94671530E0343110F00C9468
:105D3200232F0E94936D0E94966DFA01A381AF3FBB
:105D420011F40C94212F0E94A16D0E94206BE83166
:105D520031F40E94A16DEA9399D0E03009F407C0B2
:105D62000E94A16DEA9392D0DA011296EC93A0916F
:105D7200510BA07839F4FA010280DA011196EC9104
:105D8200E01509F45DC0DA0113962C91ADE02A9F6B
:105D9200F001E45FFC4F0F01DA011296EC91D001A1
:105DA200EC930E94A16DEA930E94991AEF3F51F081
:105DB200ADE02A9FF001E45FFC4FBF012A9FF00192
:105DC2000E94D66ADA011296EC91E03089F00E94C4
:105DD200A66DDF010E94AC6DEC93ADE02A9FF0014D
:105DE200E75FFC4FDF01E0914F0BEF70EC9313C0C4
:105DF2000E94AC6DE03021F40E94A66DA0E003C0C9
:105E02000E94A66DA8E0A083ADE02A9FF001E75FA3
:105E1200FC4FA7E0A0830E94A16DEA930E94991A09
:105E2200EF3F19F0ECE0E0930A04DA011296EC91EC
:105E3200DA011196EC932A93E1E0EA930E94F75D6E
:105E42003F5F73CF0E94327726960895E7E0E09392
:105E5200CF076AD0A8950E942734A8950E946C3675
:105E6200A895EFEFE093690BE093400BE093EA0B08
:105E7200E093E50BE09313060E94B16DEC7F29F0ED
:105E8200A8E0B0E0E0E00E948B7508950E94B66D34
:105E92000E94BA6D17FD02C0103011F4E0E091C308
:105EA200E12F8FC30E94B66D0E94BA6D17FD10E0FC
:105EB2001A3008F41F5FE0EAEA930E94DD670E944D
:105EC200C26D7FC30E94B66D0E94BA6D17FD02C0FB
:105ED200103011F4E0E075C31150E0EAEA930E9439
:105EE200DD670E94C26DE1E06CC31A930A9310E071
:105EF2000E9485660E942A74A8950E942361E03060
:105F020021F4E0EA0E94C96D09F002C001E001C07B
:105F120000E00E9434611F5F003011F4153008F078
:105F220001C0E6CFE02FFEC20E94CE6D77C40E9470
:105F3200CE6D0E94DB6D0895A881B9810E94217700
:105F420024F4A83EE3E0BE070CF005C00E94E16D18
:105F52000E94966137C3E0E035C3EA81E03011F474
:105F6200EFEFEA83A881B9810E94217724F4A83E49
:105F7200E3E0BE070CF006C00E94E16DED81EA93FA
:105F82000E94C26174C10E942D7720E030E0283E59
:105F9200E3E03E077CF4A8953A932A93CDDF1E2FC7
:105FA2001F3F29F0EFEFEA933A932A93D6DF2F5F50
:105FB2003F4FEDCF0E9434774BC01A930A93E0E033
:105FC200F0E0E093180CF093190CAA81A03468F465
:105FD2000E94DD670E94EA6DE55FFB4F8F010E9420
:105FE200EF6DE8E1FCE00E94F86DE091180CF09191
:105FF200190C3BC11A931FEF1F5F1A93DEDFA981B1
:10600200BA81EA17FB0711F0113408F001C0F4CF8E
:10601200E12F18812CC11A930A930E94F66AA0916B
:10602200D507EA0F0E2F013408F00FE31091D507C0
:10603200101758F41A93C1DFAA81BB81EA17FB0734
:1060420011F4E12F03C01F5FF3CFEFEF1981088135
:10605200249608950E942B7710E0103418F50E94C0
:10606200E966E8E2F0E00E94A574E050FC4FAF015F
:10607200E0EAEA93FA0170960E94FC6DEC713E2F01
:10608200E0EAEA93FA013F960E94FC6D0E2FEF813F
:10609200E31719F4EE81E01709F002C0E12F03C003
:1060A2001F5FDBCFEFEF0E943277289608951A9395
:1060B2000A93E091400BAA81EA1709F1A034A8F4EF
:1060C2000E94DD670E94EA6DE050FC4F8F01E0EA1A
:1060D200EA930E94C5681A930A930E94156D0E9462
:1060E200E361EA81E093400B0AC0EFEFE093400BDB
:1060F2000E94156D0E94006EE0E0E0934B0BB5C06C
:106102000E94056E0E94EA6DE050FC4F8F01AA8149
:10611200A03460F4E0EAEA930E94C5681A930A93F5
:106122000E94156DE0E2EA930E944B629EC01A93B0
:106132000A93E091690BAA81EA17B9F00E94DD6720
:106142000E94086E40F40E94126E0E94F86DEA816D
:10615200E093690B0AC0EFEFE093690B0E94246998
:106162000E94006EE0E0E093740B7FC00E94056E17
:106172000E94086E20F40E94126E0E94DB6D75C0B0
:106182001A930A93E091EA0BAA81EA1761F10E943D
:10619200DD670E941D6E08F50E94EF6DEBEEFBE0DD
:1061A2000E94F86DEA81E093EA0BE0E0E0931006CA
:1061B200A091EC0BA13020F0A091EC0BA83008F0DC
:1061C2000BC0AFE8BBE0E091EC0B0E94466BAE0F58
:1061D200BF1FEC91E093100606C0EFEFE093EA0BCD
:1061E200E0E0E093EB0B41C00E94056E0E941D6E41
:1061F20030F40E94EF6DEBEEFBE00E94DB6D35C0E8
:106202001A930A93E091E50BAA81EA17F1F00E9432
:10621200DD670E94256E70F4E0EAEA930E948F66C1
:106222001A930A93E6EEFBE00E94F86DEA81E0938E
:10623200E50B0BC0EFEFE093E50BE6EEFBE00E940F
:10624200FD690E948F660E9461630FC00E94056E05
:106252000E94256E50F4E0EAEA930E948F661A9338
:106262000A93E6EEFBE00E94DB6D1981088123961A
:106272000895E6EEFBE00E94FD690E948F660E948F
:106282006163E881EF5FE093E70B2196089524971D
:106292000E942B77E3EDFBE00E94FD69E8E0F0E06D
:1062A2000E94106AAA85A03438F5AB85A13010F09F
:1062B200A63008F005C0EB850E94466B0E942D6E49
:1062C200EB85E030C9F4E0E0EE83EF83E887E9870D
:1062D20040E050E020E030E02530E0E03E0754F4BA
:1062E200F9010E942D6E0E9446690E94486E2F5F3E
:1062F2003F4FF2CF0E945D6E4AC11A930A93AB815F
:10630200A13010F0A63008F01DC0EB810E94466B50
:106312000E9457740E945374DF010E94DD67AE0F22
:10632200BF1FE8E0F0E00E94A574E050FA4E8F0132
:10633200E0EAEA930E946E6E1A930A93E3EDFBE0A1
:106342000E94DB6D198108810C949B360E942D7787
:10635200EC810E94206BE83119F40E94347730C23C
:106362000E94B16B309729F00E94B16B0E94BB6B07
:10637200EC830E9458190E2F10E0101710F00C94A5
:1063820010320E94736E83DFA5EDBBE00E94EB68C2
:10639200A091D70BB091D80B8091D90B9091DA0BC9
:1063A2000E94086A0E9467740E943A74E093D70BB5
:1063B200F093D80B6093D90B7093DA0B0E94736E33
:1063C2009CDFE0EAEA93EE810E94466BEE0FFF1F2C
:1063D200E050F04F0E94FC6DE270F9F4ED81E09321
:1063E200DB0B0E94B16B309761F40E9489690E94B5
:1063F200026AEF5EF84DDF010E94E067EA0FFB1FC1
:1064020002C00E94B16BE093DC0BF093DD0BE091D4
:10641200DD07F091DE070E94786E1F5FAECF0E940B
:106422003477CEC11A930A930E940D6AECE2F0E02F
:106432000E94106A0E94EF6C0E947E6E10E010347F
:1064420008F51A9334DEE091D807EA931A931FDF16
:106452000E94876EEA0FFB1F0F010E94876E0E9447
:10646200016DDF01CB01E091D70BF091D80B609168
:10647200D90B7091DA0B0E943A74D0010E945375C5
:106482001F5FDDCFA091D007A330B9F500E0003146
:10649200A0F50E9426670E948F6E69F510E01A30FF
:1064A20050F5E02FE05DEA93E0EFF9E10E94946E8F
:1064B200E12FE05D0E949B6EE1F40E94A06E0E94BB
:1064C200FA6CEA0FFB1FFF93EF930E94FA6C0E9493
:1064D200016D7F936F93FF93EF930E94CA58AF9120
:1064E200BF918F919F910E943A74AF91BF910E9488
:1064F20053751F5FD4CF0F5FCACF10E01A3090F4EC
:106502000E94FA6C0E94016DA091DF07B091E00732
:106512008091E1079091E2070E943A740E947E6E98
:106522001F5FECCF09911991089524970E942B7750
:10653200EA85EA9342DD9F01022E032A19F13A937A
:106542002A9358DD1E2F40E050E0E0E0EE83EF8317
:10655200E887E987AA851A1791F4012F003478F4A5
:106562000A932BDD2E173F0741F4EB85EA930A933A
:106572008EDE0E9446690E94486E0F5FEFCF0E9436
:106582005D6E05C0EB85EA93EB85EA9380DE0E949F
:1065920032772C9608951A93A895A981A63088F48B
:1065A200E3EDFBE00E94FD69E8E0F0E00E94106A82
:1065B20010E0103430F4E981EA931A939EDE1F5FF3
:1065C200F8CF1881229608951A9311E0163020F41C
:1065D2001A93E1DF1F5FFACF66C3E1E0E093EB0BB2
:1065E200E093EC0B76C3A8950E942469E2E0F3E005
:1065F200FA93EA930E946E6E0E94A36EE093720B6E
:106602000E94AC6EE093730BE0E0E093740B61C305
:10661200A895E0E4FBE00E94FD69E9E2F0E00E9457
:10662200106A0E94156DE8EFF2E0FA93EA930E9475
:106632006E6E0E94A36EE093490B0E94AC6EE093D3
:106642004A0BE0EBE0934F0B44C30E942B770E946E
:106652009969E03228F0AEE0B0E0E0E00E948B758C
:1066620000E062DCA091750BB091760BA633E2E1FB
:10667200BE0741F110E01A3030F41A93B4DF1A93D6
:1066820075DD1F5FF8CF10E0103430F41A93C0DFCD
:106692001A9336DD1F5FF8CF10E0103830F41A93EA
:1066A2009CDF1A93A1DD1F5FF8CF8EDFA9E0B0E077
:1066B200E0E00E948B75E6E3F2E1E093750BF09364
:1066C200760B01E010E0183210F00C94CE330E94E9
:1066D200D0670E94B36E9F010E94D0670E94B36E82
:1066E200AF010E94D0670E94BB6E3496E491E03005
:1066F20011F0E13089F4D901AC910E94D0670E9477
:10670200BB6E3596E491EA1730F40E94D0670E947E
:10671200BB6E0E94C06E3FC0E230B9F4DA010E9443
:106722004975E031A7E2FA072CF4DA010E944975B3
:10673200FF2352F40E94D0670E94BB6E36960E94DD
:106742005875DA01ED93FC9326C0E33059F4D90170
:10675200AC91AF3F31F40E94D0670E94BB6E0E94A1
:10676200C06E19C0E430B9F4D901AC91AF3F99F4CD
:1067720000E00E94D0670E94BB6E3596E4910E172E
:1067820050F40E94D0670E94BB6E0E94C06E2F5FC1
:106792003F4F0F5FEECF1F5F96CFC9DB10E0133084
:1067A20060F41A932DDDA091E60BA43020F01A9329
:1067B20060DD1A934BDD1F5FF2CFE02F0E9432772C
:1067C20026960895E881EF5FE883A881A43610F049
:1067D200E0E0E883E8817DC20E94C56E309679C20E
:1067E200A091EE0BBB27E091ED0BA4C0F9DF32972D
:1067F20074F00E94CC6EE091ED0B0E94D36E0E9469
:10680200DB6DE091ED0BEA93DDDFE093ED0B089594
:106812000E94CC6EE091EE0B0E94D36EFA93EA9343
:106822000E94E3610895EBEDFBE00E94DB6E0E94A3
:10683200CC6EE091EE0B0E94D36E0E94DB6DE09174
:10684200EE0BEA93BFDFE093EE0B08950E942D77E3
:10685200E0E0E093ED0BE093EE0B10E030E0343635
:1068620080F5A8950E94CC6E3A93B6DFFA93EA932C
:10687200EBEDFBE00E94F86D00E0A091DB0BA13094
:1068820010F0A03808F001C001E0E12FE03041F43F
:10689200013029F43093EE0B3093ED0B11E00FC071
:1068A200E13031F4003019F43093ED0B12E007C0FF
:1068B200E23029F4013019F43093EE0B13E03F5F1C
:1068C200CECF36C21A93A091860BA870B9F010E011
:1068D200E981FA810E94E966AE17BF077CF4ED8177
:1068E200E093DB0BEB81FC81E851FC4F0E94E26EEE
:1068F200E0E0F0E00E94786E1F5FEACF18810C940E
:106902006439E881EF5FE883A881A43610F0E0E003
:10691200E883E881DEC1E881E150E883A881A436FA
:1069220010F0E3E6E883E881D4C1A091F00BBB2725
:10693200E091EF0BF0E031960E94CA6AEC59FF4FEA
:10694200DF01E4E6F0E00E94027508950E94C56E40
:10695200E050FE4FBEC10E94E76EE881EA93B3D1D8
:10696200B8C11A9310DBE1E0E0933D0B9CC1A895FE
:1069720010E0143680F41A939FD1A091E00BAF3F40
:1069820031F40E94EA6EAF3FEFEFBE0711F01A93A7
:10699200E2DF1F5FEECF0E94EF6E689420F883C1A2
:1069A2000E942D771091F00BAD81AA23C2F5E091E0
:1069B200EF0BE11719F0AD81AA230AF02FC01A9349
:1069C2007BD10E94EA6EEE81FF81EA17FB0729F470
:1069D200E885A091E00BEA1709F01DC00E94786BD0
:1069E200EC81FD810E943F74EA17FB0754F40E9478
:1069F2009C6D0E94F56E0E94D26BE0E0EC83ED8309
:106A020008C00E949C6D0E94F56EEC83FD830E947B
:106A1200926B1A9358D10E94FA6EC9CF48C0E09186
:106A2200EF0BE11729F0AC81BD810E9421770CF0B8
:106A32001DC01A9341D10E94EA6EEE81FF81EA17CE
:106A4200FB0729F4E885A091E00BEA1709F00BC0D7
:106A52000E949C6D0E94F56E0E94D26B1A9333D1F4
:106A6200E0E0EC83ED830E94FA6ED9CFAC81BD8168
:106A72000E9421771CF459DF33970CF418C0E88583
:106A8200E093E00BEE81FF810E94B66BEC81FD8109
:106A92000E94D26BE091EF0BEA9315D1E091EF0BDC
:106AA200EA932FDFE093EF0BE0E0EC83ED83689451
:106AB20020F8EC81FD810E9434770C94FD381A9302
:106AC200A0911A0CA03061F4E0911D0CF0911E0C03
:106AD200FA93EA93E8EBFBE00E94196CE03009F4C8
:106AE2000BC0E1E0E0931A0CE091EF0BE0931C0C79
:106AF200E091EF0BE0931B0CA0911A0CA13011F066
:106B02000C94DD35E091F00BA0911C0CEA1711F406
:106B12000C94CE35E0911C0CEA93FDDEE0931C0C44
:106B2200EA93CAD0A091E00BA13010F0A03808F08F
:106B32002DC0E0911B0CEA93EEDEE0931B0CA091BA
:106B42001C0CEA1711F1EA93BED0E091990BE030E8
:106B5200B1F410E0133098F40E948B6D41F00E9462
:106B62003F6DE081AE2FE0911C0CEA1709F005C0E1
:106B72000E943F6DA0911B0CA0831F5FEBCF0E9470
:106B8200E76EE0911C0CEA939ED006C00E94E76E6D
:106B9200E0911C0CEA9397D00FC0E0911B0CE0939C
:106BA200F00BE0E0E0931A0C689420F80E94FB627C
:106BB200E0931D0CF0931E0C76C01A93A8951091C9
:106BC200F00BE091EF0BE117A1F00E94686B54F417
:106BD200EB81A091E00BEA1729F40E94EA6E0E9471
:106BE200FF6E09F003C0E12F1881A4C00E94FA6E63
:106BF200E8CFEFEF18819EC00E94786B0E94217748
:106C020084F4E0911006E87031F4E091E507A09178
:106C1200E00BEA1731F40E94AC6B0E94BB6BE034CC
:106C220008F002C0E1E00895E0E008950895A89513
:106C3200E091EF0BA881EA1759F0E8810E94506DAC
:106C420011F0E88146C0E881EA935BDEE883F0CF89
:106C5200EFEF3FC01A93A8951091F00BE091EF0B64
:106C6200E117C1F00E94686B7CF4E0911006E870B5
:106C720031F4E091E507A091E00BEA1729F40E94B4
:106C8200EA6E0E94FF6E09F002C0E12F04C00E946A
:106C9200FA6EE4CFEFEF1881239608951A931091BC
:106CA200F00B1A93C4DF19910895E881EA9329DE63
:106CB200E883EA93BCDF0DC00E94CC6E0E94046F91
:106CC2000E94F86D06C00E94CC6E0E94046F0E9462
:106CD200DB6D219608950E942D770E94EF6E10E0E1
:106CE20030E0343628F5A8953A93E6DF00E0A0912B
:106CF200E00BA03808F401E0E12FE03041F401306C
:106D020029F43093F00B3093EF0B11E00FC0E13018
:106D120031F4003019F43093EF0B12E007C0E23087
:106D220029F4013019F43093F00B13E03F5FD9CF0F
:106D32000E9434772496089524970E942D770E940A
:106D4200A144E4EFF9E10E94FD690E9440450E94DE
:106D5200DA44E091D807E03061F0EFEFF9E10E9408
:106D6200FD690E944045E091D8070E940D6F0E9484
:106D7200116F0E94DA440E94133200E00A30A0F43C
:106D82000A930E9498300E942469EFE0EA930E94DD
:106D92001A45E02FAAE5B6E00E94156F0E94016D28
:106DA2000E94196F0F5FEACF0E94EE44E8E0FAE119
:106DB200FA93EA93EFE0EA930E9440450E940C693D
:106DC2000E94F7440E94DA440E94F0440E94DA448E
:106DD20010E0103110F00C947F370E948969E1179E
:106DE200E9F5EEE0FAE10E94FD690E9440450E9449
:106DF200D067FA93EA930E94116FE0E0E093D5071F
:106E0200A091D507A03440F5E091D807EA93E0912C
:106E1200D507EA930E9496320E9446693097C9F0DC
:106E2200E091D507EA930E9458300E944669FA938E
:106E3200EA930E941F6F0E9440450E94156DEAE08E
:106E4200EA930E941A450E944F690E94F7440E94E9
:106E5200DA440E945A69D4CF0E94246F0E94D067FC
:106E62000E948F6E11F00C947D37EEE0FAE10E94E1
:106E7200FD690E9440450E94D067FA93EA930E94FE
:106E8200116F0E94286FE0E30E949B6E29F40E941A
:106E9200A06E0E949B589F0100240216030654F51F
:106EA2000E94E66C0E94CA58EC83FD836E837F8346
:106EB2000E94E66C0E94306F3A932A930E941F6FE1
:106EC2000E9440450E94346FEAE0EA930E941A450C
:106ED200EC81FD816E817F810E94196F0E94286F73
:106EE200E1E30E949B6E29F40E94A06E0E949B58CF
:106EF2009F01D2CF0E94246F1F5F6BCF0E94B544C7
:106F02000E943477289608950E942D77AD81BE8124
:106F12002C910E94396F0E94D0670E942E670E94B6
:106F22001268ECE3EA930E94FF5CEC81EA930E9410
:106F32005D5D2A93ED81EA930E949A43EEE3EA9320
:106F42000E94FF5C0E94F66B0E942E670E94FC6BFF
:106F52000E943E6F333409F431E2313320F0EC8188
:106F6200E05DE31708F407C0E32F0E945E6CE25570
:106F7200FF4FE4912E273D3311F0313209F401C065
:106F8200CACF3D3319F4AD81BE812C93E32F0E9409
:106F92003477279608950E942B7720E0AF81B88539
:106FA2005C910E94396F0E94D0670E942E670E94F6
:106FB2001268E2E0EA930E945D5D5A930E94F143F7
:106FC2000E94F66B0E942E670E94FC6B0E943E6F2D
:106FD200303310F03A3308F00EC0203009F450E09C
:106FE20021E0A52FEAE00E94FF74AAE0EA9FF001E7
:106FF200E30FE0535E2F3B3211F4533608F001C029
:107002005F5F3D3211F4513008F401C05150333406
:1070120029F4203009F431E250E020E03D3319F444
:10702200EE81E51708F005C0AF81B8855C9130E0CC
:1070320020E03D3311F0313209F401C0B4CF3D33C9
:1070420019F4AF81B8855C93D4C00E942B7720E0FD
:10705200AF81B8854D915C910E94396F0E94D067D3
:107062000E942E670E941268AE81A23051F4E6E0BF
:10707200EA930E945D5DFA010E9421680E94C74363
:1070820008C0E5E0EA930E945D5D5A934A930E942C
:10709200D3430E94F66B0E942E670E94FC6B0E94F3
:1070A2003E6F303310F03A3308F020C0203011F434
:1070B20040E050E021E04031E7E25E0734F0DA01DF
:1070C200E0E1F7E20E940275AF01493BEBE05E07A7
:1070D20034F0DA01E8EEF3E00E940275AF01DA0162
:1070E2000E94436F0E94486FD097AD013B3221F45A
:1070F2004033E5E75E070CF002C04F5F5F4F3D3261
:1071020021F40024041605060CF002C04150504040
:10711200333431F4203009F431E240E050E020E031
:107122003D3311F0313209F401C098CF3D3321F4DF
:10713200AF81B8854D935C935CC00E942B770E940F
:10714200396F20E050E04FEF0E94D0670E942E6717
:107152000E94F767EF81F885FA93EA93E885EA934C
:107162000E942D5DE52FE10FF0E00E942E670E9444
:10717200FC6B0E943E6F303310F03A3308F021C0AE
:107182003053431729F04F3F09F05F5F20E005C0FD
:10719200A22FAF5FEA2FE3702E2FE52FAF81B885C4
:1071A2000E944D6F0F01E32FA8EEB5E00E94156F0C
:1071B200AE0FBF1FE22F0E944D6FE491D001EC93FE
:1071C200432F3B3219F4EE815E1708F002C05F5F75
:1071D2004FEF3D3211F4513008F402C051504FEFDD
:1071E200EE815E1720F4313211F03D3309F401C013
:1071F200ABCFE32F0E943277299608951A930A9310
:10720200A091510BECEDEA231E2F00E00D3040F46B
:107212000E94516F0E94556FE11711F00F5FF6CF78
:107222000E94516FEA0FFB1F0E9458750E949466DC
:10723200E02F3DC4A1E5BBE0E8810E945A6F11F442
:10724200E3E701C0E9E4EA930E94FF5C3AC40E94CA
:107252002B770E94396F0E94D0670E942E670E948E
:10726200F767CCDF5E2F0E94F66B0E942E670E94AA
:10727200FC6B0E943E6F3D3211F0363311F45030F8
:1072820009F401C051503B3211F0333311F45C3038
:1072920008F001C05F5FA091510BE1E0EA232E2FBD
:1072A200E52FA0E0B2E00E94156F0E94556FE20F39
:1072B200E093510B3D3311F0313209F401C0CBCFD1
:1072C200E32F0E943277269608950E942D770E941E
:1072D200396F0E94D0670E942E670E94F7670E9452
:1072E200606FAE0FBF1FEC91E17019F4EBE1FAE1B0
:1072F20002C0EFE1FAE1FA93EA930E94165D0E945E
:10730200F66B0E942E670E94FC6B0E943E6F303328
:1073120010F03A3308F00EC00E94606FEA0FFB1FB4
:107322000F010E94606FAE0FBF1FAC91E1E0EA2730
:10733200D001EC933D3311F0313209F401C0C9CFD1
:10734200E32F0E943477259608950E942D770E949C
:10735200636F0E94696F0E9498660E946D5D0E9431
:10736200156DEAE0EA93E9DEE13209F45CC40E94B9
:1073720098660E9498660E94216CE3E2FAE10E94FC
:107382009466ECE4FBE00E94FD695FDEE13209F401
:107392004AC40E9498660E9498660E94216CE9E2A3
:1073A200FAE10E949466E0914E0BEF5F0E2FEDB76B
:1073B200FEB7FA93EA930F93EAE0EA93ECDD0F91BA
:1073C200E13209F430C400240216030624F4E02F4B
:1073D200E150E0934E0B0E9498660E9498660E94CC
:1073E200216CE2E3FAE10E949466E3E6FBE00E948C
:1073F2006D6F09F418C40E9498660E9498660E94F4
:10740200216CE8E3FAE10E949466E5E6FBE00E9463
:107412006D6F09F408C40E9498660E9498660E94E3
:10742200216CEEE3FAE10E949466E0E5FBE00E9443
:10743200766F09F4F8C30E9498660E9498660E94CB
:10744200216CE7E4FAE10E94946601DFE13209F47B
:10745200EAC310E0133010F00C94E03A0E949866F0
:107462000E9498660E94216CE12F0E94256CEDE437
:10747200FAE10E9494660E947E6F0E946D5DA4E50F
:10748200BBE00E94D0670E94826F09F4CCC3E9E09E
:10749200F0E00E94F3660E946D5DA7E5BBE00E94EA
:1074A200D0670E94826F09F4BEC30E9498660E9450
:1074B20098660E94216CE12F0E94256CE8E5FAE1B2
:1074C2000E9494661A9301DFE13209F4ACC30E9470
:1074D2007E6F0E948C6F49F40E94FD6A0E94416A8D
:1074E2000E94966F09F49FC30AC00E94FD6A0E941F
:1074F200416A0E94FD69A9DDE13209F494C30E9448
:1075020098660E9498660E94216CE12F0E94256C69
:10751200EAE5FAE10E9494660E947E6F0E946D5D28
:10752200A0E6BBE0EE27A10FBE1F2C913327EDB7DB
:10753200FEB73197FA93EA933F932F93E0E0EA93F1
:1075420084DD2F913F91E13209F46DC3A0E6BBE0E7
:107552000E94D067EA0FFB1F2083123070F50E9451
:1075620098660E9498660E94216CE12F0E94256C09
:10757200E1E6FAE10E9494660E947E6F0E946D5DD0
:10758200A7E6BBE0EE27A10FBE1F2C913327EDB774
:10759200FEB73197FA93EA933F932F93E0E0EA9391
:1075A20054DD2F913F91E13209F43DC3A7E6BBE0E0
:1075B2000E94D067EA0FFB1F20831F5F4BCF33C3AC
:1075C2000E942D7710E01A930E947D6C0E94696FD1
:1075D2000E9498660E949E6F0E94B16B0E941D6875
:1075E2000E9498660E948A660E946D5D0E94086AE7
:1075F2000E9421680E94B1430E94AA6F0E948A667B
:107602000E946D5DE091650BF091660B0E9421680E
:107612000E94B1430E9498660E943068E8E6FAE14F
:107622000E949466E0914E0B0E94AF6F0E94AA6F77
:107632000E943068E3DD0E944B69E091500BE0301C
:1076420029F0E091500BEA930E94F14300E00330ED
:10765200C8F50E949866E02F0E9471670E946D5DD6
:107662000E942D6BEA930E94F143EBE2EA930E949F
:10767200FF5C0E94346BEA930E94F1430E944B69C3
:107682000E943B6B51F40E94436B0E9416680E9459
:1076920021680E94C743E3E707C00E94436B0E9430
:1076A20016680E941D68E9E4EA930E94FF5C0E944A
:1076B2004B690E94506BEA930E94F7430E94B36F9A
:1076C2000F5FC5CF0E94A1453E2F3B3211F410340B
:1076D20008F001C01F5F3D3211F4113008F401C0FF
:1076E20011503D3439F41A930E9458302EDE1A9309
:1076F2000E948130313209F066CF95C20E942D7707
:1077020010E00E94925D012F0E9498660E94986686
:107712000E946D5DECE6FAE10E94946631E036303B
:1077220020F5103800F50E9498660E940D670E94AD
:1077320012681A930E94C130E12F0E94AF6F0E941B
:107742004B69A091EB0BE3E00E94B76FA091EC0BA9
:10775200E7E00E94B76FE0911006EA93E8E0EA934F
:107762000E949A4313953F5FDACF0E94620E0E94F5
:10777200A1453E2F3D34F1F50E94DC6B102F1038ED
:10778200C8F51A930E94C1300E9498660E949866BA
:107792000E94216CE0E8FAE10E949466E12F0E94C7
:1077A200AF6F0E94BC6F0E94C06F0E946D5DE3E8E4
:1077B200FAE10E949466EBEEFBE0FA93EA93E3E0CF
:1077C2000E94C46F09F42FC20E94C06F0E94216CF4
:1077D200E9E8FAE10E949466ECEEFBE0FA93EA93A0
:1077E200E7E00E94C46F09F41EC21A930E94F530AA
:1077F2001F5FC5CF313211F0103808F001C081CFC0
:1078020012C20E942D770E94925D0E94696F0E94AF
:1078120098660E946D5DEFE8FAE10E94946610E0BE
:10782200133008F51A930E9401310E9498660E9453
:1078320009680E941268E12F0E94AF6F0E94BC6F1C
:10784200E091E60B0E94C96FE091E90B0E94C96FBB
:10785200E091E70B0E94C96FE091E80BEA930E9466
:10786200F7431F5FDDCF0E94A1450E2F0D3411F0AB
:107872000C94813C0E94DC6B10E0133010F00C94ED
:10788200813C1A930E9401310E9498660E94986678
:107892000E94216CE2EAFAE10E949466E12F0E94C2
:1078A200AF6F0E94BC6F30E0343028F50E94C06F89
:1078B2000E94216C0E940D670E94CD6F0E94587534
:1078C2000E9494660E946E6E0E948A660E94216CDB
:1078D2000E940D670E94CD6F32960E94D8670E9467
:1078E2000D670E94CD6F3596E4910E94C46F09F432
:1078F2009AC13F5FD9CF1A930E9427311F5FBDCF34
:1079020092C11A930A930E94636F00E0083210F04A
:107912000C94583D0E94570E0E9498660E949866E9
:107922000E94D26F0E94BB6E0E94587531960E94CF
:1079320094660E944B690E946E6E0E948A660E9443
:10794200D26F0E94BB6E3496E491E038A9F40E9493
:1079520089691E2FEDB7FEB7FA93EA931F93E0E110
:10796200EA9319DB1F91E13209F4A1C0E12FA9E0EA
:10797200B0E00E948B7597C0E238A9F40E94996921
:107982001E2FEDB7FEB7FA93EA931F93E0E1EA9355
:1079920002DB1F91E13209F48AC0E12FAEE0B0E0D0
:1079A2000E948B7580C0E138E1F40E94B16D1E2FF8
:1079B200EDB7FEB7FA93EA931F93E3E0EA93EBDAAB
:1079C2001F91E13209F473C00E94570E0E94B16DFB
:1079D200E11731F0E12FA8E0B0E00E948B75FFCFF4
:1079E20062C0E03069F40E9426670E94BB6E329644
:1079F2000E94D867E1E00E94C46F09F458C053C0E6
:107A0200E13079F40E9426670E94B36E0E942E67CD
:107A12000E94BB6E3596E4910E94C46F09F447C080
:107A220042C0E23069F40E9426670E94BB6E329621
:107A32000E94D867EFE0EA9308DBE132C1F133C07C
:107A4200E330E9F40E9426670E94BB6E3596E4910A
:107A5200ABE00E946F75EA1B0E940D6F0E948A665E
:107A62000E94D26F0E94B36E0E942E670E94BB6E6C
:107A72003596E491EA9348DAE132C9F014C0E43071
:107A820091F40E9426670E94B36EE0931F0CF0935C
:107A9200200C0E942E670E94BB6E3596E491EA93F9
:107AA2004CDBE13221F00E94982F0F5F2FCF09911A
:107AB20019910895E8810E94256CE6E2FAE10E949C
:107AC2009466219608951A930E94DC6B10E013309D
:107AD20010F00C94BC3D0E9498660E9498660E9429
:107AE200216C1A93E7DFECE0F0E00E94F3660E945B
:107AF2006D5D1A939FDB0E947E6F0E948C6F49F42A
:107B02000E94FD6A0E94416A0E94966F09F464C352
:107B12000AC00E94FD6A0E94416A0E94FD6995DACC
:107B2200E13209F459C3123020F50E9498660E948E
:107B320098660E94216C1A93BDDFE5EAFAE10E9481
:107B42009466ECE0F0E00E94F3660E946D5D0E9494
:107B5200B36FEAE0F0E00E94F3660E946D5DA7E673
:107B6200BBE00E94D067EA0FFB1F0E94766F09F408
:107B720033C31F5FACCF30C30E942D7710E01A933E
:107B82000E947D6C0E94696F0E9498660E949E6F9F
:107B920021E000E0033060F50E94D367E22F0E94EB
:107BA200A26B0A9387DF0E943B6B49F40E94436BEE
:107BB2000E9416680E9421680E94C74306C00E9464
:107BC200436B0E9416680E941D680A9333DB2F5F85
:107BD200023060F40E94AA6FE22F0E94A26B0E9400
:107BE200496B0E942E680E94B36F2F5F0F5FD2CF46
:107BF2000E94A1453E2F3B3211F4103408F001C01F
:107C02001F5F3D3211F4113008F401C011503D34B0
:107C120039F41A930E94583056DF1A930E94813029
:107C2200313209F0ACCF0E943477249608950E9435
:107C3200DC6B0E9498660E9498660E946D5DEBEA7A
:107C4200FAE10E949466E1E0E093D807E8EDF7E0FC
:107C5200FA93EA93E5E0EA939ED9089522970E9467
:107C62002B770E94A1450E2FE091D207E03011F050
:107C72000C94DD3F0132D1F4EEE6F5E0A091F10B78
:107C8200B091F20BEA17FB0761F4E7E0E093CF074C
:107C9200EAE2EA93E4EBFAE10E94FD690E94875A64
:107CA200D9C1E0E0E093BB050E94D66F0D3331F4F9
:107CB200E091BB05F0E00E94316704910D3441F47C
:107CC200EAE2EA93E7EBFAE10E94FD690E94875A31
:107CD200063449F4E6E9F5E0E093F10BF093F20B98
:107CE200E0E0E093BB05003311F00B3229F4E091A0
:107CF200BB05EF5FE093BB050D3229F4E091BB05B4
:107D0200E150E093BB05013329F491DFED3311F427
:107D12000E94DD6F033321F48ADFED3309F40CD8BE
:107D2200063329F4E0E0E093D8070E949D3604333D
:107D320029F4E0E0E093D8070E94DD6FA091DA0712
:107D4200A13010F40C94753F023301F570DFED336E
:107D5200E9F40E94EA6FD1F4E091D807EA930E9415
:107D6200CC3230E0303190F40E940D670E948F6E69
:107D720059F4E32FE05DEA93EAEBFAE10E94946E94
:107D8200E0E3EA930E94A85A3F5FECCF053331F556
:107D9200E0E0E093D8070E94EA6F01F511E01630A7
:107DA200E8F41A930E94CC3230E03031A8F40E94F9
:107DB2000D670E948F6E71F4E32FE05DEA93EAEBA8
:107DC200FAE1FA93EA93E12FE05DEA93E0E3EA93C2
:107DD2000E94A85A3F5FE9CF1F5FE1CF013451F4FF
:107DE200EAE2EA93EDEBFAE10E94F46CE1E0E0935F
:107DF200CF0730C10A3409F4BFDE073311F00C9407
:107E0200753F0E94925DE0E0EA930E94B70EE1E0C6
:107E1200E093D307E0E0F0E0E093CB07F093CC07E8
:107E2200E4E1F6E00E94FD69E5E4F0E00E94106AF8
:107E32000E94FB62EE83FF830E94F36F0E94C5687B
:107E42000E940763E030B1F00E9432120E94FB628E
:107E5200EE83FF83A091D00BA03021F00E941B2C57
:107E6200E03009F407C00E946A69EF56F84FAEE0AD
:107E72000E947069E5E0F0E0FA93EA930E94BD4542
:107E820040E050E00E94481BE03868F00E94481B26
:107E9200EF573E2F313010F0313108F004C0E32F9C
:107EA2000E94DC69AF015A934A930E94F0184093F2
:107EB200CB075093CC070091D605E0E0E093D605BE
:107EC200013211F00B3209F401C0B6CF0B3221F4AA
:107ED200E1E0EA930E94B70E013209F0A1CFE0E09F
:107EE200E093D307E093D605A091DA07A23011F010
:107EF2000C94D63F093309F404DD053409F481DC1E
:107F0200083309F45DDB023409F4F8DB0334B9F514
:107F12001091F00B0E94925D00E0E091EF0BE117EF
:107F220011F0063008F01EC00E9498660E94266773
:107F32000E9412681A930E945D361A930E94F143BE
:107F42000E944B69E091E00B0E94C96FE091E30B44
:107F52000E94C96F0E94AC6B0E941D680E94FA6E5B
:107F62000395DBCF0E94620E0E94A1450E2F0132C3
:107F720021F0E091EF0BE11709F401C0CBCF0434FB
:107F8200A1F40E94EA6F89F4A0918A0BA03021F437
:107F9200A091880BA03039F0E0E0EA930E94986645
:107FA2000E9498665FD30E94B234E091D207E0301B
:107FB20011F40E94E90E49C0E130D1F4A091D70733
:107FC200AB3010F4013209F405C00E94EC150E9496
:107FD200620E0DC0E0E0E093D5070E94F86F0E94A8
:107FE200F46CE0E00E94FD6FE2E0E093D2072DC066
:107FF200E23059F5013269F4E0E0E093D2070E94E1
:10800200925DEAE2EA93E7EBFAE10E94F46C0E94E5
:10801200E90E0B3211F00D3359F40E94F86FFA9306
:10802200EA93E1E3EA930E94875AE1E00E94FD6F3E
:108032000D3259F40E94F86FFA93EA93E2E3EA935D
:108042000E94875AE2E00E94FD6FA091CF07A33001
:1080520009F407CE0E943277289608951A93E3E036
:10806200E093D0070E94925D0E9498660E949866F3
:108072000E946D5DE3ECFAE10E9494660E949866AC
:108082000E948A660E946D5DE8EFF5E00E94FD693C
:10809200E0E1F0E00E94106A10E0E091800B1E1710
:1080A20000F50E948969E117D1F0E12FE05DEA93C2
:1080B200EBECFAE1FA93EA93E0E3EA93E0E00E9460
:1080C2009B6E49F40E94D067E850FA4FA1E0A0836A
:1080D200E12FE05D01C0EEE2EA930E94FF5C1F5FC8
:1080E200DCCF0E94D66FE0E0E093BB05E093D207BD
:1080F2000E94E90E71C00E940270E89422F80E9468
:10810200066DE2E7EA930E945A59E091F107EA9379
:108112000E945A59EFE0EA930E945A59A091EE0741
:10812200AA3221F41A930E94754B1BC0A091F10749
:108132000E94D067E55EF44FE081EA1721F4E091F6
:10814200F107E03351F40E94E966A55EB44FE09175
:10815200F107EC931A930E94754B22FC02C00E9415
:10816200455A3AC00E940270E091F107E053AE2FE7
:108172000E94D067E45DF44FE081EA1769F51A9333
:108182000E94754BA091EC07A23019F40E940A706C
:1081920009F402C00E941070A091EC07A33019F4F8
:1081A2000E940A7009F402C00E941070E0E0E0939D
:1081B200EC07E093230C0E94D067E45DF44FBF010B
:1081C2000E94D067E45DF44FE081EF5FAE2FEAE0FA
:1081D2000E94FF74DB01EC9319910895E881E0306D
:1081E20029F4E0E3EA930E945A5906C0E881E85074
:1081F2000E940D6F0E948B590C949F440E942B7712
:1082020025FC2DC20E940A7011F40C9483420E9434
:108212001670E057F84F9F01D9011196EC91E430A6
:1082220041F50E941C70F901A681A03021F4A281BF
:10823200B381109709F007C0E4EDFAE10E940B6DDB
:108242000E94367015C00E943A700E943D700E94D2
:108252004170E7EDFAE10E940B6D0E9444700E94AA
:108262004A70F901A085B185BA93AA930E948B59ED
:1082720014C0E730C9F40E941C70EAEDFAE10E94D2
:108282000B6D0E9444700E944170EDEDFAE10E9474
:108292000B6D0E943D700E948B59D9010E94507053
:1082A2000E94327726960895E93089F40E941C7064
:1082B200E0EEFAE10E940B6D0E9456700E9441703E
:1082C200D9010E9450700E9432770C94DD45E6304D
:1082D20031F5EAE2EA930E942A5AE3EEFAE10E94B9
:1082E2000B6DD901EC910E945970E091840B0E94B0
:1082F2005970EBE4EA930E945A590E943D700E9421
:108302008B59E4E5EA930E945A590E9444700E94F4
:108312005D700E9410700E9432770C94DD45E5304A
:1083220021F50E94AC6CF096EA930E942A5AE2E789
:10833200EA930E945A59D901EC91EA930E945A5940
:108342000E9461700E943D700E944170E1EDFAE16D
:108352000E940B6D0E9444700E948B59D9010E94A9
:1083620050700E9432770C94DD45E83031F50E945E
:108372001C70E6EEFAE10E940B6DF901A681AA9348
:108382000E94B86C309719F00E94B16B04C0D901F9
:108392001696EC91F0E0FA93EA930E948B590E94B0
:1083A20036700E94455AD9011196E0E0EC930E9482
:1083B20010700E9432770C94DD45E130B1F5A09146
:1083C200D007A53029F4E091840BE65F1E2F01C08F
:1083D20011E0E12F0E9466700E94D0670E946E70C9
:1083E2000E9461700E943D700E944170E9EEFAE1C4
:1083F2000E940B6D0E9444700E944A70D901179628
:10840200EC910E940D6F0E948B59A091D007A5306C
:1084120041F40E947270A481B581BA93AA930E941A
:10842200FF590E9478700C94DD45E330B9F40E9444
:10843200AC6CF0960E9489700E94AC6C0E946E70C7
:108442000E949070ECEEFAE10E940B6D0E94447063
:108452000E945D700E9494700C94DD45EB3071F5C2
:108462000E94A3700E94A6700E949070EFEEFAE143
:108472000E940B6DF901A681AA93B0DE0E94727070
:10848200A781AA93ABDE0E947270A085B185BA93D0
:10849200AA930E944A700E9444700E944A70F90195
:1084A200A481B581BA93AA930E944A700E94567021
:1084B2000E945D700E9494700C94DD45EC3091F442
:1084C2000E94A3700E94A6700E949070E2EFFAE1EF
:1084D2000E940B6D0E9456700E945D700E94947003
:1084E2000C94DD45EE3071F40E94A3700E94A670D8
:1084F2000E949070E5EFFAE10E940B6D0E94787085
:108502000C94DD450E94AA7061F0A091EC07A030A6
:1085120041F4A091890BA13021F40E948969E130D4
:1085220009F427C0A0913C0BA03041F0E0913E0B32
:10853200F0913F0B0E94D66CE130D9F4E1E30E9446
:108542008970E0912D0B0E9459700E9490700E94D8
:108552008969EA930E94244BE093EC070E94455AF2
:108562000E94FB62E093210CF093220CE0E0E09386
:108572003C0BA091EC07A03051F0E091210CF0915E
:10858200220C0E94D3680E940763E13009F025C0E3
:10859200A091EC07A23019F40E940A7009F402C0FB
:1085A2000E941070A091EC07A33019F40E940A7087
:1085B20009F410C0A091230CA33030F00E94107077
:1085C200E0E0E093230C06C00E941670EF56F84FCD
:1085D200A8E0A083E0E0E093EC07A0913D0BA1307E
:1085E200F1F5E091F00BA091EF0BEA1799F1EAE2B5
:1085F2000E948970E0912B0B0E9459700E9490702A
:10860200E091F00BEA930E945D360E943A70E0918D
:10861200E00B0E940D6F0E944170E8EFFAE10E94A8
:108622000B6D0E94AC6BFA93EA930E944A700E940F
:108632009C6D0E94B0700E94455AE091F00BEA9343
:108642000E94AC34E091F00BEA930E948234E093F2
:10865200F00B05C0E0E0E0933D0B689420F80E9427
:108662003277AAC21A930A930E941B2CE030D9F0E7
:108672000E946A69E057F84F8F01EC81FD81D801B1
:108682001296ED93FC93EA81FB81D8011896ED9343
:10869200FC93EE81D8011696EC93D8011196E4E092
:1086A200EC930E94E66A198108810C944546E881A0
:1086B200E03011F40E94B370A881A13021F4E0E10E
:1086C200F6E00E94BA70A881A23021F4ECE1F6E053
:1086D2000E94BA70A881A33021F4EAE2F6E00E9477
:1086E200BA70A881A43021F4E0E3F6E00E94BA70E7
:1086F20025C10E94B37008951A930A93E0E0E093B3
:108702007805E093790510E0143190F400E003302D
:1087120068F4A3E01A9FF001E158FA4FDF01EE2757
:10872200A00FBE1FE0E2EC930F5FF1CF1F5FECCF13
:10873200E2C31A9311E0E981E11788F00E94D06741
:10874200E255FF4FE491AA81EA2319F0E12FE05D9F
:1087520001C0E0E2EA930E94FF5C1F5FECCF3AC1E6
:108762002A97A091D20BA13040F0EA85FB856C8557
:108772007D850E945C750AD008C00E94BF700E946D
:10878200C3700E94BF700E94075D44C12A970E9475
:10879200BF700E94CE700E94D7700E94BF700E946C
:1087A200075D38C12A970E94BF700E94EA700E943A
:1087B2007F6D0E94BF700E94075D39C12A970E9497
:1087C200BF70E7E1FBE1FA93EA93EE85FF850E9431
:1087D20021680E947F6D0E94BF700E94075D27C1C1
:1087E2002A970E94BF70EAE1FBE105C02A970E9426
:1087F200BF70EEE1FBE1FA93EA93EE850E94686DA9
:108802000E94BF700E94075D2B9608950E942D77EB
:1088120010E0E1E3E093EE08E89431F8EA930E9475
:108822002A5AE2E2FBE10E940B6D00E0E0917D0535
:108832000E17E0F40E942667E158FA4FE081E03219
:1088420058F4E3E2EA930E945A590E942667E158DB
:10885200FA4FE081E05D05C00E942667E158FA4FB9
:10886200E081EA930E945A590F5FE0CF0E94455A75
:108872000E94FB629F010E946E153A932A93E8ECD4
:10888200F0E00E94196C0E2FA0E031FCA1E0A030B4
:1088920011F4003009F001C0EECF31FE07C0E0E074
:1088A200E0937D05E89431F8E1E007C01F5F1230E4
:1088B20008F4AFCFE0E0E0937D050E943477249680
:1088C2000895E0917C05E03021F4E881EA930E946A
:1088D2000E56A0917C05A13079F4A0E09299A1E016
:1088E200A13031F4A8950E94CA680E942A74F5CF7B
:1088F200E881EA930E94AD57A0917C05A230F1F481
:10890200E0917D05F0E0E158FA4FA881A083E09163
:108912007D05EF5FE0937D05E0917E05EF5FE093DB
:108922007E05A03218F4EF5FE0937E05A0917E05EC
:10893200A83320F06BDFE0E0E0937E0521960895F6
:10894200A091800BA13020F0E2E0E0937C050BC007
:10895200E1E0E0937C05E0919A00EF76E0939A00E3
:10896200E3E3E093990008950E94246F0E94246F2C
:1089720020D0EBE1EA93A5DFE9E6EA93A2DFA0913A
:108982007C05A13051F40E94D668E0919A00E0691A
:10899200E0939A00E9E1E0939900A0917C05A2306E
:1089A20021F434DFE0E0E0937E05E0E0E0937C0533
:1089B2000895EDE0EA9385DFEAE0EA9382DF089525
:1089C2001A9310E0E9811E1728F4EA81EA9379DF0D
:1089D2001F5FF8CF188123960895EDE201C0EDE301
:1089E200EA93E8E2EA93ECDFE4DF08952A97A091A4
:1089F200D20BA13038F00E94BF700E94CE700E944C
:108A0200D77004C00E94BF700E94C370FE010E9412
:108A1200FD690FD02E9608952A970E94BF700E947A
:108A2200EA700E947F6DFE010E94FD6902D02C96C1
:108A320008951A930A9310E0EA81E03011F408E2F3
:108A420001C00A81AB81BC81EE27A10FBE1FAC9190
:108A5200A03011F0101708F007C0AB81BC810E9452
:108A6200F2702FDF1F5FEECFEA81E03039F0EA814A
:108A72001E1720F4E0E20E94F870F9CF27C01A9383
:108A82000A9310E0EA81E03011F408E201C00A81A1
:108A9200E12FAB81BC810E944D6FE491E03011F077
:108AA200101708F009C0E12FAB81BC810E944D6F05
:108AB200E4910E94F870ECCFEA81E03039F0EA816B
:108AC2001E1720F4E0E20E94F870F9CF19810881A4
:108AD20025960895E091BF05A091BE05EA17C1F061
:108AE2000E94FD700E94396AEC91E093C1050E94D8
:108AF200FD700E94416AE181E093C005A091BF052B
:108B0200AF5FEAE00E94FF74E093BF05E1E00895E1
:108B1200E0E008950E940371A981A0830E9403717D
:108B22003196A881A083A091BE05AF5FEAE00E94C2
:108B3200FF74E093BE050C94734BE091D605089543
:108B42001A93E091D605E03059F40E946E150E9406
:108B5200EC6A21F4A091D605A03009F001C0F5CF4E
:108B62001091D605E0E0E093D6050E94EC6A09F088
:108B720011E2E12F0C94E94A0E942D770E94FB62D8
:108B82008F010E946E15EC81FD81E00FF11FFF93B2
:108B9200EF930E94FB62AF91BF91AE1BBF0B9D0191
:108BA2000024021603061CF40E94EC6A09F001C0BC
:108BB200E8CFE0E00E943477269608951A930E9447
:108BC200D269E050FD4FA0E0A0830E94D269E55F28
:108BD200FC4F108117FF05C0E12F0E940971A0E030
:108BE200A08316FF05C0E12F0E941071A0E0A083B0
:108BF2000E94D269E55FFC4FA0E0A0830E94D26987
:108C0200E65FFC4FA0E0A0830C94724B0E942D778C
:108C120030E0EE81ADE0EA9FF001E55FFC4F1081AC
:108C220016FF17C0E12FEF730E2F0E94177111F07C
:108C32003A3008F009C00E941F71DF010E940D67DF
:108C42000E9425713F5FF1CF0E941F710E94486F01
:108C5200EC9317FF17C0E12FEF730E2F0E941771CD
:108C620011F0343108F009C00E942B71DF010E941B
:108C72000D670E9425713F5FF1CF0E942B710E9408
:108C8200486FEC930E94347727960895A0970E942C
:108C92002B77EDA5FEA5A9A9BAA9EA0FFB1FAF0183
:108CA200E0E0F3E0EE83FF8310E01431C0F5AE8123
:108CB200BF81AC91A03049F1EE81FF81A381B481E3
:108CC200EFA5F8A9EA17FB0701F5EE81FF81A18163
:108CD200B281E9A9FAA9AE17BF07BCF0EE81FF8104
:108CE200A181B2814A175B0784F00E943171AE0FF5
:108CF200BF1FE9A9FAA9AE17BF073CF00E94317164
:108D0200AE0FBF1F4A175B070CF402C01A9356DF5F
:108D1200EE81FF813D96EE83FF831F5FC6CFE0E0C9
:108D2200F3E0EE83FF8310E0143110F00C943C4723
:108D3200AE81BF81EC91E03011F00C943547EAA589
:108D4200EC93E9A9FAA9AE81BF811196ED93FC9348
:108D5200EFA5F8A9AE81BF811396ED93FC93EDA523
:108D6200FEA5AE81BF811596ED93FC93EBA5AE8176
:108D7200BF811796EC93E0910404A0910A04EA27BC
:108D8200AE81BF811896EC93E0910B04AE81BF8156
:108D92001996EC93E0910C04AE81BF811A96EC9384
:108DA200AE81BF811B960E9484671C96E0E0EC9323
:108DB200E887E8A5F9A5309741F00E943C710E942E
:108DC2004171E4E1EA930E94C063EEA1FFA13097F2
:108DD20051F00E943C71E8A5F9A5FA93EA93E4E107
:108DE200EA930E94AC63E0E0EC8F0E943C710E9427
:108DF20097633E2F3B30C8F000E00E942B71E08168
:108E0200E03011F0053008F002C00F5FF6CF0E948B
:108E12002B71E081E03049F40E942B710E9446716F
:108E2200E058AE81BF811B96EC93E0E0EA8B3130D3
:108E3200C8F000E00E941F71E081E03011F00431BF
:108E420008F002C00F5FF6CF0E941F71E081E03090
:108E520049F40E941F710E944671E05CAE81BF819D
:108E62001B96EC93E12F08C0EE81FF813D96EE83C5
:108E7200FF831F5F59CFEFEF0E943277E396089589
:108E82001A930A930E9451713097A9F1E0915D05FE
:108E9200E03061F50E945171049000925D05E0910D
:108EA2005D05E03031F4E0E0F0E00E94BA70E0E00D
:108EB2001AC00E9456710E9451710E945875F59510
:108EC200E7958F01D801E0E0F1E00E94D074E093D1
:108ED2008700D801E0E0F1E00E940275E09386008D
:108EE2000E945671E0E4E0938B0005C0E0915D05BD
:108EF200E150E0935D050991199108950E942D7743
:108F020000E020E033E010E01431B8F5D901EC9133
:108F1200E03079F111960E9449750E945E7124F544
:108F2200D90113960E944975AC81BD81EA17FB07EE
:108F3200DCF4F90101801280D90115960E9449756D
:108F4200E00DF11DAE81BF81AE17BF076CF4F901D0
:108F520003801480D9011796EC910E94F26AAC81C9
:108F6200BD81AE17BF070CF004C0E12FEF5F0E2FDB
:108F720004C0235F3F4F1F5FC7CF003049F0E0912D
:108F82005E05E01721F0A0915E05A03009F401C052
:108F920022C0A0915F05A53079F40A93E1E0EA933B
:108FA200B9DD00935E0500936005D901EC91E09371
:108FB2006105E3E0E0935C05A0915F05AE3119F431
:108FC200E4E0E0935C05A0915C05A33018F0E5E0D5
:108FD200E093630507C0E0E0E0935F05E0935C0582
:108FE2000E9463710E94347728960895E0915E058D
:108FF200E03091F0A0915F05A93220F4EA93E2E01B
:10900200EA9388DDA0915F05AD3330F0E0915E0513
:10901200EA93E4E0EA937EDDE0E0E0935C05E0932E
:109022005F050E946371E0E0E0935E05E0936205F4
:1090320008950E94925D60DB0895E981EBBBE7E150
:10904200E09365001F98E6E1E0936500E7E1E093B5
:109052006500E881EBBBEFE1E0936500EEE1E093B0
:109062006500EFE1E09365001F9A0C94734B1F9823
:1090720008951F9A08950E94CA680E942A74EBE11B
:10908200E0936500EAE0F0E00E948569EFE1E09399
:1090920065000E9426680E942A74E1E0EA93E2E0F9
:1090A200EA93CBDF0E94B16621F4E2E0EA93E2E4C4
:1090B20003C0E2E0EA93E2E8EA93BFDFE7E0EA9383
:1090C200EFE7EA93BADFE8E0EA93E7E1EA93B5DF94
:1090D2000E946971E1E2EA93E8E8EA93AEDFE2E234
:1090E200EA93E3E3EA93A9DFE3E2EA93ECECEA939F
:1090F200A4DFE4E2EA93ECECEA939FDFE5E2EA9391
:10910200EBEBEA939ADFE6E2EA93EBEBEA9395DF85
:10911200E7E20E946F71E8E20E946F71E9E20E9449
:109122006F71E5E0EA93E8E0EA9387DFE6E0EA932D
:10913200E7ECEA9382DFE0E0F0E00E947471E0E0A5
:10914200F0E0E0935A05F0935B050E94FA66E3E0D3
:109152000E940067E0E0E0930D04EDE0E0930E046E
:10916200089521970E942B774A85EF810E94797199
:109172000E9458758F01E0E1EA93EF85EA935DDF83
:10918200E2E1EA93EB85FC85AF85B889EA0FFB1F24
:10919200EA9353DFE9E00E947D71E1E1EA930E94E4
:1091A2008271EA0FFB1FEA9348DFE9E1EA93EF8558
:1091B2000E9487710E947D715ADF2EE13FE1E0E05B
:1091C200EE83E885F985AE81B0E0EA17FB079CF0F3
:1091D20050E0451760F01BBB20936500309365009B
:1091E2000BBB20936500309365005F5FF2CFEE8189
:1091F200EF5FEE83E6CF0E943A48E0E10E948C7175
:10920200E2E1EA93EFE9EA930E941E48E9E00E9454
:109212008C71E1E1EA93EFE7EA930E941E480C9415
:10922200184A0E942B77EE810E9479710E9458752C
:109232008F010E948271EA17FB0739F4EF81F885EA
:10924200AB85BC85AE17BF070CF023C0E7E10E94D7
:109252008C71E7E10E948C71E9E1EA93EE850E944C
:1092620087710E9491712EE13FE15B854F81451725
:1092720060F01BBB20936500309365000BBB20930D
:109282006500309365005F5FF2CF0E943A480E940A
:1092920069710E948271AE17BF073CF4EF81F885B5
:1092A200AB85BC85EA17FB0709F01BC0E9E1EA932D
:1092B200EE850E9487710E9491712EE13FE15D85EA
:1092C2004985451760F01BBB20936500309365000C
:1092D2000BBB20936500309365005F5FF2CF0E9465
:1092E2003A480E9432772F96089524970E942B774E
:1092F200EB85F0E0EE0FFF1F0E945374E887F987B9
:1093020030910804EA850E9479710E9458750E9482
:109312005C741E2FEA850E9479710491E0E0EF836C
:10932200AF81A03110F00C94184AE0E0EE83E09196
:109332000904AE81AE1710F00C940E4AE8E10E94C7
:109342007D7140E0423010F00C94044AE42FEE0F9D
:10935200EE0FEE0FE39FF001AE85BF85F0E0EA0F5E
:109362005E2FE42FA885B9850E944D6FE659F94F0B
:109372002491203011F40C94014A27FF3BC0E9E10B
:10938200EA935A930E941E481F98EFE1FEE10BBB3D
:10939200F0936500E09365001BBBF0936500E093DA
:1093A200650031FF0AC00BBBF0936500E0936500D6
:1093B2001BBBF0936500E093650026FF1AC00BBB50
:1093C200F0936500E09365001BBBF0936500E093AA
:1093D200650031FF0BC00BBBF0936500E0936500A5
:1093E2001BBBF0936500E09365005F5F220F5F5F38
:1093F200E4CF1F9A220F31FD5F5F5F5F0C94BA4981
:109402004F5F0C94A349EC85FD853196EC87FD876F
:10941200EE81EF5FEE830C949849E885F9853296E8
:10942200E887F987EF81EF5FEF830C9491490E94FF
:1094320032776096089523970E942B77A895E98545
:109442000E9479710E9458750E945C740E2FE98502
:109452000E947971149130910804E0E0EF83EA856B
:10946200AF81AE1710F00C94BE4AE0E0EE83E091BB
:109472000904AE81AE1710F00C94B94AE8E10E94DB
:109482007D71E0E0E887EB85A885AE1710F00C94BB
:10949200AF4AE885F0E00E945574DF010E940D6733
:1094A2000E94A574AE85BF85EA0FFB1FAF01E88954
:1094B200F98924913196E88BF98B203011F40C94C0
:1094C200AA4A27FF3DC0E9E1EA934A930E941E4857
:1094D2001F98EFE1FEE10BBBF0936500E09365009E
:1094E2001BBBF0936500E093650031FF0AC00BBB24
:1094F200F0936500E09365001BBBF0936500E09379
:10950200650026FF1CC00BBBF0936500E09365006D
:109512001BBBF0936500E093650031FF0CC00BBBF1
:10952200F0936500E09365001BBBF0936500E09348
:1095320065004F5F5F4F220F4F5F5F4FE2CF1F9A71
:10954200220F31FF02C04F5F5F4F4F5F5F4F0C949E
:109552005E4AE885EF5FE8870C94444AEC85FD8516
:109562003196EC87FD87EE81EF5FEE830C94384AEB
:10957200EF81EF5FEF830C94304A0E94327762965C
:109582000895E091F80AEA930E945A59E091F90A83
:10959200EA930E945A590895F4DF0E9498710E943A
:1095A2009871E881F9810E94B0709CC01A930E9460
:1095B2009B581E2F103021F0E12FE150E093F60A64
:1095C200E0DFE091F60AEF5F0E940D6F0E944170AA
:1095D200199108950E942D7731E00E94E06CA0332A
:1095E20020F00E94E06CA43308F028C030E00E9412
:1095F200A271E270E6951E2F0E94A271E1700E2FF9
:10960200A091100B1A1729F4E1E0EA27E093100B5E
:1096120031E0A091110B0A1729F0E1E0EA27E0936B
:10962200110B31E0E091110BEE0FE05DA091100BF8
:10963200EA0FEA930E945A590E94E66CE32F0E94B5
:109642003477249608951A9310E00E94AA7011F4B8
:109652000C94714B0E940934E6E2FBE10E940B6D0F
:10966200E091DB0B0E940D6F0E944170E9E2FBE189
:109672000E940B6DE091DE0BF091DF0B0E94B07047
:10968200A091DC0BB091DD0BA031E7E2BE074CF4F8
:10969200ECE2FBE10E940B6DE091DC0BF091DD0B43
:1096A20018C0EFE2FBE10E940B6D0E94AC67A4E6DA
:1096B200B0E00E94A574A091DC0BB091DD0BEA0F23
:1096C200FB1F0E94E26EE091DC0BF091DD0BE0519A
:1096D200F742FA93EA930E948B590E94367011E086
:1096E200E12F18812296089524970E942B770E94D9
:1096F200A871E0E0EC930E944458E13010F40C941D
:10970200714EE091F80AEB3441F4E091F90AE33248
:1097120019F40E949B581E2FE0C2E435B9F4E0917F
:10972200F90AE33221F40E949B58EE83FF83E09111
:10973200F90AEF3451F40E949B581E2F1A93EF81BD
:10974200F885FA93EA930E94AE2FC7C2E23411F071
:109752000C94FF4CE091F90AE13269F4AA85AF3F1B
:1097620041F4E0E0EA930E9498660E9498660E94A3
:1097720033430E94B234E091F90AE134E1F40E94E9
:109782009B581E2F113071F4A091EC07A13019F4EF
:109792000E94AA7009F402C00E941434E0E0E0932F
:1097A2003C0B09C0E1E0E0933C0B0E94FB62E093BA
:1097B2003E0BF0933F0BE091F90AE534A9F4E2E3A2
:1097C200FBE10E940B6D0E94F133F3973CF00E9483
:1097D2009B580E94E26E0E94AD7101C0E0E3EA93E1
:1097E2000E945A590E943670E091F90AE63411F546
:1097F2000E94B97119F40E949B58AF01E885F9855E
:109802000E94BB6B0E2FE0919C0BE03011F0109187
:109812009C0B003420F0A0918A0BA13021F40E940D
:10982200C5710E94D134AA85AF3F21F40E94C5714F
:109832000E943343E091F90AE23511F00C94BC4CDA
:109842000E94B97119F40E949B58AF0130E0A091B7
:109852008A0BA03021F40E948969E13009F027C007
:109862000E94212CE03011F10E94C66BE55AF84F9C
:10987200A885B985A083B1830E94C66BEF59F84FC2
:10988200DF01EA850E94E26A0E94C66BE15AF84F44
:1098920010830E94C66BE05AF84F40830E94C66B49
:1098A200E65AF84FA1E0A0830E94CC6B62C00E94EE
:1098B2001B2CE23010F40C94BA4C1A930E94CD7116
:1098C2000E94DE353E2F3F3F29F00E94786BA4179D
:1098D200B5070CF412C00E949C6DE41BF50B0E94AC
:1098E200D26B0E94876B19F4E0E0E093E00B3A93AD
:1098F2000E946436689420F803C0E0E0E887E987B4
:109902000E946A69E057F84FDF01EA85F0E0E55E00
:10991200F44FE081EC930E946A69EE56F84FA885F5
:10992200B985A083B1830E946A69E856F84FDF01C6
:10993200EA850E94E26A0E946A69EA56F84F108339
:109942000E946A69EF56F84FA5E00E947069E885A7
:10995200F985309771F01A930E94CD71FA010E9435
:109962003F74FA93EA930E9433430E94C5710E94A6
:109972006334689422F8E091F90AE335F1F50E9424
:109982009B58E887F9870E941670EF56F84FE081DE
:10999200E23089F40E941670E856F84F0080118078
:1099A2000E9489690E94936AEA17FB0721F4A09139
:1099B200EC07A23009F01FC00E941670EE56F84F55
:1099C200DF010E944975DF01E885F985EA17FB0787
:1099D20079F40E941670E656F84FE081EA930E94ED
:1099E2001670E057F84FE081EA930E94132003C0FB
:1099F200E7E0E0930906689422F86FC1E43411F0BD
:109A02000C94694DE091F90AE33559F4E5E3FBE181
:109A12000E940B6D0E9434560E945970E1E0E0935F
:109A2200EF08E091F90AE03511F00C94684D0E94BC
:109A3200D27111F40C94684D20E00E94E06CA032C7
:109A420040F00E94E06CA23221F00E94E06CAB3345
:109A520009F43DC0E22FE03061F40E94E06CA332D1
:109A620011F421E005C00E94A271EA930E940E56F1
:109A72002BC0E13049F40E94E06CA43211F422E0E0
:109A820001C020E010E020C0E23011F0E330E1F448
:109A92000E94A271EA930E94D362EF3FA1F0E12FEC
:109AA200E295E07FEF930E94A271EA930E94D36253
:109AB200AF91EA0F1E2F2F5F243021F41A930E94D8
:109AC2000E5620E001C020E00E94E66CB6CF05C130
:109AD200E33411F00C94D94DE091F90AE534B9F46C
:109AE200E2E3FBE10E940B6D0E94F133F3974CF02D
:109AF2000E949B58E05FF84D0E94E26E0E94AD7199
:109B020001C0E0E3EA930E945A590E943670E09144
:109B1200F90AE634D9F441E050E00E949B580E2F36
:109B22000E94D871E13019F40E949B58AF01E09174
:109B32009C0BE03011F010919C0B1A930E94266747
:109B4200E05FF84D0E94DC710E94D134E091F90A85
:109B5200E335A1F40E94E1710E94206BE83141F4E7
:109B6200E091400BEA930E94532F689420F806C0BC
:109B7200E885EA93EFEFEA930E941320E091F90A55
:109B8200E134A9F4E8E3FBE10E940B6D0E94E1716C
:109B9200EA930E9458300E94411FE03011F0E1E345
:109BA20001C0E0E3EA930E945A590E94367095C0C0
:109BB200E63511F00C94464EE091F90AE33411F0C7
:109BC2000C94454E0E949B581E2F113010F40C9499
:109BD200454EA091D007A13011F0A930C1F50E94E5
:109BE200D871E03021F0A09159061A1709F02EC061
:109BF20011500E949B58AF011A930E94E41A3E2F03
:109C02000E94296C0E94416A0F010E94296C0E94E5
:109C12001668E40FF51FD001ED93FC930E94D871F2
:109C2200E03089F00E949B58AF010E94326C0E9482
:109C3200416A0F010E94326C0E941668E40FF51F00
:109C4200D001ED93FC931A930E94EE111DC01630C1
:109C5200D8F41150A12FEAE00E94AF74A3E2EA9F68
:109C6200F001E15AF94FBF01A12FEAE00E94FF740F
:109C7200F0E0BB01AAE0B0E00E947D74DB01AE0F10
:109C8200BF1F14960E94A96928C0E93431F5E091FA
:109C9200F90AE03551F40E949B581E2FE0E0EA9346
:109CA2001A930E942B30E0931306E091F90AEC34E8
:109CB200A1F40E945D58E0930D060E94D871E03035
:109CC20021F00E945D58E0930E060E94D871E030A8
:109CD20021F00E945D58E0930F060E94F8570BCDC9
:109CE2000E9432772B960895A0910E0BA03521F495
:109CF200A0910F0BA03408F005C0E0910F0BEA937E
:109D02000E948130A0910E0BA33521F4A0910F0B7C
:109D1200AA3008F005C0E0910F0BEA930E94B73019
:109D2200A0910E0BAB3421F4A0910F0BA03808F0D8
:109D320005C0E0910F0BEA930E94F530A0910E0B43
:109D4200A63521F4A0910F0BA03108F005C0E091D7
:109D52000F0BEA930E942731A0910E0BA43511F448
:109D62000E94982FE2D60895EAE5F6E0FA93EA9384
:109D7200E091F80AEA93E0E8F0E00E94106A0895A0
:109D82000E94E871A0E0A083E091F60AE0930F0B35
:109D9200E091F80AE0930E0B08950E942B770E943F
:109DA2004458E13010F40C940452E0910E0BA0914F
:109DB200F80AEA1709F098DFE091F80AE33239F578
:109DC200E091F90AEC3431F4CFDFE4E0E093CF071D
:109DD2000E94EE71E091F90AE435C1F4C5DFE09129
:109DE200260CE03029F0EF77A9E0B0E00E948B75F5
:109DF200E091270CE03029F0EF77AEE0B0E00E946E
:109E02008B750E94EE71E7E0E093CF07F9C2E93467
:109E1200E9F4E091F90AE434C1F40E94D271A9F0A4
:109E220010E010E0183178F4AAEDB6E00E94D06795
:109E3200EA0FFB1FFF93EF930E945D58AF91BF9112
:109E4200EC931F5FEFCF0E941F0EDAC2EB34E1F5F5
:109E5200E091F90AE13211F487DF35C0E53211F4FD
:109E620043DF31C0E33299F40E94F47121F00E9481
:109E7200FF710E94C1300E94E871E081EB3429F445
:109E8200E0E0E093EB0BE093EC0B7ADF1CC0E134F3
:109E9200D1F40E949B589F012093EB0B0E94057204
:109EA20091F00E949B589F01A091EB0BF901E27087
:109EB200F070EA2BE093EB0B0E94057221F00E94F6
:109EC2009B58E093EC0B9CC2E33581F5E091F90AD3
:109ED200E13211F449DF29C0E33299F40E94F471AE
:109EE20021F00E94FF710E9498300E94E871E08187
:109EF200E33529F4E091F60AEA930E94F43240DF56
:109F020014C0EE3491F40E94306F10E01A3068F4FD
:109F1200AAE6BBE0EE27A10FBE1F0E94D067E65063
:109F2200F54FE081EC931F5FF1CF6AC2E63511F085
:109F32000C94E34FE091F90AE13211F415DF41C0CC
:109F4200E33299F40E94F47121F00E94FF710E94A1
:109F520001310E94E871E081E63529F4E091F60AC8
:109F6200EA930E943A310CDF2CC0E63531F40E94AC
:109F72009B589F012093E70B24C0E53471F40E94A3
:109F82009B589F012093E60B0E94057229F00E94C4
:109F92009B589F012093E90B14C0E43591F440E0F3
:109FA20050E00E949B589F01022E032A11F042E0CA
:109FB20050E00E94057219F00E949B58AF01409335
:109FC200E80B1EC2E43511F00C94B850E091F90A86
:109FD200E33231F40E949B583197E093F60AC6C0EF
:109FE200E03511F00C94B75010E00E94E06CA03202
:109FF20050F00E94E06CAD3331F00E94E06CAB3364
:10A0020011F01E3008F00DC00E94D067E650F54FE7
:10A012000F010E94A271D001EC931F5F0E94E66CB7
:10A02200E4CF0E94D0670E940B72EDE30E9410728F
:10A0320011F00C94B750E4E5E0930E0B10E00E948F
:10A04200D0670E94BB6E3496E491EF3F11F40C94FA
:10A05200B750EAEFFAE00E94E9670E94BB6E0E94E5
:10A06200D8670E946F63E03011F00C94B5500E94E3
:10A07200D0670E94BB6E3496E491E03851F40E949E
:10A082009B58E058FF4FE093260CE0E8E093270C42
:10A092006BC0E23839F40E949B58E058FF4FE093BE
:10A0A200270C62C0E13839F40E949B58A8E0B0E066
:10A0B2000E948B7559C0E03011F0E13061F40E94CA
:10A0C200D0670E94B36EFF93EF930E949B58AF91AB
:10A0D200BF91EC9349C0E23069F40E94D0670E94BC
:10A0E200B36EFF93EF930E949B58AF91BF91ED9394
:10A0F200FC933AC0E33061F40E94D0670E94B36ED1
:10A10200FF93EF930E947C58AF91BF91EC932CC0C8
:10A11200E43051F50E94D0670E94BB6E3596E491FF
:10A12200EA930E9432590E94D0670E94B36EE09374
:10A13200240CF093250C00E00E94D0670E94BB6EB5
:10A142003596E4910E1780F40E942667E650F54F8B
:10A15200E081A091240CB091250CEC93A4E2BCE028
:10A162000E94EB680F5FE8CF1F5F69CF49C1E035FE
:10A1720011F00C940152E091F90AE33299F40E9431
:10A18200F47121F00E94FF710E9458300E94E87120
:10A19200E081E03529F4E091F60AEA930E9409335E
:10A1A200EFDD2EC1E13211F4DFDD2AC1E134D1F459
:10A1B2000E949B581E2F00E00D3098F40E94516FB0
:10A1C200EA0FFB1F3396E491E11749F40E94516FA5
:10A1D2000E94556FA091510BEA2BE093510B0F5F38
:10A1E200EBCF0EC1E63559F5E0E0E093F70AA4E5BE
:10A1F200BBE00E941572FF93EF930E949B58AF91B0
:10A20200BF91EC93EBE2EA930E940B58E03059F0D5
:10A21200A7E5BBE00E941572FF93EF930E949B5843
:10A22200AF91BF91EC930E941872A091F70AA330EC
:10A2320018F40E94057209F401C0D9CFE1C0ED34CF
:10A24200D1F4E0E0E093F70AA0E6BBE00E941572C9
:10A25200FF93EF930E949B58AF91BF91EC930E94A2
:10A262001872A091F70AA33018F40E94057209F43B
:10A2720001C0EACFC5C0E735D1F4E0E0E093F70AC8
:10A28200A7E6BBE00E941572FF93EF930E949B58D2
:10A29200AF91BF91EC930E941872A091F70AA2307D
:10A2A20018F40E94057209F401C0EACFA9C0E4348F
:10A2B200C9F5E0E0E093F70A0E949B589F01E2E0B3
:10A2C200EA930E941758AF01E3E70E94107259F413
:10A2D2000E941E72BF01D9010E94DD6AE40FF51FC0
:10A2E200DB01ED93FC93E9E40E94107279F40E9481
:10A2F2001E7220833183A1E5BBE00E9415720F011B
:10A30200A1E5BBE00E9425720E94356C0E94187282
:10A31200A091F70AA33018F40E94057209F401C053
:10A32200CBCF6EC0EE3499F40E94306F10E01A3039
:10A3320068F4A1E4BBE0EE27A10FBE1F0E94D06724
:10A34200E650F54FE081EC931F5FF1CF59C0E33443
:10A3520059F4E2E2EA930E940B580E949B58E09360
:10A362004C0BF0934D0B4CC0E33589F40E949B5883
:10A372009F0100240216030624F42B30E0E03E077E
:10A382000CF004C0F9013197E0934E0B39C0E5356A
:10A3920029F40E949B58E093500B32C0EF3491F4A1
:10A3A2000E949B581E2FECE2EA930E940B58E12F69
:10A3B200E295E07FEF930E949B58AF91EA0FE09302
:10A3C2004F0B1EC0E035E1F4E0E0E093F70AA3E6AC
:10A3D200BBE00E9425720E94416AFF93EF930E94A4
:10A3E2001259AF91BF91ED93FC930E941872A09104
:10A3F200F70AA23018F40E94057209F401C0E7CFEF
:10A402000E94F857CCCC0E943277269608950E947B
:10A412002D770E944458E13010F40C94C254E0911C
:10A42200F80AE332A9F4E091F90AE03519F4EBE312
:10A43200FBE109C0E83419F4ECE5FBE104C0E335C3
:10A4420031F4E7E7FBE1FA93EA930E946A5997C273
:10A45200E934B9F4E091F90AE43491F40E941E0E51
:10A4620090D80E94297210E0183140F4AAEDB6E0AB
:10A472000E94F2700E949B591F5FF6CF0E942972C0
:10A482007EC2E43511F00C94D252E091F90AE43222
:10A4920021F40E94C56880D883C0E33211F486D8C3
:10A4A2007FC0E03511F00C94D1526BD8A091F60A1E
:10A4B200A83210F00C94D1520E942D720E94D867DB
:10A4C2000E946A59EDE3EA930E945A590E942D7242
:10A4D2003496E491E03839F40E9489690E940D6F44
:10A4E2000E948B595DC0E23839F40E9499690E943A
:10A4F2000D6F0E948B5954C0E13839F40E94B16D3E
:10A502000E940D6F0E948B594BC0E03011F0E13078
:10A5120041F40E943172E0810E940D6F0E948B59BA
:10A522003FC0E23041F40E943172DF010E9449755E
:10A532000E94357235C0E33039F40E943172E081F5
:10A54200EA930E94AA592CC0E43051F50E9431725C
:10A55200E093240CF093250C10E00E942D723596A6
:10A56200E4911E1790F40E94D067E650F54F0F0158
:10A57200A091240CB091250CEC91D001EC93A4E2B3
:10A58200BCE00E94EB681F5FE8CF0E942D723596F7
:10A59200E491F0E00E940B720E94346F0E94F55920
:10A5A200EEC1E33579F5E091F60AEA930E9498301C
:10A5B200E091F90AE43229F4EAE0F0E00E9439720B
:10A5C20020C0E33219F40E94D74A1BC0EE34C9F40A
:10A5D2000E94C24A10E01A3058F40E94D067E65036
:10A5E200F54F0F01AAE6BBE00E943D721F5FF3CF59
:10A5F200E0E0E093040B0E94346F0E94F5590E9440
:10A602003670BDC1E63511F00C944453E091F60A60
:10A61200EA930E940131E091F90AE43229F40E949E
:10A62200D3670E94CD4A2EC0E33219F40E94D74A62
:10A6320029C0E53459F40E94C24AE091E60B0E9417
:10A642000D6F0E944472E091E90B19C0E63529F4BE
:10A652000E94C24AE091E70B12C0E43599F40E94CD
:10A66200C24AE091E80BE03011F0E1E301C0E0E31F
:10A67200EA930E945A590E944A72E091E80BF0E074
:10A682000E94B0707CC1E03511F00C948D54E091C1
:10A69200F60AEA930E945830E091F90AE43229F46A
:10A6A200E0E4F0E00E94397236C1E33219F40E940C
:10A6B200D74A31C1E13411F00C94A1530E94C24A2D
:10A6C20012E0A091510BECEDEA233E2F00E00D3099
:10A6D20078F40E94516F0E94556FE31739F40E947B
:10A6E200516FEA0FFB1F3396149102C00F5FEFCF39
:10A6F2000E94D0670E94B070E0914F0BE03089F069
:10A70200E2E9FBE10E940B6D0E94AC6D0E940D6FAD
:10A712000E944472E0914F0BEF700E940D6F0E94F5
:10A722004170E091500BE03051F0E5E9FBE10E940D
:10A732000B6DE091500B0E940D6F0E944170EBC0B7
:10A74200E43479F50E944E72A091F70AA33040F5E5
:10A75200E091F70AE03011F00E944A72A1E5BBE0F5
:10A76200E091F70A0E945A6F61F4AAE5BBE00E94E9
:10A7720025720E941668FA93EA930E94FF59E3E752
:10A7820009C0AAE5BBE00E9425720E9416680E94D9
:10A792003572E9E4EA930E945A590E941872D4CFA2
:10A7A200B6C0ED34C1F40E944E72A091F70AA330F4
:10A7B20088F4E091F70AE03011F00E944A72A0E6B4
:10A7C200BBE00E9425720E9454720E948B590E9423
:10A7D2001872EBCF9CC0E735C1F40E944E72A09173
:10A7E200F70AA23088F4E091F70AE03011F00E94F3
:10A7F2004A72A7E6BBE00E9425720E9454720E9430
:10A802008B590E941872EBCF82C0E63521F50E9467
:10A812004E72A091F70AA330E8F4E091F70AE03013
:10A8220011F00E944A72A4E5BBE00E9425720E94C8
:10A8320054720E948B59EBE2EA930E945A59A7E59F
:10A84200BBE00E9425720E9454720E948B590E94A2
:10A852001872DFCF5CC0EE34C1F40E94C24A10E02D
:10A862001A3058F40E94D067E650F54F0F01A1E468
:10A87200BBE00E943D721F5FF3CFE0E0E093040B68
:10A882000E94346F0E94F55942C0E33499F40E9449
:10A89200C24A0E94346FEDE9FBE1FA93EA930E9407
:10A8A200B16B0E9421680E947F6D0E94346F0E94EA
:10A8B200F5592DC0E03599F40E94C24A0E94086AF7
:10A8C200FA93EA930E94165A0E944A72E091650B2B
:10A8D200F091660BFA93EA930E94165A18C0E33578
:10A8E20031F40E94C24AE0914E0BEF5F0DC0EF348B
:10A8F20091F40E94C24A0E94AC6D0E940D6F0E94A8
:10A902004472E0914F0BEF70F0E00E943572EBE37E
:10A91200EA930E945A5933C0EB3489F5E091F60A62
:10A92200EA930E94C130E091F90AE43229F4E0E8A6
:10A93200F0E00E94397223C0E33219F40E94D74A30
:10A942001EC0E134E1F40E94C24AA091EB0BE1E0A7
:10A95200EA230E940D6F0E944472A091EB0BE3E088
:10A96200EA230E940D6F0E944472E091EC0B0E9458
:10A972000D6F0E948B59E0EAFBE10E940B6D37D309
:10A9820048CDB9C21A930E94196BE6EFF8E00E9413
:10A99200DB6C0E945872E181E43471F40E945872B7
:10A9A20002800E948969E05DE01529F00E945872D8
:10A9B200E281EA3209F401C05BC00E945D720E942A
:10A9C2005872E1810E9461720E945872E2810E9473
:10A9D20061720E9464721C910E94587233960E94A6
:10A9E200DB6CE12FE23139F40E94A8711397E6E0A3
:10A9F200EC93D3D93DC0E13139F40E94A871139789
:10AA0200E2E1EC9304DD34C0EF30B1F40E94A871AE
:10AA12001397EEE0EC930E94EB4AE13039F4A091F7
:10AA2200EB07A03019F00E94AA7009F402C00E943C
:10AA320014340E9469721CC0EE30D1F40E94A871D5
:10AA42001397EFE0EC930E94EB4AE13089F4A09176
:10AA5200EB07A03019F00E94AA7009F402C00E940C
:10AA62001434E0E0E093EB07EFEFEA930E94754BBA
:10AA72000E94A871E0E0EC9347C11A930E94066D10
:10AA82000E94A06EEAE7EA930E945A590E946472F9
:10AA920011971C91E12FE23131F4E6E0EA930E9432
:10AAA2005A597BD937C0E13131F4E2E1EA930E948D
:10AAB2005A59ADDC2FC0EF3099F40E9490700E9479
:10AAC200EB4AE13039F4A091EB07A03019F00E9473
:10AAD200AA7009F402C00E9414340E9469721AC05A
:10AAE200EE30C1F4EFE0EA930E945A590E94EB4A19
:10AAF200E13081F4A091EB07A03019F00E94AA7016
:10AB020009F402C00E941434E0E0E093EB07EA93F8
:10AB12000E94754B0E94A871E0E0EC93A091EE07B1
:10AB2200AA3211F00E94455AEFC0EFEFE0930E0BEC
:10AB3200E0930F0B0895AC81A03310F0AA3308F014
:10AB420006C00E947072E0530E9478729AC2AC8171
:10AB5200A13410F0A73408F006C00E947072E753C7
:10AB62000E9478728EC2A881B981E0E0EC9389C21A
:10AB7200AA93EA93FA93EFB7EA931A930A931BB153
:10AB82000CB1E091600CF0E0E25DF34F0083A09124
:10AB9200600CAF5FA093600CA23319F4E0E0E09385
:10ABA200600C09911991D2C10A921A92FA926A938F
:10ABB2007A938A939A93AA93BA93EA93FA93EFB702
:10ABC200EA930E947D7249F0A091EF08A03021F033
:10ABD2000E94180EE13009F401C011C0E091C70CC7
:10ABE200F0E0EE59F34FE081ECB9A091C70CAF5FF2
:10ABF200A093C70CA43619F4E0E0E093C70CE991E6
:10AC0200EFBFF991E991B991A991999189917991BE
:10AC12006991F9901990099018951A930E947D7282
:10AC220059F45D9B09C0A091EF08A13021F40E9464
:10AC3200180EE03009F013C01091C60C0E94D067C4
:10AC4200EE59F34FA981A0831F5F143609F410E077
:10AC5200E091C70CE117E1F31093C60C02C0E98141
:10AC6200ECB91881F4C30E947D7221F40E94180E7F
:10AC7200E13009F001C01DC24FC0AA93BA93EA9312
:10AC8200FA93EFB7EA931A930A9310919B000091FB
:10AC92009C00E12FEC71A9F4E091900DF091910DDF
:10ACA200E853F34F0083A0E9BDE00E94EB68E83C63
:10ACB200A0E0FA0731F4E0E0F0E0E093900DF093C9
:10ACC200910D09911991E991EFBFF991E991B9912A
:10ACD200A99118951A930E9483720E948872D9F3DF
:10ACE2000E948372E853F34F1081A2E9BDE00E94F3
:10ACF200EB68E83CA0E0FA0731F4E0E0F0E0E09332
:10AD0200920DF093930DE12F199108950E94837291
:10AD12000E94887209F0CDC1E0E008950E942D776B
:10AD2200F5DFE03021F0A091290CA03009F0E3C05A
:10AD3200D1DF1E2FA0919C0DA53618F0E0E0E09324
:10AD4200960D3091960DE091960DE03059F4113048
:10AD520019F4E4E0E093960D1A3519F4EAE0E09371
:10AD6200960DC1C0E430C1F4E0E0E093960D1A32D2
:10AD720029F00E948969E05DE11769F41093EE07FA
:10AD82001093970DE5E0E093960DE0E0E093290C37
:10AD9200E1E0E093990DA7C0E530A9F4E0E0E0938B
:10ADA200960D0E948969E05DE11761F00E948F7241
:10ADB2000E949872E091990DEF5FE093990DE6E0A1
:10ADC200E093960D90C0E63091F4E091990D0E94C7
:10ADD20098720E948F72EF5FE093990DE0E0E0932A
:10ADE2009A0D133019F4E7E0E093960D7CC0E7303A
:10ADF20011F0E83059F41A93EAE9FDE0FA93EA9384
:10AE0200E6E9FDE0FA93EA9396DE6DC0E93081F45B
:10AE1200E0E0E093960D173131F4E0919A0DA091A4
:10AE2200970DEA1709F003C0E4E5E093290C5BC033
:10AE3200EA3041F4103011F4EBE001C0E0E0E093BD
:10AE4200960D51C0EB3071F4E0E0E093990D109350
:10AE5200980D1093970DECE0E093960DE0E0E093EF
:10AE6200290C41C0EC3091F50E949D7210830E9422
:10AE72008F72EF5FE093990DE091980DE150E093AE
:10AE8200980DA091980DA03021F4A091970DA030BB
:10AE920009F00FC0EDE0E093960DE091990D0E944C
:10AEA200466BEA50F74FA0E0A0830E949D72A0E09B
:10AEB200A083A091980DA03021F4A091970DA0300D
:10AEC20009F403C0E0E0E093960D0DC0ED3059F4B3
:10AED200E0E0E093960D1D3031F4EAE5E093290CB1
:10AEE200EFEFE093280CE091960DE31719F0E0E004
:10AEF200E0939C0D15CF0E94347724960895AA936F
:10AF0200EA93FA93EFB7EA93E0919E0EA0919D0E19
:10AF1200EA1791F0E091ED07E03019F0E89426F895
:10AF22000AC00E94A372F0E0E030A1E0FA0719F42F
:10AF3200E0E0E0939E0E03C0E89425F826F8E09145
:10AF4200280CE03019F0E0E0E093960DE991EFBFB4
:10AF5200F991E991A99118951A93E0919E0EA09109
:10AF62009D0EEA1721F4E0919B00E072C1F4E0919A
:10AF72009D0EF0E0E356F24FA981A08310919D0E41
:10AF82001F5F0E94E966A030E1E0BE0709F410E00D
:10AF9200E0919E0EE117E1F310939D0E03C0E9814B
:10AFA200E0939C00188153C2E0E0E0939E0EA091D2
:10AFB2009D0EA13020F00E94A372689426F8089595
:10AFC200AA93BA93EA93EFB7EA93E091280CE030A0
:10AFD20041F4E0E0E0939E0E0E948969EF5FE09306
:10AFE200ED07E991EFBFE991B991A99118950E94F6
:10AFF200E06CA03220F00E94E06CAB3309F403C095
:10B002000E94E66CF4CF0E94E06CAB3311F40E9414
:10B01200E66C08950E94E06CE881EA1729F40E9428
:10B02200E66C3197E1E0F0C4E0E0EEC40E942D77D7
:10B0320000E010E0EEE20E94107201F520E030E044
:10B04200EC81D901F0E0AE17BF07C4F4D8010E9429
:10B05200436F8F010E94E06CA03320F00E94E06CED
:10B06200AA3308F008C00E94A2710E945E6C0E0F03
:10B072001F1F0E94E66C2F5F3F4FE2CFF8010E9434
:10B082003477259608950E94E06CA03228F00E9441
:10B092005872E181E03208F40EC00E94A271E0937E
:10B0A200F80A0E94E66C0E94A271E093F90A0E94DB
:10B0B200E66CE1E00895B2C31A930A9300E010E04F
:10B0C2001230B8F40E94A271EA930E94D362EF3F59
:10B0D20071F0E02FE295E07FEF930E94A271EA9374
:10B0E2000E94D362AF91EA0F0E2F0E94E66C1F5F9F
:10B0F200E7CFE02F1DC31A930A9310E00E946472F7
:10B102000C910B3311F0003208F412C0013310F02D
:10B11200093308F007C0E02F0E945E6CE255FF4F32
:10B12200E4911E2B0E94E66C0E9464720C91E9CF9E
:10B13200E12FFEC20E942D7700E010E00E94E06C39
:10B14200AD3221F40E94E66C31E001C030E00E9491
:10B15200E06CA03320F00E94E06CAA3308F00DC02E
:10B16200D8010E94436F0F010E94A271E0530E9416
:10B17200F26A8F010E94E66CEACF303021F4F801C6
:10B182000E943477CCC4F8010E943F740E94347745
:10B19200C6C424971A93E0E0E983EA83EB83EC8345
:10B1A2000E94E06CAD3221F40E94E66C11E001C015
:10B1B20010E00E94E06CA03320F00E94E06CAA3301
:10B1C20008F021C0A981BA818B819C81EAE0F0E07C
:10B1D20060E070E00E94AA747F936F93FF93EF93F5
:10B1E2000E94A271E053AF91BF918F919F91FF276F
:10B1F200662777270E943A74E983FA836B837C83FC
:10B202000E94E66CD6CF103029F4E981FA816B8175
:10B212007C81E9C4E981FA816B817C810E9443745B
:10B22200E2C40E942D7786DF8F0120E030E0EEE25B
:10B232000E94107211F47EDF9F01112322F4F901A2
:10B242000E943F749F01A091D20BA13030F0D8012F
:10B252000E94DD6AE20FF31F8F01F8010E9434772A
:10B262005EC41A9310E00E94D271E9F00E94E06C71
:10B27200A03258F00E94E06CA23239F00E94E06CD9
:10B28200AB3319F0E9811E1708F00DC00E94D06798
:10B29200E650F54F0F010E94A271D001EC931F5F9F
:10B2A2000E94E66CE3CF0E94D0670E940B72188165
:10B2B200CEC0E8810E946172E881A091120BEA0F70
:10B2C200E093120BE881A091130BEA27E093130B92
:10B2D2009BC31A9310E0E12FA981BA810E944D6F9E
:10B2E200E491E03049F0E12FA981BA810E944D6FCB
:10B2F200E4910E94B172EFCF95C31A9310E00E94BD
:10B30200B67239F0A981BA810E94F270D2DF1F5F52
:10B31200F6CF88C364970E94BF700E94BE72E88D08
:10B32200F98D0E9421680E947F6D0E94BF70E5DF47
:10B332006696089564970E94BF70E9EAFBE1FA936A
:10B34200EA93E88D0E94686D0E94BF70D6DF659611
:10B3520008951A93ECE3EA93ACDF11E0193080F41C
:10B362000E94D067E255FF4FE491A981EA2319F0C8
:10B37200E12FE05D01C0E0E2EA939BDF1F5FEECFC9
:10B38200EEE3EA9396DF188162C064971A930E94F3
:10B39200C3720E94BE72EA8DFB8D0E9421680E94D8
:10B3A2007F6D0E94C3720E9497631E2FED891E1744
:10B3B20020F4E0E30E94B172F9CF0E94C3729DDFD4
:10B3C200188110C064970E94BF700E94BE72E88DFF
:10B3D200F98D6A8D7B8D0E945C750E947F6D0E9443
:10B3E200BF708BDF689608950E942972E881F98107
:10B3F200FA93EA9382DF0E94297229C0A881B98157
:10B40200E4E6F0E00E94D0740E943572EEE2EA9324
:10B4120050DFA881B981E4E6F0E00E940275FA9358
:10B42200EA93E2E0EA93B1DF12C0A091D20BA1301D
:10B4320030F0E881F981FA93EA93E0DF08C0E8810D
:10B44200F9810E943572EEEAFBE10E940B6D2296B1
:10B45200089525FE06C0E5E0F0E00E948569A89502
:10B46200F8CFEDE9FDE0E093140BF093150BE1E06A
:10B47200EA931FDFE0E0E093120B0E94C8720E9481
:10B4820089690E945970C0C21A930A93A091800BD5
:10B49200A03021F40E948969E03009F001C048C15E
:10B4A200E091280CE03009F043C1E3E0EA9301DFC8
:10B4B200E091120BE295EF70EA930E94EA621E2F6E
:10B4C200E091120BEF70EA930E94EA620E2F1A9338
:10B4D200F0DE0A93EEDEE7E1EA93EBDEEDE9FDE072
:10B4E2000E94A8710E946C75EA1BE0939D0E6894FD
:10B4F20025F81EC1EE81EA93ACDFEC81FD810E944A
:10B502000B6D0E94CC725EDFBFDF21C2EB81EA933A
:10B51200A0DF0E94196ADDDE0E94C872B5DFFFC299
:10B52200ED81EA9396DFEB81FC810E940B6DEA814B
:10B53200EA93BFDEE981E03011F0EA93BADEE881F6
:10B54200E03011F00E94C8729FDF269608950E9493
:10B552002B7710E0E2EBFBE1A885B985EA17FB0740
:10B5620019F444E150E002C048EC50E0EA85E0936F
:10B57200EE08E89431F8EA930E94CD71EA85EA93E5
:10B58200EA85EA93E0E0EA93CBDF0E94FB629F0147
:10B592000E946E150E94D3720E9407630E2F31FC27
:10B5A20002C0003009F001C0F3CF31FE04C0E894BC
:10B5B20031F8E1E004C01F5F1230C0F2E0E00E9407
:10B5C20032772B9608951A930A93E091F609E030A8
:10B5D20009F4AEC0E0E0E093EF08E2E0EA931DDB9D
:10B5E20010E003E00E94D0670E94D87271F00E94BE
:10B5F200D067EA50F64F0E94156B0E94D067EA505E
:10B60200F64FE0810E271F5FEDCFE3E0EA9305DB03
:10B61200E02FE295EF700E94DD72E02FEF700E9442
:10B62200DD72E7E1EA93F9DA83C01A930A93E091B3
:10B63200F609E03009F47CC00E949969E03021F0FB
:10B64200E091F809EA3209F405C00E949969E05DC7
:10B65200E093F809E0E0E093EF08EAE5EA93DDDA47
:10B66200E0E0EA93DADA10E00E94D0670E94D87232
:10B6720011F01F5FF9CF1F5F012F0A93CEDA10E09E
:10B682000E94D0670E94D87271F00E94D067EA507F
:10B69200F64F0E94156B0E94D067EA50F64FE08188
:10B6A2000E0F1F5FEDCFE02FE195EA93B6DAEDE0E2
:10B6B200EA93B3DA3DC01A930A93F894E0E0E09378
:10B6C200ED07E0919E0EE0939D0E7894E091F609CD
:10B6D200E03071F1EAE5EA933FDCE0E0EA933CDC3A
:10B6E20010E00E94D0670E94D87211F01F5FF9CF5C
:10B6F2001F5F012F0A9330DC10E00E94D0670E9486
:10B70200D87279F00E94D067EA50F64FE081EA934E
:10B7120023DC0E94D067EA50F64FE0810E0F1F5FD4
:10B72200ECCFE02FE195EA9317DCEDE0EA9314DC2D
:10B732000991199108951A930E94196BE091F107EA
:10B74200EA93B7DDE4E4EA93B4DDE091EF07EA932C
:10B75200B0DD14E00E94D067E251F84FE081E4309E
:10B7620040F00E94D067E251F84FE0810E94B1722E
:10B77200F1CFE0E0EA939DDD58DF19910895CEDA2A
:10B78200A091290CA43529F4A0E025FCA1E0A03069
:10B7920009F03AC0E091F007E03581F4E091F10759
:10B7A200EA93E6E0EA930E948B45A091F107A03864
:10B7B20020F0E091F107E093600523C0E03721F427
:10B7C200E0E0E09360051DC0EA3519F40E943E55A1
:10B7D20018C0EA3711F4AFDF14C0E23519F40E9441
:10B7E2007C400FC0E23719F40E94B3400AC00E94A5
:10B7F200F928E091EF07A091EE08EA1711F4689496
:10B8020031F8E0E0E093290CA091290CAA3531F43B
:10B812000E94C35450DFE0E0E093290CE0E0089579
:10B82200A0912C0CA13050F0E0912C0CE150E0934F
:10B832002C0CE03019F4E1E0E0932D0CA0E025FCA3
:10B84200A1E0A13049F4A0E026FCA1E0A03021F45F
:10B85200A091ED07A03009F001C0A6DBE091ED0751
:10B86200E03019F0E150E093ED070895E0919C0D6E
:10B87200EF5FE0939C0DE0912B0CEF5FE0932B0CBC
:10B88200E091280CE03019F0E150E093280C089583
:10B89200A0919B0BA13041F0A0919B0BA23021F013
:10B8A200A0919B0BA53029F4E1E0E0939000ECE934
:10B8B200E9B90895EA81E0937A05E881E0937B058E
:10B8C200E0910504E061E093050429C10E942B7711
:10B8D200A0917A05A43120F4A0917B05A33008F051
:10B8E20034C0E0917A05F0E0ACE0B0E00E94A574CB
:10B8F2008F01E0917B05F0E0A4E1B0E00E94A57425
:10B902009F010E94E372ECE0F0E00E94E872F0E036
:10B912000E9453740E942B68EE81E030B1F0E091F6
:10B922007A05A3E0EA9FF001E158FA4FDF01E091C6
:10B932007B05F0E0AE0FBF1F4C9155270E94E372CA
:10B942004A93E0E0EA930E9476490E943277279672
:10B952000895E0910504E07141F0E2E0EA93B6DF78
:10B96200E0910504EF7EE093050408950E94ED72D4
:10B97200AF39E0E0BE0744F4A091F50BB091F60BAD
:10B98200AF37E0E0BE070CF037C00E94F2720E94AF
:10B99200736E0E947649A0915805B091590554974B
:10B9A20034F4A0915A05B0915B0513970CF012C0C4
:10B9B200E0915805F0915905A3E0B0E00E947D7432
:10B9C200E158FA4FA0915A05B0915B05EA0FFB1FAF
:10B9D200A981A083E0910804ACE0EA9FF0010E94F3
:10B9E200ED720E944D6F0E94FF72E0915805F09136
:10B9F200590531960E9474710C949461E881EA931E
:10BA0200E0910B04EA93B2DF219608951A9310E0B5
:10BA12000E94B67239F0A981BA810E94F270EEDFFB
:10BA22001F5FF6CF1881239608951A930A9300E0B8
:10BA320010E00E940473E03021F00832E0E01E07BB
:10BA42000CF007C00E940473EA93D8DF0F5F1F4F08
:10BA5200F0CF1981088163C01A930A9300E010E0C5
:10BA6200F801AB81BC810E940B7331F0EA81D801ED
:10BA7200F0E0AE17BF070CF009C0F801AB81BC8142
:10BA82000E941073BBDF0F5F1F4FEACF198108813D
:10BA9200ABC00E942D770E94ED72EFE9F0E0EA1B45
:10BAA200FB0B31978F010E9415730E94E3720E9473
:10BAB200A7660E94347733C00E942D77AC810E9422
:10BAC2001D730E2F11270E9415730E94E3720E94AC
:10BAD200A7660E94347788C0EA81FB810E94747154
:10BAE200E881F981E0935A05F0935B05AA81BB8155
:10BAF200ECE0F0E00E94A5740E94FF72A881B98177
:10BB0200E4E1F0E00E94A57406C0EA81FB810E9494
:10BB1200FF72E881F981E093F50BF093F60B24961E
:10BB220008950E942573143128F41A930E94DF4568
:10BB32001F5FF9CF0E9498660E9498660E949D66D8
:10BB4200EFE7F0E00E942B6810E0153048F4A5E121
:10BB52001A9FF001E551FB4FA0E0A0831F5FF5CFD4
:10BB620010E0143148F4ABE01A9FF001E15FFB4FA3
:10BB7200A0E0A0831F5FF5CFE0910504EF7EE09384
:10BB820005040C9432610E9425731431E0F40E9482
:10BB92002D73DF01EB81FC81AE17BF0774F00E94A9
:10BBA2002D73DF010E94FF6E44F0ADE01A9FF00199
:10BBB200E55FFC4FE081E03009F403C01A930E9474
:10BBC200DF451F5FE2CF0E949866ED81FE81FA9306
:10BBD200EA930E949D66A985BA85EF81F885EA1BE2
:10BBE200FB0B0E942B68188125960895A2970E944C
:10BBF2002B77E9A5ADE0EA9FF001E050FD4F8F0100
:10BC0200D8011B96EC91E03009F403C2D8011B96CF
:10BC1200EC91E9A3E07859F0FE013696FA93EA93A3
:10BC2200EBA10E940971FA93EA930E948163E9A150
:10BC3200E07459F0FE013696FA93EA93EBA10E9462
:10BC42001071FA93EA930E948163FE013696FA9389
:10BC5200EA930E949763E8A3E0910804EB8FE091D6
:10BC62000904EA8F0E94FA66D80111962D913C913F
:10BC7200D80113964D915C91D80115960E94497591
:10BC8200EEA3FFA3D8011796EC91F0E0ECA3FDA37D
:10BC9200D8011896EC91EC8FE0910904A0E10E9482
:10BCA2003273EAA3FBA30E94D3720E9441710E94E5
:10BCB2004171ECA1EA930E94B248D8011996EC9125
:10BCC200EC8FAC8DAF3011F4E8E0EC8F0E94D372B0
:10BCD2000E9436730E94DC710E943B730E943F7384
:10BCE2000E9446730E9449730E94D3723A932A9328
:10BCF200EAA5FBA5E40FF51F0E945273EEA1FFA176
:10BD0200E20FF31F0E94DC710E9436730E94497396
:10BD1200A8A5A130A1F43A932A93FA0131960E9480
:10BD22004673FA93EA93FA0131960E945273F9012B
:10BD320031960E94DC71F90131960E944973A8A5DF
:10BD4200A230D1F40E943F7331970E944673FA9356
:10BD5200EA93EAA5FBA5E40FF51F31970E945273FF
:10BD6200EEA1FFA1E20FF31F31970E94DC710E9446
:10BD7200367331970E944973E8A5E03011F40C94B0
:10BD8200DA5FD8011996EC91EC8FE0910804ACE0EF
:10BD92000E9455730E94D074ED8FA8A1EA1710F487
:10BDA2000C94185FE1E0E0930904E03021F0ECA18B
:10BDB200FDA1B5970CF402C00E945B73AAA1BBA1BE
:10BDC200ECA1FDA1EA1BFB0BDF010E941E6AEAA3A4
:10BDD200FBA3ABA1AA231AF4E0E0EAA3EBA3A8A178
:10BDE2000E941D73AEA1BFA1F0E00E946373EE8FAB
:10BDF200A8A5A13021F40E9467730E946C73A8A5C4
:10BE0200A23021F40E9467730E947673E0E0E9A3F6
:10BE12000E947E73AE0FBF1FEC91E03039F00E949A
:10BE22007E730E9410730E948373F2CFC2C0E1E05E
:10BE3200E0930904E03031F0ECA1FDA1E734A0E089
:10BE4200FA070CF402C00E945B73E8A1EF8FEAA12B
:10BE5200FBA1EE0FFF1FACA1BDA1AE1BBF0BE3E028
:10BE6200F0E00E94D074EAA3FBA3ABA1AA2322F4C0
:10BE7200E1E0F0E0EAA3FBA3EF8DE150EF8FEF8D5D
:10BE8200F0E0DE011696AE0FBF1FAC91A03219F0A2
:10BE9200AF8DA13008F404C0EF8DE150EF8FEFCFEA
:10BEA200AF8D0E941D73AE2FEEA1FFA1B0E0EA1785
:10BEB200FB0714F3EF8DE03011F4ED8DEF8FAF8DB2
:10BEC200ECE00E9455730E946373EE8FA8A5A13027
:10BED20021F40E9467730E946C73A8A5A23021F41A
:10BEE2000E9467730E947673E0E0E9A30E947E736A
:10BEF2000E940B7321F0EF8DA9A1AE1708F007C0C5
:10BF02000E947E730E9410730E948373EFCFAF8DE5
:10BF1200E8A1EA1BAE2FED8DEA1768F0AF8DE8A11C
:10BF2200EA1BACE0EA9FF001A09108040E9455735D
:10BF32000E94637301C0E0E0EE8FA8A5A13069F40E
:10BF42000E94677331960E94E872AFE00E943273DA
:10BF52000E948B7331960E94CF68A8A5A23059F433
:10BF62000E9467730E94E872AFE00E9432730E94DF
:10BF72008B730E94CF680E947E73AE0FBF1FAC917D
:10BF8200A03219F4E9A1EF5FE9A30E947E730E9437
:10BF92000B7339F0AF8DE9A1EA1BAE2FED8DEA17D5
:10BFA20008F407C00E947E730E9410730E9483737C
:10BFB200ECCFD8011C96EC91E03029F10E94FA6690
:10BFC2000E94D372A2DDF801A485A43698F4E0E0C1
:10BFD200E0930B04F801A485AA3028F0A485AA9363
:10BFE2000E94F14306C0D8011C96EC91E05DEA93F1
:10BFF20005DD09C0ECE0E0930B04E2E5EA93FEDC28
:10C00200EDE4EA93FBDCEB8DE0930804EA8DE09328
:10C0120009040E943277AA9608951A9310E0E894D0
:10C0220027F8143170F40E94F668E03011F00E9493
:10C0320003691F5FA895E12FE37011F40E94671551
:10C04200F0CFE0E0E0930B040E9467150AC11A9357
:10C0520010E01431D0F40E94F668E03081F00E94C2
:10C062002D73DF01EB81FC81EA17FB0744F40E9488
:10C072002D73DF01E981FA81AE17BF070CF002C010
:10C082000E9403691F5FA895E4CFE0E0E0930B04F0
:10C0920018810C946D631A9310E0143190F40E948D
:10C0A200F668E03029F00E94FD68E081E17009F451
:10C0B20006C01A93E0910504E170EA9397DD1F5FD1
:10C0C200ECCFCFC02C970E942B77AD89BE890E94FE
:10C0D2001E6AED8BFE8BAB89BC890E941E6AEB8BBC
:10C0E200FC8BED89FE89A98DBA8DEA0FFB1FE98FC2
:10C0F200FA8FEB89FC89AF89B88DEA0FFB1FEF8BB2
:10C10200F88FED89FE89AD89BE890E949273EE8710
:10C11200FF87688B798BEB89FC89AB89BC890E948C
:10C1220092730E9499730E94D876EA87FB876C8784
:10C132007D8700E010E0EB89FC89E017F10714F439
:10C142000C94E460F8010E9467740E9402760E94D7
:10C152009E73AE81BF81888599850E948A76AA8561
:10C16200BB858C859D850E948A760E9499730E9468
:10C17200A3730E94CB75AF015A934A930E94EA655A
:10C182002E2F33270E94A873E98DFA8DE01BF10B45
:10C192000E94AF73ED8DFE8DE01BF10B0E94B9730F
:10C1A2000E94A873F801A98DBA8DEA0FFB1F0E94A5
:10C1B200AF73F801AD8DBE8DEA0FFB1F0E94B973FC
:10C1C2000F5F1F4FB8CF0E9432776B960895E091B0
:10C1D200180BE0937100E0E0E0937400E2B3E360D7
:10C1E200E2BBE1B3E360E1BB8BE18A95F1F7E1B336
:10C1F200EC7FE1BBE4E4E093740085E88A95F1F713
:10C202000895E2E001C0E0E0E093180BE0DF08955A
:10C212001A931FEFF6DF16D0E03089F4E9810E940D
:10C22200BF7341F4EDB7FEB7FA93EA931F930E94EE
:10C23200C4731F9118D088EC90E00197F1F7E3DF07
:10C24200E12F70C01A9314EAE4EA0E94C87341F421
:10C252000E94CD73183011F0103111F4E0E001C0EA
:10C26200E2E019910895E4E9E0937400E0E00895B2
:10C272001A93E981E1600E94D27331F40E94CD7376
:10C28200103411F4E0E04EC04CC01A93E9810E94D0
:10C29200D27331F40E94CD73183111F4E0E042C040
:10C2A20040C01A93E9810E94D27331F40E94CD7387
:10C2B200183211F4E0E036C034C01A93E981E0305C
:10C2C20011F0E4EC01C0E4E80E94C87379F40E9422
:10C2D200CD73E0917300AA81BB81EC93103511F00C
:10C2E200183521F4E0E018810C945566E1E01881DC
:10C2F2000C9455661A93E981E093740010E0E09182
:10C302007400E07811F4163908F005C08DE08A95C2
:10C31200F1F71F5FF4CFE0917400E07811F0E0E0F4
:10C3220001C0E1E01881229608950E942D773D8197
:10C332000C8120E087DFE03011F5EE810E94C96DAB
:10C34200F1F43A93AEDFE030D1F40E94D673B9F43F
:10C3520079DFE030A1F4EE810E94BF7381F4EDB782
:10C36200FEB7FA93EA931F930E94C4731F91E030C1
:10C3720031F479DFE12F0E9434770C94FF6327DFD9
:10C38200D9CF0E942D7730E00E811D815BDFE03036
:10C3920099F4EF810E94C96D79F40E94D67361F419
:10C3A2001A937FDFE03041F4EC81EA937ADFE030E8
:10C3B20019F459DFE0E002C00ADFE8CF0E943477C7
:10C3C2002896089522970E942B7750E02B853A8574
:10C3D200A89538DFE03011F00C944562EE850E949A
:10C3E200C96D11F00C9445622A935BDFE03011F0C5
:10C3F2000C9445623A9355DFE03011F00C9445629B
:10C4020021DFE03011F00C944562EE850E94BF738B
:10C41200D9F5E0E0EE83EF83EC85FD8531970E944C
:10C422005E7149F4EDB7FEB7FA93EA931F930E9447
:10C43200C4731F9109C0EDB7FEB7FA93EA931F9335
:10C44200E1E0EA933ADF1F910E2FEE81FF81A8858A
:10C45200B985EA0FFB1F1083EE81FF813196EE83CF
:10C46200FF83003039F4EC85FD85AE81BF81AE17C4
:10C47200BF0708F001C0D0CFEC85FD850E945E7138
:10C4820019F4F1DEE0E002C0A2DEA3CF0E9432770F
:10C492002F96089568970E942B7720E0E0E0EC8FBA
:10C4A200ED8F31E0A895E9A1FAA1662777270E94CE
:10C4B2000276EA87FB876C877D87EE8D0E94DB73AD
:10C4C2000E949E73AA85BB858C859D850E94D87625
:10C4D200EA8BFB8B6C8B7D8B0E945C75FE017296E6
:10C4E200FA93EA930E945766EE8BFF8B688F798FDF
:10C4F2000E94E1730E94C975AF010E94E173AE8D83
:10C50200BB27882799270E9463750E94A373DE01C7
:10C512005A960E94C975ED93FC930AA119A192DE65
:10C52200E030D1F5EDA10E94C96DB1F50E94D6733C
:10C5320099F51A93B6DEE03079F5303051F14F5F5C
:10C542005F4FEC8DFD8D3196EC8FFD8FAC8DBD8DE7
:10C552001197EBA1FCA1EA17FB0711F430E018C018
:10C56200EC8DFD8D3197AF8DB8A10E94107399DECD
:10C57200EE8DDA01F0E0EA17FB0751F474DEEA8D82
:10C58200FB8DA9A1BAA1EA0FFB1FE9A3FAA38BCFE6
:10C59200D4CF69DEE0E002C01ADEC1CF0E9432775A
:10C5A200A6960895A881A03310F0AA3308F004C01B
:10C5B200E881E0530C94D863A881A13410F0A73429
:10C5C20008F004C0E881E7530C94D863EFEF0C94B1
:10C5D200D863A881AA3020F4E881E05D0C94D86386
:10C5E200A881AA3020F0E881E95C0C94D863E8E5E0
:10C5F2000C94D8631A930A93F8940091190B109132
:10C602001A0B7894F8010991199108951A930A93D3
:10C61200F1DF8F01EA81FB810E94F56EE01BF10BD5
:10C62200DF010E9421772CF4E0E0198108810C944B
:10C632008366E1E0198108810C9483660E948A6610
:10C642000E9498660E946D5D0E949868E6EBFBE18D
:10C652000E9494660E94FA660895EAE6F6E1FA9369
:10C66200EA93EAE6F0E0FA93EA930E94B268E4E021
:10C67200EA93E6E2EA93EEE0EA930E941C4AE2E0E1
:10C68200F7E10E94EC66E3E5F0E0FA93EA93E8E072
:10C69200EA93E2E3EA93E1E0EA930E941C4A0895F6
:10C6A20099818881009641F0BD81AC81FB81EA814C
:10C6B20005900D920197E1F7FD81EC810C94836660
:10C6C200B981A881109631F0FC81EB816A81619376
:10C6D2001197E9F7EB81FC8125960895E991F9918B
:10C6E200A991B9911D900590011421F40020D1F770
:10C6F200EE2708951018E1F3E1E008F4E2500895FE
:10C70200E991F991A991B991CD0161916D93662356
:10C71200E1F7FC010895E991F991A991B991CD014F
:10C7220005900D920020E1F7FC010895A991B991BD
:10C73200EE27FF276D91662311F03196FBCF089506
:10C74200AA27BB27E991F9910590002011F01196D3
:10C75200FBCFFD0108957991E991F991A991B991E0
:10C76200CD01772351F07A9561916D936623C9F7D4
:10C77200772319F07A956D93FBCFFC0108956991A7
:10C78200E991F991A991B991CD01662351F06A9588
:10C7920005900D920020C9F7662319F06A950D9253
:10C7A200FBCFFC0108955D9BFECFE881ECB9219699
:10C7B20008951A930A93AC81BD810E9449753097FE
:10C7C200C1F0AA81BB810E9449758F01309749F05F
:10C7D2000230E0E01E0760F0F80131978F01ED931F
:10C7E200FC93AC81BD810E94EB683197AE81A0833E
:10C7F20003C0EE81EA93D7DF198108812796089555
:10C802002C970E942B7710E0E88DF98D3196E88FF6
:10C81200F98F3197E4912E2FE03011F40C94BD651D
:10C82200E12FE03039F4253211F411E002C00E9408
:10C83200ED73A1C1E130C1F4253219F40E94ED7308
:10C8420099C112E0E0E0E98B00E02D3211F401E041
:10C8520092C12B3219F4EBE2E98B8DC1203219F42B
:10C86200E0E2E98B88C102C0E23039F450E013E023
:10C87200203311F400687FC102C0E330A1F42033F9
:10C8820010F02A3308F009C0A52FEAE0EA9FF00170
:10C892005E2FE22FE0535E0F6EC140E02E3211F4A4
:10C8A20014E069C110C0E430A1F4203310F02A333F
:10C8B20008F009C0A42FEAE0EA9FF0014E2FE22F10
:10C8C200E0534E0F58C12C3619F4026015E053C1E3
:10C8D20004C0E53011F00C94BC65E22FE33649F454
:10C8E2000E94F873EE89FF89A481AA930E94FE73C5
:10C8F20041C1E33741F40E94F8730E9408740E9418
:10C9020097631E2F0AC0E037A1F40E94F8730E94B9
:10C9120008740E94A1631E2F08600F77403011F047
:10C92200411708F001C0142F40E0E0E0E88B30E04E
:10C9320078C0E43611F0E93611F4046002C0E5373C
:10C94200A1F4EAE0E88B01FF08C0E0E0FAEC6AE952
:10C952007BE30E9466681AE023C0E0E1F7E260E050
:10C9620070E00E94666815E01BC0E83511F40860AB
:10C9720004C0E83711F00C94BB65E0E1E88B01FFDD
:10C9820008C0E0E0F0E060E070E10E94666818E054
:10C9920007C0E0E0F0E160E070E00E94666814E049
:10C9A200403011F00F7701C041E001FF08C00E9442
:10C9B200F873AE89BF8914960E944D7515C002FFA7
:10C9C2000AC00E94F873AE89BF8914960E94497505
:10C9D2000E94677409C00E94F873AE89BF891496D9
:10C9E2000E94497566277727EC87FD876E877F87C8
:10C9F20002FF16C0AF85AA2362F4EC85FD856E8521
:10CA02007F850E944374EC87FD876E877F87EDE206
:10CA1200E98BE989E03019F01F5F4F5F01C00B7F9E
:10CA2200342F00FD14C0151710F4351708F00FC08D
:10CA320007FF08C002FF04C00B7F2989115001C003
:10CA420020E301C020E20E94ED735150ECCF141795
:10CA5200B0F4006102FF0AC00B7FE989EA930E94E9
:10CA6200FE73503009F0515011504150E0E3EA9307
:10CA72000E94FE73503009F051504150E8CF312FDF
:10CA8200E889E030D1F43030B9F003FF08C0EE811C
:10CA9200FF813196EE83FF833197E49105C0AE8129
:10CAA200BF81ED91AE83BF83EA930E94FE73503043
:10CAB20009F051503150E7CF53C00E9410740E94C8
:10CAC200D5742E2F2A3030F003FF02C0295C01C03A
:10CAD200295A01C0205D04FD23C0213350F40E9475
:10CAE2006B68A130E0E0BE07E0E08E07E0E09E0761
:10CAF20009F40BC0431740F4531710F000FF01C0B4
:10CB020014C020E207FF0CC020E3006102FF08C04E
:10CB12000B7FE989EA930E94FE73503009F051506D
:10CB22000E94ED73503009F0515031500E94107440
:10CB32000E941075EC87FD876E877F87E8890E94C7
:10CB42006B68FF27662777270E94D5740E94666864
:10CB5200E885F9856A857B850E941D7709F0ADCF4E
:10CB620000FF08C0503031F05150E0E2EA930E94D9
:10CB7200FE73F8CF10E048CE0E9432776A9608958D
:10CB8200FF92F82E22971A930A93DE010E943674BE
:10CB92008D01DE0116960E9436740E944975EA8361
:10CBA200FB83DE0114960E9436740E944975FA9343
:10CBB200EA931A930A93FE0136960E94F36620DEE8
:10CBC200AA81BB81E0E0EC93198108812496FF9051
:10CBD2000895A991B991EE27002460E8E894162EF1
:10CBE200169407941E2A1EF0A015B10518F0A0197C
:10CBF200B109E62BB7FBAA0FBB1F669580F7089514
:10CC02007B816A81F981E88177FB770F67FD71602B
:10CC1200972F9E5781F078F0983190F4AA27BB277E
:10CC2200882708948795B795A7959A95D1F7EA230F
:10CC3200FB23682305C0E8947727EE27FF276627A2
:10CC42006F77769508F4606877F9A991B99189911F
:10CC52009991EA17FB076807790797FB08950E94E5
:10CC6200CC720E94197419F40E9420741DC0E6F758
:10CC7200A881B9818A819B81E0E0F0E060E87FE3EE
:10CC82000E94A37311C00E94CC720E94197419F4FD
:10CC92000E94207409C0E6F30E942074A0E0B0E074
:10CCA20080E89FE30E943C76249608950E942574B2
:10CCB2000E941D7739F4A881B9810E94EF6C0E940D
:10CCC200537520C0AA81BB818C819D810E942577EA
:10CCD20034F40E9425740E945C75C1DF05C00E9475
:10CCE20025740E945C75CFDFA881B9810E945375BB
:10CCF200A881B9810E944D75AA81BB818C819D81D9
:10CD02000E94A37326960895E4E6F0E0FA93EA936C
:10CD12000895E1E0F0E0FA93EA930895E4E0F0E0A8
:10CD2200FA93EA930895FA93EA930C94165DE0E07D
:10CD3200F0E0FA93EA930895EFE9F0E0FA93EA93C8
:10CD42000895E0E2F0E0FA93EA930895EFE0EA93BF
:10CD52000C94B248E0E0E0930A04E0930B040895D7
:10CD6200A8E0B0E00E947775E0300895EBE9F0E0CA
:10CD7200FA93EA930895E4E1F0E0FA93EA93EEE19C
:10CD8200F0E0FA93EA9308950E944746EFCFEDE26E
:10CD9200EA93CDCFE0E4F0E0FA93EA93ECCFEBE252
:10CDA200EA93C5CFE1EFFFEFFA93EA9308950E9469
:10CDB2004746F8CFE0E6F0E0FA93EA93DCCFEDE401
:10CDC200EA93B5CFA5E01A9FF001E45CFD4F089508
:10CDD200A12FB0E00895FA93EA93EAE5F0E0FA931E
:10CDE200EA930895FA93EA93A2CF0E94620E0C94FA
:10CDF2000E60E1E0E0930804E09309040895E093F3
:10CE02000A04E0E0E0930B040895FA93EA93EEE15A
:10CE1200F0E0FA93EA930895E32FF0E00895A091E9
:10CE2200F10BB091F20BBD01A3E0B0E00E947D7462
:10CE3200E60FF71FE491E0300895A091BB05E3E00F
:10CE4200EA9FF001EF5F0E2F0895E02FF0E00895C2
:10CE5200E6E9F0E0FA93EA930895FA93EA93F5CFBC
:10CE6200A091F10BB091F20BBD01A3E0B0E00E94E2
:10CE72007D74E60FF71F0895ABE03A9FF001E45B83
:10CE8200FD4F0895FA93EA930C944746E091780B8C
:10CE9200A0EA0E94AF742E2FE091790BA0E80E94C5
:10CEA200AF745E2F08953A930E945830A091410BBF
:10CEB200AD320895E0914F0BE295EF70E0930A04D2
:10CEC200E0914F0BEF70E0930B040895A02FBB2766
:10CED200E22FF0E00E94A5743396FA93EA93089544
:10CEE200ED5FF0E0FA93EA930895E22FE450F0E068
:10CEF200FA93EA93E52FE450F0E0FA93EA93E32FF2
:10CF0200E058EA9314CFE0E0EC93AE81BF8108953C
:10CF1200E1E0E0930804E2E0E09309040895E52FDC
:10CF2200F0E00895EA1BA9E0B7E0F0E00E94577430
:10CF32000895A0E021FCA1E0A1300895E1E6F0E02F
:10CF4200FA93EA93EAE4F0E0FA93EA93ECE1F0E090
:10CF5200FA93EA930895E981F0E00895EE0FFF1F36
:10CF6200EA5CFD4F0E9458750895A4E3B2E0F0E038
:10CF7200EE0FFF1FEA0FFB1F0E9458750895DB0199
:10CF8200AE1BBF0BE2E0F0E00E946C75EA1B089555
:10CF9200FA93EA93E4E1F0E0FA93EA930895E12F39
:10CFA200F0E00895E3E0F0E0FA93EA9308950E9436
:10CFB2005875FA93EA930895EA81F0E00895EC81B6
:10CFC200F0E00895ABE0EA9FF001E752FA4F0895CE
:10CFD200FA93EA93E4CFE150ADE0EA9FF0010895BD
:10CFE200ED5FFC4FDF010E9449750895FA93EA93C1
:10CFF2000E946D5D0C944A5DEA930E945830E1E410
:10D00200FBE0FA93EA93EAE0EA930E942D5D8FCE69
:10D01200E12FEF5FF0E00895E6E0F0E0FA93EA93A3
:10D02200F7CFFA93EA930C946D5DEE0FFF1FAE0FEC
:10D03200BF1F0E9449750895FA93EA930C94D34353
:10D042000E9467740E945C750895E4E1F0E0FA932F
:10D05200EA930895FA93EA9379CEF0E0EDCFE2E015
:10D06200F0E0DFCFE0916805F09169050895E09165
:10D072006405F09165050895AE0FBF1FE3E0F0E08F
:10D082000E94D0740895FA93EA931A930A930C9427
:10D092008012FA93EA933A932A930C948012A09105
:10D0A2006C05B0916D050895A0916E05B0916F0564
:10D0B2000895A0E0B0E00E94737508950E946C7517
:10D0C200EA1BFB0B0E9467740895E887F9876A8759
:10D0D2007B870895A885B9858A859B850895A2E0F6
:10D0E200B0E00E94737508950E9467740E94FA74FA
:10D0F2000895A4E0B0E00E9473750895EC83FD8367
:10D102006E837F83AC81BD818E819F810895A6E06D
:10D11200B0E00E9473750895E0E9F1E0FA93EA93B2
:10D122000C942A74E6E3F0E0FA93EA930895E2E0BD
:10D13200E0930804E09309040895EA930E94FF5CD7
:10D1420058CEEAE0EA930E945843E0916C05F091D0
:10D152006D050895E8E1F0E0FA93EA93E8E2F0E081
:10D1620079CFE6E4F0E0FA93EA930895E8E8F0E094
:10D17200FA93EA93D7CFEAE0EA930E945843E09108
:10D182006E05F0916F050895E8E2F0E0FA93EA93F4
:10D192000895E2E3F0E0FA93EA930895FA93EA93AA
:10D1A2000C94865DFA93EA93AFCDE8ECF0E0FA9343
:10D1B200EA930C942A740A921A92FA926A937A93D4
:10D1C2008A939A93AA93BA93EA93FA93EFB7EA935C
:10D1D2001A930895ED91FD913196FE93EE93089581
:10D1E200E4EFF1E0FA93EA930895ADE01A9FF001BB
:10D1F200E050FD4FE0810895ADE01A9FF001E65F37
:10D20200FC4F08951A93E1E0EA930C94F75DE2E093
:10D21200EA930C94F75DE091DF07F091E0076091EB
:10D22200E1077091E2070E945C750895E091D707CB
:10D23200E150AAE5B6E0F0E00E945774AE0FBF1FBE
:10D242000E944D750895EAE6FBE0FA93EA93089589
:10D25200EAE0EA930C942D5DE091D807EA93E0911D
:10D26200D507EA930E949632A091D50BB091D60BC6
:10D2720010970895A091D70BB091D80B8091D90B3C
:10D282009091DA0B0E9425770895E091D50BF091E9
:10D29200D60B0895E0E2EA930C94FF5CE091D70B81
:10D2A200F091D80B6091D90B7091DA0B0E945C75EA
:10D2B2000895E091D507EF5FE093D5070895EF5FFA
:10D2C2000E948B75E150EAE0F0E0FA93EA930C9445
:10D2D2002A74E091C907ABE0EA9FF0010895A083A8
:10D2E200E9ECF7E0FA93EA930C940E2CE5E0F0E017
:10D2F20098CEE1E0EA930E94500E4BCF0E942A742E
:10D30200E0E0EA930C94500EFA93EA930C942A7498
:10D31200A9E0B0E00E9477750895E091040CEF5FF8
:10D32200E093040C0895E1E0EA930E94500E90CD40
:10D33200AEE0B0E00E94777508951A930A93A09127
:10D34200D0070895E0E0E0930B0CE0930A0C0895F7
:10D35200E0E0F0E0ED93FC930895EA81D801EC93CC
:10D36200E9ECF7E0FA93EA930E940E2C1981088106
:10D372000895E12FACE8B0E0F0E0EE0FFF1FEA0FF6
:10D38200FB1F0E9458750895A3E21A9FF001E65A06
:10D39200F94F0895A3E21A9FF001E45AF94FE08190
:10D3A2000895E981ADE0EA9FF0010895E65FFC4F40
:10D3B200A1E0A0830895ACE8B0E0F0E0EE0FFF1F1B
:10D3C200EA0FFB1F0E9458750895A091CD07B091F6
:10D3D200CE07EA2BFB2BE093CD07F093CE070895FF
:10D3E200E150A7E1EA9FF0010895A7E10A9FF00149
:10D3F200EC5EF94FAF010895FA93EA93E0E0EA9305
:10D402000895F0E0A4E6B0E00E94A5740895E091CA
:10D41200630BF091640B0895EAE5F6E0EDCFFA9321
:10D42200EA930C946163E881F0E0E65AF94F0895BB
:10D43200E981FA81FA93EA930895E2E0F0E00E942A
:10D44200D0740895A1E5BBE0E091D107F0E0089522
:10D45200A4E5BBE0E091D107F0E0AE0FBF1F089555
:10D46200A7E5BBE0E091D107F0E0AE0FBF1F089542
:10D47200EE0FFF1FAE0FBF1F0895AAEDB6E04FCD0E
:10D48200EE0FFF1FEA0FFB1F0895A7E11A9FF0019D
:10D49200EC5EF94FEE83FF83AE81BF810895EE818A
:10D4A200FF81A481AA930C94A9190D901C90AE81BE
:10D4B200BF811296EC91F0E0E00DF11DDB01ED93DE
:10D4C200FC930895ED91FD913197FE93EE930895AB
:10D4D2000E94481BEF770E2EAA85BB851296EC910F
:10D4E200E0150895A3E20A9FF001E15AF94F089569
:10D4F200BD01AAE0B0E00E947D74E60FF71FE88745
:10D50200F987A1810895E057F84FEC87FD87AC8534
:10D51200BD85119608951296EC91AC85BD8516963F
:10D52200EC930895D001F0E00895A885B985189686
:10D532000E9449750895AC85BD85EC93E9ECF7E04E
:10D54200FA93EA930C940E2CE885F985A281AA93AA
:10D552000895EA85FB85FA93EA930E948A19E030DE
:10D562000895AA85BB85EC91EA93E3E0EA930C94D3
:10D572008B45AA85BB85E0E0EC93E2E0E0930906E7
:10D582000895BF0100801180AE81BF811296EC9197
:10D5920008950E946C75EA1BFB0B0895DB01ED9365
:10D5A200FC93AE81BF811296AECCE45FFC4FE0816A
:10D5B200E058DB01EC930895E4E6F0E00E94A574E4
:10D5C2000895F0E0ED93FC930895E9ECF7E0FA9307
:10D5D200EA930C940E2CE091D007A091CF07EA17A2
:10D5E2000895F0E0E00DF11D0895A091780BE0910F
:10D5F200790BEA9FF0010895AAE5BBE0D0CCA4E53F
:10D60200BBE0EE27A10FBE1FEC910895A7E5BBE09A
:10D61200EE27A10FBE1FEC910895BD01AAE0B0E074
:10D622000E947D74DB010895E081EA930C940E560A
:10D63200E6EFF9E0E093140BF093150B0895EA93EB
:10D642000E9458300C945319BD01AAE0B0E00E9428
:10D652007D74E60FF71F0895A4E5BBE0EE27A00F47
:10D66200BE1FEC910895A7E5BBE0EE27A00FBE1FF9
:10D67200EC910895A1E5BBE0EE27A00FBE1FEC914F
:10D68200E1700895AAE5BBE0E0CBE150F0E0089537
:10D69200A7E6BBE0EE27A00FBE1FEC910895A0E61F
:10D6A200BBE0EE27A00FBE1FEC910895EA81ADE02A
:10D6B200EA9FF001E65FFC4FA0E0A083EA81EA93D3
:10D6C2000895ABE00A9FF001E952FA4F08951A93C8
:10D6D2000E945D36A091E30BB091E40B0E9421778A
:10D6E2000895ABE00A9FF001E352FA4F0895A0912A
:10D6F200E30BB091E40B0895FA93EA930C94852D11
:10D70200FA93EA930E9407463A9381CDE091E30BA4
:10D71200F091E40B30970895AFEFBFEFA083B18390
:10D722000895E0E0F0E0E093E30BF093E40BE09384
:10D73200E00B08950E94FB62E093100CF093110C31
:10D742000895F0E06ECCFA93EA9382CDFA93EA93CD
:10D75200E0E0F0E80895E091E10BF091E20B08952A
:10D76200E0914C0BF0914D0B0895E093E10BF09397
:10D77200E20B0895FA93EA930C94FB2FE057F84FCB
:10D78200FA93EA930E94A32220CFE091C707ABE06D
:10D79200EA9FF0010895E7ECF7E0FA93EA930C941C
:10D7A2000E2CE093E30BF093E40B0895E88DABE0CD
:10D7B200EA9FF00108950E94925DE0E0EA930C94E2
:10D7C200620FE0E0F0E0E093DB07F093DC07E1E0DA
:10D7D200E09309040895E0910E04E550F0E002CBD5
:10D7E200E091DB07F091DC0727CCE0915805F0913E
:10D7F200590531970895FA93EA930C945B5CA0E083
:10D8020024FCA1E0A0300895E7E0EA93E0E0EA9387
:10D812008ECA0E94FB62E093E907F093EA0708953B
:10D82200E091DD07F091DE07FA93EA930C94F81A7F
:10D83200FA93EA930C940763E0E0E0930A0C0895EC
:10D842000E946D5D0C944A5DEF5CEA930C94FF5C60
:10D85200AAE9B6E0E1CAAAE5BBE0E091D107F0E0AF
:10D862000FCEAAEDB6E0D8CAAE0FBF1FEC91E160B1
:10D87200D001EC930895E091D007EA93E0E0EA93B7
:10D882000C944924EA930E9458430E94A1451E2FFA
:10D892000895EAE2EA93E5ECF9E1AECD0E94D924DB
:10D8A200E1E0EA930C94C1241F771A930C94583048
:10D8B200A091DB07B091DC070895E053F0E00895F2
:10D8C200F7DFEA17FB070895FA93EA930E94211BF8
:10D8D200E0300895E093DD07F093DE070895E093CA
:10D8E200CF07E0E0E093E60708950E94875A0E947E
:10D8F200FA25E093DA0708950E9458300C94925D5D
:10D90200E1E4FBE020CF0E9455220E9416190E94FA
:10D912009E45E03008950E94A1451E2F1A930E9451
:10D922002D26103808951A93E091C105EA930895BF
:10D93200E091DD07F091DE07C7CFE091400BEA935B
:10D942000E94632FE03008950E94FB62E093120C64
:10D95200F093130C0895D90118960E944975089501
:10D96200E4E6F0E060E070E00E94FA7408950E943C
:10D972005830F6CE0A93E091C105EA930895E091FA
:10D98200E507EA930A930C94A731ABE03A9FF001C2
:10D99200EF51FA4FE0810895ABE03A9FF001E15276
:10D9A200FA4FDF010E9449750895FA93EA93E8EE6F
:10D9B200F3E03ECFE093160BF093170B0895A0917E
:10D9C200160BB091170BAC910895A6E1BBE002CC07
:10D9D200E091F207E053E093D8070895E0E0F0E029
:10D9E20060E070E00895FA93EA93E0E3EA930C941E
:10D9F200875AE12FAAE5B6E0F0E00E945774089535
:10DA0200AE0FBF1F0E944D750895E091EF07EA9394
:10DA12000C942A5AFA93EA930C946A590E94E35995
:10DA2200EBE3EA930C945A59E1E4FBE0FA93EA93AC
:10DA32000895E89423F8E0E0F0E04CDFE0E0E093C2
:10DA4200D5070A93E1E0EA930C944924E89423F879
:10DA5200E0E0F0E03FDFE0E0E093D507EA930C94EA
:10DA6200C124A881B981EC91EF5FEC930895ABE0FA
:10DA72001A9FF001EF56F84FE0810895ABE01A9F2C
:10DA8200F001E952FA4F0895ABE00A9FF001E85223
:10DA9200FA4F0895A083ABE00A9FF0010895EA933C
:10DAA2000E945D360E94FD35E0300895ABE00A9F8A
:10DAB200F001E652FA4F0895FA93EA93ECEEF9E197
:10DAC200FA93EA93EA85ABE0EA9FF0010895FF2713
:10DAD200662777270E945C7584E00E94C1652896BC
:10DAE2000895AC81BD81EE27A00FBE1F0895E02FDF
:10DAF200AC81BD81F0E0EA0FFB1F089584E00E9433
:10DB0200C16528960895EE27A30FBE1FEC91D001A0
:10DB1200EC930895ABE01A9FF001E852FA4FE081CE
:10DB2200E0300895A9E0B7E077C90E945774EA0F80
:10DB3200FB1FAF010895E091E30BF091E40B089510
:10DB4200E32FA091D507EA0F0895ADE02A9FF001D7
:10DB5200E85FFC4F0895E0914F0BE295EF70089556
:10DB6200A8E0B0E00E94777508951A93E0EAEA937C
:10DB720023CAE054F14FFA93EA930E9496611E2F52
:10DB82000895E054F14FFA93EA931A930C94C26108
:10DB9200EA930E944661E0300895E0EAEA93EEE5F6
:10DBA200F0E0FA93EA93E0E0FFE0FA93EA93E5E724
:10DBB200FBE00895FA93EA93E0E2EA930C944B6255
:10DBC200E0EAEA93E981FA81E050FE4EFA93EA93A1
:10DBD2000895A8E2B0E00E94A5740895E0EAEA93ED
:10DBE200E2E0F0E0FA93EA931A930A930895FA9323
:10DBF200EA930C94E361FA93EA930C949661EDE252
:10DC0200EA93EAE0F0E00BCC1A930A93D5C9ABE0B1
:10DC1200B0E00E94A574E050F24F8F01AA81AA30B1
:10DC22000895E0EAEA93EBE0F0E0FA93EA931A93BC
:10DC32000A93E9E6FBE00895EE0FFF1FE050F04F74
:10DC42008F01AA81A03808950E945774E058F14FBD
:10DC52008F01AA81A33008950E9457740E945374C1
:10DC6200DF01EA85F0E0AE0FBF1FE8E0F0E00E94BE
:10DC7200A574E050FA4E8F01E0EAEA93E8E0F0E0A2
:10DC8200FA93EA931A930A93E3EDFBE0B0CF4E0FB7
:10DC92005F1FE091D70BF091D80B6091D90B709177
:10DCA200DA0BAE81BF81888599850E943A74EE8332
:10DCB200FF836887798708954093D50B5093D60BDD
:10DCC200EE81FF8168857985E093D70BF093D80BBD
:10DCD2006093D90B7093DA0B0895E8E0F0E0FA93C1
:10DCE200EA930895ED81EA93ED81EA930895E09332
:10DCF200DE0BF093DF0B0C94F733E093DF07F09326
:10DD0200E0076093E1077093E2070895E0914E0BFC
:10DD1200AAE5B6E0F0E00E9457740895E850FA4F81
:10DD2200E081E1300895FA93EA93E091D807E05D4B
:10DD3200EA930895EA930E94A85AE1300895E2EF27
:10DD4200F7E038CE0E945163A881AF5FEAE00E94FB
:10DD5200AF74E05D0895A881AF5FEAE00E94FF74AE
:10DD6200E05D08950E945574E854FF4F32960E9478
:10DD7200587508950E945574E854FF4F08953696D9
:10DD8200E491D901EC930895E881F0E0A5E0B0E0D8
:10DD92000E94A5740895E0EAEA93E5E0F0E0FA93C0
:10DDA200EA930895EA930E94ED33FA93EA93EBED36
:10DDB200FBE00895FA93EA93EFEFEA93E5E0F0E0EF
:10DDC2002ECBE093DC0BF093DD0B0895E0EEFBE04D
:10DDD200F1CFA091E10BB091E20B0895E0E0E09366
:10DDE200EF0BE093F00B0895AC81BD81EA0FFB1FAE
:10DDF20008951A930E9482341E2F0895E981FA81B0
:10DE0200EA17FB070895EB81EA930E94A734FA937D
:10DE1200EA93E0EEFBE00895F0E0FA93EA930895C6
:10DE22000E940D450C94DA44F0E00E945774089564
:10DE32000E945C750E94F7440C94DA440E940D45DE
:10DE4200E5E1FAE1D9CA0E94DA440C94DA4420E00E
:10DE520030E0E12FE05DEA93E8E1FAE164CFEAE045
:10DE6200EA930C943259EAEFFAE0FA93EA930895AE
:10DE72001091580500915A0508950E94A1453E2F20
:10DE82000C94AA5CEAE0F0E00E94A5740895DF0118
:10DE9200EE27A30FBE1F0895F0E0EA0FFB1F0895BF
:10DEA200E02FA0E0B2E0C0CFEA0FFB1F3296E49170
:10DEB2000895F0E0AE0FBF1FEC91E1700895A1E567
:10DEC200BBE07DC80E94925DE1E0EA930C94620F90
:10DED2000E94620E0C949866FA93EA93E091D20B38
:10DEE200EA930E942638E1320895FA93EA93E3E630
:10DEF200EA930E94CC37E1320895E6E0F0E00C9418
:10DF0200F366EA0FFB1FFA93EA93E0E1EA930E94B9
:10DF1200CC37E13208950E946D5DA1E5BBE0EE27AA
:10DF2200A10FBE1FEC91E1700895FA93EA93E2E02B
:10DF3200EA930E942638E13208950E946D5DE12F36
:10DF4200EF5FEA930E94F143EAE3EA930E94FF5CE7
:10DF5200D7CCE7E0F0E0FA93EA930895EF5FEA9313
:10DF62000C94F143E3E7EA930C94FF5CEA23EA930F
:10DF72000E94F7438FC9EAE3EA930C94FF5CE8E05E
:10DF8200F0E00C94F366EA930E94CC37E1320895F4
:10DF9200EA930E94F7437EC90E945574E853FA4FF0
:10DFA20008950E946D5D0C942667EEE6F5E0E0931D
:10DFB200F10BF093F20B08950E941332E0E0E0932C
:10DFC200D7070E94EC150E94620EE1E0E093D207AF
:10DFD20008950E94925D0E94BB100E94A1450E2FDF
:10DFE2000D330895EE81FF81FA93EA930895EAE2F0
:10DFF200EA93E0ECFAE10895EA930E943C160C944D
:10E00200620E1A93E091EF07E0531E2FE3EFF7E061
:10E01200D1CCE091C907A091CA07EA170895EAECAA
:10E02200F7E0FA93EA930C940E2CE091CA07ABE066
:10E03200EA9FF0010895A0912B0BAF5FEAE00E94E6
:10E04200FF74E0932B0BEAE2EA930E942A5AE2E57C
:10E05200EA930E945A59E0912B0BE05AEA930E94EC
:10E062005A59EEE0EA930C945A59EBE3EA930C9472
:10E072005A59EEECFAE1CECCD9011696EC91CCCEFF
:10E082000E948B59F2CFF901A281B381BA93AA936C
:10E0920008950E948B59EAE3EA930C945A59119617
:10E0A200E0E0EC930E94455ABACFD901EC91B4CE8C
:10E0B200E05DEA930C945A590E948B590C94455A8C
:10E0C200EEE0EA930E945A59D4CFE05DEA930E94AF
:10E0D2002A5AE2E5EA930C945A59E45DF44FE0813E
:10E0E200E7CFEAE3EA930E945A59F90108950E94A0
:10E0F200455A0E94FB62E093210CF093220CE2E06D
:10E10200E093EC07D9011196EC930E9432770895BF
:10E11200EA930E942A5AE2E5EA930C945A59EEE0F5
:10E12200EA930C945A590E94FB62E093210CF093FB
:10E13200220CE2E0E093EC07D9011196EC930E94E5
:10E1420032770895E091D00BC0CFE091D00BF0E090
:10E15200C4CFE091EE0BA091ED0BEA170895FA936C
:10E16200EA938ECFE6E1F6E0E093BC05F093BD05BD
:10E172000895E093BC05F093BD050895FE01FA935E
:10E18200EA930895E6E0FBE1FA93EA93EE85FF85D0
:10E19200688979890E945C75B1CCEAE0FBE1FA9367
:10E1A200EA93AE85BF8588899989DACB0E945C752E
:10E1B200AA89BB898C899D89E4E6F0E060E070E081
:10E1C2000E9414750E945C7588E00E94C1652C96BD
:10E1D2000895E3E1FBE1FA93EA93EE85FF850C945F
:10E1E2002168EE27A10FBE1FEC91EA930895EA93EE
:10E1F2000E9462441F5F0895E091BF05A2ECB5E062
:10E20200F0E00895E091BE05A2ECB5E0F0E038C977
:10E21200EF73A5E1EA9FF001E551FB4F0895EF731B
:10E22200ABE0EA9FF001E15FFB4F0895AC81BD8155
:10E23200EE27A30FBE1FAC91A0300895ABE00A9F5A
:10E24200F001E15FFB4F0895EA0FFB1F0F01AC8164
:10E25200BD8159CCA5E10A9FF001E551FB4F08951C
:10E26200EE81FF8101801280AE81BF8115960E94EE
:10E272004975D0010895FE013896FA93EA930895FC
:10E28200EAA5FBA5FA93EA930895FA93EA93FE01AD
:10E292003A96FA93EA930E94816330E0E02F089560
:10E2A200E091BC05F091BD050895ACEBB5E0ED91B0
:10E2B200FD913296FE93EE930895AE81BF81EA17E7
:10E2C200FB070895E0E0E0936005E093610508959F
:10E2D200E7E1EA93E1E0EA930C941E48EA93E7E768
:10E2E200EA930C941E48E0935805F093590508955B
:10E2F200AAE4B6E0F0E0C4C8EA93ED85EA930C9490
:10E302001E48E985FA85AD85BE850895EA930E9487
:10E312001E48E8E10895EA93E0E0EA930C941E486F
:10E32200EA93EC85EA930E941E480C943848E881EF
:10E33200F981FA93EA930E948B59ECE2EA930C94E6
:10E342005A59A091160BB091170BEC910895A09118
:10E35200140BB091150B0895EE81FF81E093DE0B53
:10E36200F093DF0B1093DB0B0E94F733E1E3089588
:10E3720041E050E00E949B58E887F987EAE3EA937C
:10E382000E940B58E13008951A93E985FA85FA93B1
:10E39200EA935A934A930895E985FA85FA93EA93A0
:10E3A2000895E2E2EA930E940B58E0300895EAE30E
:10E3B200EA930C940B58FA93EA935A934A9308956A
:10E3C2000E949B583197E887F987E8850895E09184
:10E3D200F60AF0E0E65AF94F0895E0E0E093260CE1
:10E3E200E093270C08950E949B583197E093F60A18
:10E3F200E0910F0BA091F60AEA1708950E94754E5C
:10E40200E091F60AEA930895ECE2EA930E940B582F
:10E41200E0300895E650F54FA0E0A0830895EA9316
:10E422000E940B58E1300895E091F70A35CDE09152
:10E43200F70AEF5FE093F70A0895AAE5BBE0E091DF
:10E44200F70AF0E00C94416AE091F70AF0E00895CF
:10E45200E2E2EA930C945A59E091F60AF0E08ACC8F
:10E46200E091F60AF0E07ECCFA93EA930C948B5991
:10E47200FA93EA930C94CD4AEE27A10FBE1FEC91BA
:10E48200D001EC9308950E948B59ECE2EA930C942C
:10E492005A59ECE2EA930C945A590E94C24AE0E0BB
:10E4A200E093F70A0895AE0FBF1FEC91B5CCE0914F
:10E4B200160BF091170B0895A4E1BBE00C94EB68E6
:10E4C20046DFEC93F9CFA091160BB091170B08958C
:10E4D200E0E0EA930E94244BE093EB070895AA81BF
:10E4E200BB81EC91E295E07FAE2FEC810895EA0FBB
:10E4F200AA81BB81EC93B5CAE091C70CA091C60C6E
:10E50200EA170895E091920DF091930D0895A0916C
:10E51200900DB091910DEA17FB070895E12FA0919C
:10E52200970DEA0FE093970DE091990D0895F0E0B1
:10E53200E251F84F10830895E091990DF0E0EA500E
:10E54200F74F0895E0919E0EF0E0E356F24FE0811E
:10E55200E0939C00E0919E0EEF5FE0939E0E089583
:10E56200EA930E945A591F5F0895A981BA81EE2742
:10E57200A10FBE1FEC91E0300895E6EAFBE1FA93A9
:10E58200EA930895FE013196FA93EA930895E88199
:10E59200EA930C945A59E881F9816A817B810E943D
:10E5A2005C7508953A932A935A934A930895EA50D0
:10E5B200F64FE081E0300895EA930E94EA62EA931E
:10E5C2000C940E561A930A933A932A930895FA9347
:10E5D200EA93E09109040895A091F30BB091F40B32
:10E5E2000895E091F30BF091F40BFA93EA93E09122
:10E5F200F50BF091F60BFA93EA930895E093F30B7F
:10E60200F093F40B0895F801AA81BB81EA0FFB1F76
:10E61200E4910895AE0FBF1FAC91A0300895AE0FE4
:10E62200BF1FEC91EA930895A0910904E4E1EA9FE7
:10E63200F0012E2F3327D5CFECE0EA9FF001A09115
:10E642000804EA9FF00108951A93E1E0E0930904B7
:10E65200E093080410E00895ADE01A9FF0010C94D5
:10E66200F167EA9FF001F0E00895EAA5FBA5E20F49
:10E67200F31F0895ECA1EA930C9412493A932A935A
:10E68200EEA1FFA1E40FF51F0895FA93EA93EDCFEF
:10E69200FA93EA93EAA5FBA5E40FF51FFA93EA932E
:10E6A200E9CFFA93EA93E6CFEA9FF001AEA1BFA1C8
:10E6B200F0E00895E2E0E0930904E0E2F0E0EAA38A
:10E6C200FBA30895AE1BBF0B0C941E6AEE8DF0E007
:10E6D200E20FF31F08953196FA93EA93ECA1FDA19C
:10E6E200E40FF51F31960C94CF68FA93EA93ECA1EC
:10E6F200FDA1E40FF51F0C94CF68E9A1F0E0DE0163
:10E7020016960895ED8DEA930E94B75CE9A1EF5F3A
:10E71200E9A30895E40FF51FDF01ECA1FDA10C941C
:10E72200416A0E94A5740E9467740E94027608954D
:10E73200AE85BF85888999890895EE83FF836887AE
:10E74200798708950E9466750E9435760895E98D4D
:10E75200FA8DE21BF30BFA93EA930895FA93EA9384
:10E76200F901AD8DBE8DEA0FFB1FFA93EA9308956E
:10E77200FA93EA93EA8DEA930C941249EA930E947F
:10E782003961E0300895E0E0EA930C945E61EA9327
:10E792000E947B61E0300895E0917100E87F1E2FB6
:10E7A2000895E0937300E4E8F2CF0A930E94526165
:10E7B200E0300895FF27662777270E9402760895A2
:10E7C200EE8DB6DFF7DF0E948A76A9A1BAA188276B
:10E7D20099270E946375B6CF2A93ED89FE89FA9331
:10E7E200EA93FE017596FA93EA930C94DA63EE8942
:10E7F200FF893497EE8BFF8B0895ED89FE89FA939A
:10E80200EA93FE017596FA93EA930C94DA63AE8961
:10E81200BF8914960E944975EE83FF83E3CBE88596
:10E82200F9856A857B85AC85BD858E859F85089532
:10E832000E940166E883F9836A837B830895E881F5
:10E84200F9816A817B810895EA81FB816C817D81F6
:10E852000895E991F991309639F080ED97E00197AA
:10E86200F1F7A8953197C9F708950024AF0DB01DAF
:10E872000895EA0FFB1F681F791F0895F195E1952E
:10E88200F0400895F09560957095E195FF4F6F4FB8
:10E892007F4F0895EE230E2EEA2F19F0EE0F0A9401
:10E8A200E9F70895EE0FFF1FEE0FFF1FEE0FFF1F98
:10E8B200EE0FFF1F0895EF2FFF27E7FDFFEF0895EB
:10E8C200FE2FFF0FFF0B6F2F7F2F08956F2F660F05
:10E8D200660B762F0895BA2FBB0FBB0B8B2F9B2F86
:10E8E20008958B2F880F880B982F0895EA17FB073E
:10E8F200E1E00CF0EE270895FA9FF02DEB9FF00D6A
:10E90200EA9FE02DF10D08957A9F702D6B9F700D97
:10E91200F89F700DE99F700D6A9F602D710DFB9F2E
:10E92200600D711DE89F600D711D8827FA9FF02D03
:10E93200610D781FEB9FF00D611D781FEA9FE02D9E
:10E94200F10D681F781F089582D0D6DF0EF496DF8E
:10E9520008958BD0D9DF0EF495DF0895002498E056
:10E96200AA0F001C0E1A10F40E0E01C0A1609A9597
:10E97200B9F7EA2FA02D08950024112490E1AA0FDF
:10E98200BB1F001C111C0E1A1F0A18F40E0E1F1EAC
:10E9920001C0A1609A9599F7FD01D001089557D061
:10E9A200EBDF0EF46BDF08953F934F935F930024E8
:10E9B20011244427552730E2AA0FBB1F881F991F35
:10E9C200001C111C441F551F0E1A1F0A460B570B21
:10E9D20028F40E0E1F1E461F571F01C0A1603A9554
:10E9E20059F7FD01BC01D001CA015F914F913F91DE
:10E9F20008953BD0D9DF0EF445DF0895AFDFEA2F4B
:10EA02000895E894B7FF04C0A095B0951196689454
:10EA1200F7FD34DFB1DFFD010EF430DF0895C4DF0E
:10EA2200FD01BC010895E89497FF09C0A095B09537
:10EA320080959095AF5FBF4F8F4F9F4F689477FD42
:10EA420021DFB2DFFD01BC010EF41CDF0895E89462
:10EA5200F7FF02C013DF6894B7FF06C0A095B09518
:10EA6200119600F8039400FA0895E89477FF02C023
:10EA720009DF689497FF0BC00024A095B09580959C
:10EA820090951196801D901D00F8039400FA089548
:10EA9200ED91FC9111970895ED91FD916D917C910D
:10EAA20013970895ED93FD936D937C9308950590CC
:10EAB200F491E02D08957A936A93FA93EA93089574
:10EAC200689401C0E89401D09DD0182E862F612D44
:10EAD200192E972F712D1B2EBF2FF12D1A2EAE2F0F
:10EAE200E12D0895119602D0FE2F1197E199FECFE4
:10EAF200FF93FFB7F894AEBBBFBBE09AEDB3FFBF85
:10EB0200FF91089507D01196EF93EF2F03D0EF9165
:10EB120011970895E19B02C0A895FCCF9FB7F89486
:10EB2200AEBBBFBBE09A8DB3E81719F0EDBBE29A1A
:10EB3200E19A9FBF0895552342F4503811F4E0FF43
:10EB420004C03196691F791F6BF050E8572711F402
:10EB52005F93CDC05F3F31F0660F000C579567950C
:10EB6200752F08955F9300200AF0CDC0C6C050E80B
:10EB7200192E1522880F991F9527550F879550E852
:10EB8200072E0522660F771F7527550F6795089583
:10EB9200689401C0E8945F93F2DF703818F07F3F09
:10EBA20008F4A5C056E1571BAAF4519558300EF44B
:10EBB200593030F0EFEFFFEF6FEF7FE777F91AC0D0
:10EBC20077275523B9F0EE0FFF1F661F771F5A955F
:10EBD200D1F710C07727583028F0EF2FF62F672F84
:10EBE2005850F9CF552331F076956795F795E7950B
:10EBF2005A95D1F700200AF445DE5F910895689492
:10EC020001C0E894309760407040B1F0002426F0D3
:10EC1200772312F4009436DE172E7EE1112032F0B3
:10EC22007A95EE0FFF1F661F111CF9CFEF2FF62FFB
:10EC3200612D5F938ADF5F9108954F93AF01FD01CC
:10EC4200DA01AB01BC01CA01402D012C142E4F91F7
:10EC52000895EA0FFB1F681F0895E095F0956095EF
:10EC6200EF5FFF4F6F4F08955F9381DF903871F12F
:10EC720050E8152604C05F937ADF903839F1703876
:10EC820021F1572F591B13F112F4D7DFFACF583164
:10EC920018F0AA27BB278827583028F0AB2FB82FA7
:10ECA20088275850F9CF552329F08695B795A7950F
:10ECB2005A95D9F7502D512562F0CBDF38F467957C
:10ECC200F795E795739513F41EC0B7DF3EDF5F91AA
:10ECD2000895EA1BFB0B680B51F010F40094BDDFA2
:10ECE2006623A2F3EE0FFF1F661F7A95CBF7EE277E
:10ECF200FF27662777275F910895EFEFFFEF6FE712
:10ED02007FEF5F910895EFEFFFEF6FE77FE75F918E
:10ED120008955F932CDF703851F3903841F301244A
:10ED22000894791F23F41CF300203AF3ECCF0F92DE
:10ED32001F932F933F934F93112722279927689F61
:10ED4200A0018F9F302D410D591F6B9F300D411D2A
:10ED5200591F8E9F27D0BF9F25D06A9F23D0BE9F69
:10ED62001DD0AF9F1BD0AE9F110D291F391F491F08
:10ED7200591FE32FF42F652F522F4F913F912F915F
:10ED82001F910F9066232AF0550FEE1FFF1F661F7B
:10ED920002C073954BF2CFDE5F910895100D211DD5
:10EDA200391F02C0200D311D491F591F08955F935D
:10EDB200DEDE703821F411200AF49FCFA4CF903800
:10EDC20009F495CF01240894970B1BF4D4F3002087
:10EDD200F3CF792F1F932F933F934F931124112732
:10EDE200222733274427552790E2AE17BF0786070D
:10EDF200410730F0AE1BBF0B860B410B089401C0DC
:10EE02008894551F221F331F111CAA1FBB1F881F66
:10EE1200441F9A9551F7F901612D4F913F912F911E
:10EE22001F91662332F0550FEE1FFF1F661F7A9562
:10EE320043F281DE5F9108953097604070400895FB
:10EE420000240A160B06089500240A160B0608066B
:10EE5200090608955A934A933A932A931A930A9366
:10EE620008955D814C813B812A8119810881089531
:00000001FF
